:020000040800F2
:1000000000A0002039230108A59700087D140108ED
:10001000A3970008A19700089F9700080000000020
:100020000000000000000000000000009D97000894
:100030009B97000800000000999700084DB1000848
:10004000A1230108A1230108A1230108A12301087C
:10005000A1230108A1230108A1230108A12301086C
:10006000A1230108A1230108A1230108A12301085C
:10007000A123010825D70008C1E10008A123010838
:10008000A1230108A1230108A1230108A12301083C
:10009000D58F0008A1230108A1230108A12301088D
:1000A000A1230108D5DF00087BDF0008F9DF000885
:1000B000C9DF0008B9DF0008A9DF0008A123010893
:1000C000A1230108A1230108A1230108A1230108FC
:1000D000A1230108B9E10008B1E10008A12301084A
:1000E0005DB10008A1230108B90C0108A123010892
:1000F00089DF0008A123010899DF0008A123010876
:10010000000000000000000000000000A123010822
:10011000A1230108A1230108A1230108A1230108AB
:10012000A1230108A1230108A1230108A12301089B
:10013000A1230108A1230108000000000000000025
:10014000A1230108A1230108A12301080000000048
:10015000000000000000000000000000000000009F
:100160000000000000000000A1230108A1230108F5
:10017000A1230108000000000000000000000000B2
:0801800000000000A1230108AA
:100188002DE9F04F2DED028B754E764B3360AFB0F5
:10019800002373600FF054F818B90FF073F806F0E5
:1001A800DFFF07F097F8704B704C1A7842F00102A5
:1001B8001A706F4A4FF47001C2F888100022099231
:1001C8000A92226842F4803222600493236803F47E
:1001D80000330A93099B013309930A9B1BB9099BB6
:1001E800B3F5A04FF2D1236813F4003318BF0123ED
:1001F8000A930A9B012B00F089805D4F5D4BFB60E1
:10020800636AB360636ADFF8A4B1DFF8A481DFF83A
:10021800A49143F080736362636943F4FC032EADD9
:10022800636103238DF86A3041F6FF7325F8503D6A
:100238004FF0904029460DF067FB4FF6FF734E488C
:10024800ADF8683029460DF05FFB4C4829460DF0A3
:100258005BFB4B4829460DF057FB584629460DF0E5
:1002680053FB294647480DF04FFB284606F0E6F8B1
:100278001A9B454AB3FBF2F3444A1360444B454A80
:100288004FF0000AC3F800A0434B5A60F02287F8E9
:1002980023200722C3F808A0404F1A60D8F8083076
:1002A8003B6099E80F0085E80F0063691A9843F4EA
:1002B80000136361636943F4001363614FF4885367
:1002C800ABF828304FF48843ABF828301BA90DF061
:1002D8001BFB1DA91C980DF017FB64200AF0EBFD11
:1002E8004FF48C722E48514614F0D3F8E3692D4A26
:1002F80043F00703E361A36943F4C523A36163697A
:1003080043F4F013636102F1E00E55E0264B12222C
:100318001A606368636063686360636843F480635A
:100328006360636823F47C136360636843F4E813D1
:100338006360236843F08073236022680B4B92014B
:10034800FBD55A6822F003025A605A6842F002024A
:100358005A60636803F00C03082BFAD14DE700BF1D
:10036800900100200F6A0008D42B002000100240E2
:1003780000ED00E00005FA05000400480008004808
:10038800000C00480014004840420F00C014002030
:100398001C1500203F19010010E000E0E81F0020B4
:1003A80064150020C07D01080020024000100048AC
:1003B80048200020AC5D0108937B506892F80FC07C
:1003C80003F00701DB0800EB83038900186A4FF08C
:1003D8000F0A0CFA01FC0AFA01F120EA010119627C
:1003E800196A10324CEA010172451962E4D10022FF
:1003F80095490023535401320E2AF9D1DFF87CA223
:100408000AF11A02FF2199540133072BF6D18F4ABA
:100418008F4B1360DFF868B28E4A03930321117083
:1004280058460021242214F034F814228BF80020B6
:100438008949039B3F6801228BF8182098F805B07A
:1004480081F800B0A3F5EE71CAF824108349A3F52A
:100458008E730B60824B03EBCB035B78CAF82830B2
:10046800BB0648BFCAF8282000237E4A40F2DC5168
:1004780022F813100133082BF7D113A800211C22EE
:1004880014F007F8BBF10E0F03D00BF0EF03082BA5
:1004980002D101238DF85C3002200AF0DBFB18B191
:1004A8004088003018BF0120C7F340038DF8523050
:1004B800C7F380138DF85430C7F340338DF84C30B0
:1004C800C7F3C03300F001008DF84F3017F4006314
:1004D8008DF8510007D098F8863103F1FF3EDEF120
:1004E800000343EB0E038DF85030C7F300438DF83B
:1004F8005530B36AB8F84801ADF86000003318BF4A
:1005080001238DF85630C7F300538DF85730B8F8EB
:100518004A31ADF85A30F804B8F8563148BF524855
:10052800ADF85830C7F380438DF85330B8F85431DC
:1005380044BFB0F85001ADF86000B3F5FA7FADF8EC
:100548005E3084BF0023ADF86030484898F8D63153
:1005580086F82C30002386F82D3043709DF85C30E7
:1005680007F00101002BC7F3C0028DF84D108DF87C
:100578004E200CBF0023022301B902B1013309EB5D
:1005880083094FF0000AD9F810309A1E1A330392E3
:100598000593039A32F8023F03924FF6FF72934293
:1005A80000F072819DF855004FEA132EDAB25FFA17
:1005B8008EF330B110012E4F3F582E48874200F07D
:1005C8005E819DF8520050B1294F2B4807EB021766
:1005D8007968814203D13889012800F050819DF85B
:1005E8004F0050B1224F244807EB02177968814227
:1005F80003D13889042800F042819DF8500050B199
:100608001B4F1D4807EB02177968814203D13889CF
:10061800022800F03481BEF1020F02D19DF84C107F
:1006280004E0BEF1010F04D19DF84D10002900F03F
:1006380026819DF8561051B39DF85C1039BB9DF882
:100648005410F9B1111F1FE09C0100205012002026
:10065800382200209D10002010090020F8160020E4
:10066800988301081010002048200020BD010020B8
:10067800C07D0108004401400008004890010020A6
:1006880054120020A2F10801012998BF0423CA4F7F
:100698009DF857104FEA02194F4431B19DF85C108C
:1006A80019B9043A032A40F2D380012B4AD1C24A2D
:1006B800DFF81083079202EB0901FF2391F80DE0A0
:1006C80088F8743088F875304868C8F8847001F183
:1006D80008030989ADF868104FF0000B02218DF866
:1006E8006B1088F878B01AA98DF86AE0069388F834
:1006F80030B0C8F834B0C8F838B0C8F83CB0C8F85A
:1007080070B088F876B088F877B00DF0FDF8069BE1
:10071800079A997852F809005A460CF00DF93846AC
:100728000FF07CF9A54BC8F88830A54BC8F88C3079
:10073800C8F890B0384608F1880108F18C020DF02D
:10074800D9FC9CE0022B49D15FFA8AF21C2101FBFB
:1007580002FC9C4ACDF81CC002EB0C08964A88F8AB
:1007680079A0012188F8781002EB09014FF0000BFD
:1007780091F80DE0486888F87AB001F10802098913
:10078800ADF8681088F882B01AA9C8F884708DF896
:100798006AE006928DF86B300DF0B6F8864B069A33
:1007A80053F8090091785A460CF0C6F838460FF00D
:1007B80035F9844BDDF81CC0834AC8F8882003EB60
:1007C8000C01824AC8F88C208831C8F890B03846A5
:1007D8000A1D0DF08FFC0AF1010A50E0032B35D1F8
:1007E8009DF85330DFF8DC81DFF818923BB198F8B8
:1007F8002EB0384608214FF6FF7200231AE0BDF8E4
:100808005E2098F82EB0BDF86030B2F5FA7F0BD9AB
:100818006F49B1FBF2F23846082192B20DF09DF80B
:100828006C4B49F82B000AE06B49B1FBF2F23846F1
:10083800012192B20DF091F8684B49F82B00C36082
:1008480098F82E30013388F82E3018E0042B16D192
:1008580096F82D80BDF858205F4B93FBF2F238468E
:10086800BDF85A30012192B20DF077F896F82D3084
:1008780006EB88080133C8F8580186F82D30039B29
:10088800059A93427FF485AE96F82D2086F8782154
:10089800534A544B92F800E0AEF117020027022A9F
:1008A8001F709C461AD8736A3B44D3ED007AF5EE64
:1008B800407AF1EE10FA02D1B36A63BB26E04A4AE5
:1008C80007EB02080FCB88E80F009CF800301037C0
:1008D8000133C02F8CF80030E5D1EDE7434B13F816
:1008E8003E908CF8009003EBCE03D3F804A0BAF145
:1008F800000FE1D04F45DFDA3B4A3B0103EB02082A
:1009080053440FCB013788E80F00F3E7384E3368BC
:10091800DF0424D41DE0374B374A13F83E0010702B
:1009280003EBCE035E68002EF0D000238342EDDA9D
:10093800C3EBC3017218DFF8D080D2F8009041F8F9
:10094800089001EB08079188B9809279BA71013350
:10095800ECE70EF0EF03082B284B20D122E09CF89F
:100968000020012AF5D9264B03EB0212103210336E
:100978009342EED053ED047AB6EE007A67EE877AAA
:1009880043ED047A53ED057A67EE877A43ED057AED
:1009980053ED037A67EE877A43ED037AE7E7BEF112
:1009A8000E0F33D11A7842F010021A70BEF1180FE8
:1009B80033D10AF019FE30E0C07D0108BDC300083C
:1009C8009DC40008900100203DCA000895C3000896
:1009D80000127A00BDC4000840420F00ADC40008F0
:1009E80010090020601500204C0800209883010899
:1009F800E81F0020C06C010884160020D4100020D5
:100A08005408002030150020851600201A7822F09E
:100A180010021A70BEF1190FCAE70AF0C9FD33684F
:100A2800DFF834B3580358BFBC4BBD485CBF012244
:100A38001A70049B049A1B7843F0040313706269CC
:100A48004FF408534FF002094FF0010A42F4001224
:100A5800ADF8683029468DF86AA08DF86B90626110
:100A68000CF052FFAF4AB049116000200AF07AFB3F
:100A7800A26942F48052A261E26842F48052E260C4
:100A880062694FF0904642F400326261326A22F4A1
:100A980070023262326A42F4A0023262326A22F092
:100AA80070623262326A42F0A0623262326A22F0C6
:100AB80070423262326A42F0A0423262326A22F4F2
:100AC80070223262326A42F4A022002732624FF06A
:100AD8000308E022304629461A928DF86C908DF86A
:100AE8006D808DF86E708DF86F7005F01DFE102208
:100AF800304629461A9205928DF86CA08DF86D80C3
:100B08008DF86E708DF86F7005F00EFEE168874EF7
:100B180041F48051E160E16821F48051E160844949
:100B2800888820F480500004000C8880888880B26F
:100B380040F480508880088800F4415040F44570A3
:100B480040EA08000880888820F470600004000CDF
:100B580040F4E0608880888B20F40060000407235C
:100B6800000C88830B82088880B240F0400008801F
:100B780070490E60616941F480216161E16941F465
:100B88000011E161216B21F010012163216B41F01B
:100B980010012163DBF8201021F07061CBF82010E0
:100BA800DBF8201041F08061CBF82010DBF8201032
:100BB80021F07041CBF82010DBF8201041F0804183
:100BC800CBF82010402158461A9129468DF86E70AE
:100BD8008DF86F708DF86C908DF86D8005F0A4FD20
:100BE800802158461A91294605F09EFD3168524BDE
:100BF800059A21F0010131603068504901403160A7
:100C08004F493161316841EA0A013160B760F760E4
:100C1800B760B16841F40041B16031683160716812
:100C280021F0784121F400417160316841EA0A01FC
:100C380031601D68434E0493304605F4006339461D
:100C4800039305F4004B13F024FC049B8DF83D90AE
:100C580015EA09058DF83E708DF83F708DF83C80D7
:100C680005930DD03848CDF838A00EA905F05CFDE5
:100C78000622072332707770F37086F802A0554673
:100C8800BBF1000F0ED004232F480E930EA905F0D8
:100C98004BFD082333710723F371012375711D443C
:100CA800B371EDB2039B6BB1022327480E930EA9D3
:100CB80005F03AFD07233373F373012375731D445D
:100CC800B373EDB20EA908231F480E9305F02CFD4F
:100CD8000923337207237572F3720123B3721D441B
:100CE800E36A1A4823F4F873E362E36A43F4D873B7
:100CF800E362636943F0805343F00103636105F0E5
:100D0800E6FA1AA805F0B8FA114B1A93EDB2114B8E
:100D18001B93012D4FF0000320E000BF780D002049
:100D280000100048E02B002035AC000800540040BB
:100D380000300140DC0F0020E81F0020FFE0CF005A
:100D48007A25E000A81200200008004808000240A8
:100D580040000050B8120020000400480CBF1A469A
:100D680080221F924FF48072BD4C20924FF4806213
:100D780021922022204622921AA94FF400521C9355
:100D88001E9323922493ADF8745005F082FA2368D9
:100D980043F0010323604FF0A0440A20A36823F026
:100DA8004053A360A36843F08053A3600AF083F81C
:100DB800A36823F08043A360A368A360A36843F0FB
:100DC8000043A3604FF0A0418B68002BFADB8B68CF
:100DD800A44A23F040538B608B6843F000538B6028
:100DE8009068A14B034043F468339360CA689F4BF3
:100DF800134043F40053CB600A6B013D22F00F020D
:100E080015430D63002401233219917800296CD011
:100E18005D1C042B375DD078EDB24FF0A04E0ED894
:100E280003EB43035A00DEF830101F23934021EAF6
:100E3800030107FA02F30B43CEF8303031E0092BF7
:100E48000ED8053B06225A43DEF834101F23934080
:100E580021EA030107FA02F30B43CEF8343020E00D
:100E68000E2B4FF006010ED8A3F10A024A43DEF812
:100E780038C01F2393402CEA030107FA02F30B43FF
:100E8800CEF838300DE00F3B01FB03F2DEF83CC032
:100E98001F2393402CEA030107FA02F30B43CEF811
:100EA8003C30092F4FF0A0420FD99369A7F10A03EC
:100EB80003EB430397690721994027EA01019161F0
:100EC80091699840084390610EE053697B1E03EBDB
:100ED800430357693821994027EA01015161516953
:100EE80003339840084350612B460434102C8BD1AF
:100EF8004FF0A042936843F0010393604FF0A04382
:100F08001A68D107FAD5DA68594C22F00202DA6079
:100F1800DA6842F00202DA60DA6842F00102DA6066
:100F28009A6842F004029A60B4F85C31002B40F0F1
:100F3800DB85B4F95E21002A40F0D685B4F960213A
:100F4800002A40F0D185B4F864310393494B4A4EE6
:100F58001B684A48B3F85630049300210C2294F8D1
:100F6800635194F86B71B4F80CA094F80FB013F0B7
:100F780090FA00211422304613F08BFA404B33606C
:100F8800404B41497360414B414A42483361022317
:100F98000B70052313700368069143F00103036087
:100FA80091463D4A0023092D137001D91D46F8E7E3
:100FB800012202FA05F140F2BA330B40002B40F04F
:100FC800878511F0450F00F08385192027211AAB7A
:100FD8000CF0B0FD002800F07B85284B2F4A1A60E2
:100FE8002F4A5A602B4A062389F80130136843F0C8
:100FF80002031360274D2B689A0702D51F4B1B6805
:101008009847DFF8A4802749BBF1000F4ED09DF820
:101018000C3013F0FF0F0AD12B6813F0020F4FF0BA
:101028007D0240F2712308BF4FF4FA7302E04FF4D7
:101038007A731A469A4505DBBAF57A6FA8BF4FF45A
:101048007A6A00E09A46531E5344B3FBF2F3013B1D
:10105800DBB203FB022288F879310A602AE000BF7C
:101068000800024000030050E010FCFF07C0FFFD2D
:1010780048200020201000203C280020B41F002019
:1010880043DE0008798F0008FA0D0020295C8F3DA7
:1010980018010020D0100020FA2B00208D8D0008A8
:1010A800398D0008782800209001002088F879B14F
:1010B800C1F800A0336898472B4A0023137017B172
:1010C800022F40F00B854FF0000A1E200A21012252
:1010D8001AAB8DF868A0C8F87CA10CF02BFD88B17C
:1010E8009DF86830482B40F02785204B204A1A602D
:1010F800204A5A60022389F803302B6843F008031A
:101108002B6002E0824600F017BD94F858310BB10D
:10111800069A137094F859310BB1174A137094F862
:101128005A310BB1104A13702B68144913F0080F89
:1011380028D0BDF91000DFED126A642290FBF2F3AB
:1011480002FB130212B207EE902AB8EEE77A07EE16
:10115800903AF8EEE77AE7EE267AB2EE047A67EE8E
:10116800877AC1ED007A0FE0FB2B00209006002063
:10117800CD8D0008A58C0008FA2B0020041700204C
:101188008988883C00230B60B34F3B7843F0020307
:101198003B70B24B4FF488429A614FF488521A85DB
:1011A8004FF00A0ADFF8B492B9F814309BB283F40E
:1011B8008843A9F81430B9F814309BB283F48853E3
:1011C800A9F81430192009F076FE012009F0CAFFA9
:1011D800192009F070FE0AF1FF3A002009F0C2FF59
:1011E8001AF0FF0ADED14FF48853A9F828302B688B
:1011F8004FF4884A1B07A9F828A009D5984BC9F8C5
:1012080018A01B689847974BA9F828A001221A70C4
:10121800954B9FED968A1B68DFF894921B7B00EE36
:10122800103AB8EEC00A20EE080A05F0A3FEB9F895
:10123800003007EE903AF8EEE77A27EE800A13F0CE
:1012480037FB8B4B9FED8B7A1880B9F8003007EE8F
:10125800903AF8EEE77A884BC7EE277AFF211A22F0
:101268009FED867AC7EE877A9FED857AC8ED607A1A
:10127800D6ED047A834E67EE887A304667EE877A31
:10128800C3ED007A13F005F9002232702A687E4B0C
:10129800012112F0020F19701FBF7170032119701C
:1012A800022118BFB1703046560741BF19784D1C4E
:1012B8001D70032548BF455412F00A0F0CD01A7848
:1012C80004218154511CC9B205254554D11C023250
:1012D800D2B2197006218154059A11688D0641BF52
:1012E8001A78551C1D70072548BF85540A0608D56D
:1012F8001A7809258554951C0132D2B21D700A2529
:1013080085546579082D01D00E2D04D11A78561C04
:101318001E700B2686541A7811F4803F4FF00C0E7D
:1013280000F802E002F101061CBFDFF85CE10232BE
:10133800F6B21E701FBF8EF80020524A4FF00E0EF4
:1013480002F806E04A0741BF1A78561C1E7010269C
:1013580048BF86541A78561CF6B24FF0120E11F494
:10136800806F1E7000F802E00ED094F80CE2BEF117
:10137800000F09D0DFF810E102328EF80020414A50
:101388004FF0130E02F806E01A7811F4007F4FF0C0
:10139800140E00F802E002F101061CBFDFF8E8E0D5
:1013A8000232F6B21E701FBF8EF80020354A4FF089
:1013B800150E02F806E0182D0DD11A781626865457
:1013C800561CF6B24FF0170E00F806E0D61C023293
:1013D800D2B21E7085540D0341BF1A78511C197082
:1013E800192348BF835400219822284813F051F844
:1013F80004F0AFFC264B274A27491A6000234B808C
:101408000B7126490A60B4F8982190B2244921F852
:1014180013000133122BF9D1224E3368D8045CBF74
:10142800B4F89E0108801B0740F1F8801E4B93F822
:101438009231062B00F2EC80DFE803F004073E6DE2
:1014480088A7A70045F2F05201E042F6F822174BB0
:101458001A8004F034FDDAE0D42B00200010004894
:1014680090060020A80600205C07002035FA8E3C74
:10147800780700200AE81C415807002000401C4655
:10148800BD378635E90F0020E80F0020AC11002099
:10149800B40E0020D2210020040E0020C42B00200E
:1014A80024200020E81F002048200020C807002032
:1014B80012000020CDCCCC3F07EE902A5FED036AE6
:1014C8007C4BB8EEE77ADFED7C7AE7EE267A42F6D7
:1014D800F82119800023FCEEE77A784A17EE901A73
:1014E80042F823100133122BF7D1754A7549116060
:1014F800754A4020137009F0EDFB002800F0888041
:1015080001234FF0070990F90000704A8DE808029E
:1015180040216F4B76E0674B42F6F8221A80684B01
:101528006C4A1A60684B102240201A7009F0D2FBEE
:1015380000286DD001234FF0000C90F90000664A96
:101548008DE8081040214FF4E1335BE0594B42F637
:10155800F8221A805A4B614A1A605B4B08224020D5
:101568001A7009F0B7FB002852D001234FF0000E83
:1015780090F900005A4A8DE8084040214FF4E133C1
:1015880009F0A3FCC8F884013EE04A4ADFF88891D4
:10159800DFF888C1DFF888E1524D534C534842F6D2
:1015A800F821118048490C22062B0A700ED000231E
:1015B80089F800308CF800308EF800301B232B702F
:1015C8000523227003704FF4E1340BE0002189F801
:1015D80000108CF800108EF8001022702121444C65
:1015E80029700370364B434A1A60402009F072FB99
:1015F80070B101230025404A90F9000040218DE890
:101608002800234609F061FC003018BF012028B9E2
:10161800082005F073FD2A4B384A1A6033682A4AB5
:1016280013F4804F1FBF082111702549344818BF93
:10163800086042F20101194003F0010003F400546C
:1016480079B11C4944F620650D8024B10821117038
:101658001B492C4C0C6020B10C21117018492A48E8
:101668000860117804395170190640F192800025FC
:10167800264CDFF8B090C8F88891294615222448EE
:10168800DFF8A48065706560A56012F002FFA9F11B
:1016980005032846C8F800300AF0CEFC1D4B02208E
:1016A8001B68E36009F016FB00283FD1802005F095
:1016B80025FD66E0C80700200000B0C4CC2A002041
:1016C80018000020CD0D010848120020491001081B
:1016D800A0860100B90D01089D0F0108A10D0108A0
:1016E800510F0108362B0020592A0020372B0020E3
:1016F80090D00300C90C0108310E01082D0E010815
:10170800010E01081D0E01080D0E0108AC0600208F
:101718001C0300200C2000205A2A0020352B002012
:10172800342B002038220020CC060020637845792D
:10173800C3490C2202FB03125278AA4204D0013397
:10174800DBB2042BF4D900236370D8F80030627838
:101758001B7890F90000002B4FF00C0303FB0213D9
:1017680014BF0325012500225B7800950192022110
:1017780009F0ABFBB34B1860002897D001200AF0A2
:101788005BFCB14B1868B14B00F5C5721A600AF0E2
:1017980001FDAF4AAF4B1360AF4AB04D80331360C1
:1017A80033680024DA032C7040F1AD800CF096FD0C
:1017B800DFF810C3DFF81093CDF810C040F22A3BD1
:1017C8004FF00108604621465A4685F8008012F01D
:1017D80060FED9F81430A248A24D43F48023C9F81A
:1017E8001430436A23F00F034362436A43EA080351
:1017F8004362022203234FF4807A0CA98DF8342027
:1018080003928DF835308DF83640CDF830A08DF83C
:10181800378004F089FFD9F81830039A43F400336D
:10182800C9F818302B8823F440731B041B0C2B8039
:101838001D23EB620EA92A8560232C862846C5F84D
:1018480014800E93ADF83E401094ADF84440ADF8C6
:101858004640ADF84840ADF84A40ADF83C8004F049
:10186800AFFDAB6943F00803AB616B6C43F4004315
:101878006B64D9F8143043EA0803C9F81430A9F5A1
:101888007D69484604F023FD1AA804F0F5FC764B60
:101898001A9310231C938023DDF810C01F931AA9F4
:1018A8004FF400534846CDF86CC02393ADF874B09C
:1018B8001E94CDF880A021942294249404F0E9FC8D
:1018C800EB6843F40073EB60D9F8003043F002038F
:1018D800C9F800300BA80D238DF82C308DF82D8019
:1018E8008DF82E408DF82F800EF07AF821465F4B48
:1018F8001A685F4B43F8212001312029F7D10BF0FA
:1019080025FF0BF023FF33685B0556D5594D5A4B1D
:10191800D5F8CC84C3F80080042009F0DBF9042151
:10192800C5F8D00409F0B2F9544B85F8D40408205E
:10193800C3F8008009F0CEF9514B524C18600821C9
:1019480009F0A4F9002185F8D5042C22204612F0CC
:10195800A0FD8E2363704FF07C0AE0234FF07D09D1
:10196800E37084F800A084F82B90474C2C220021C7
:10197800204612F08EFD8A2363701020A023E370A6
:1019880084F800A084F82B90C5F8D88409F0A2F94F
:101998001021C5F8DC0409F079F985F8E004202065
:1019A800C5F8E48409F096F92021C5F8E80409F09F
:1019B8006DF985F8EC040FF05DFC3368334A13F4D5
:1019C800002318BF0123137009F04EFA304B18603A
:1019D800304B5A79052A194602BF2F4B4FF4C8726B
:1019E8001A802E4B4FF47A721A802D4A137843F0DE
:1019F800080313702B4A137823F00203137032681C
:101A080040F6020313406BB1274B284A1A60284B53
:101A180003221A70274B01221A70274A00231380C9
:101A2800264A13808B683360254B01221A703B7855
:101A380063F07F033B702FB0BDEC028BBDE8F08FE5
:101A48003C5E0108E01C002020100020100F002040
:101A58008013002064220020181D0020790D00202A
:101A6800000400480044014034440140CC5D0108B2
:101A78007A0D002090010020C41000201C110020C5
:101A880068110020EC10002021110020742800208B
:101A9800A807002048200020C60E0020F42B0020B4
:101AA800D4100020FD2B0020BC100020C4210020F1
:101AB8002011002010010020B00F0020B20F0020DC
:101AC800780D0020310300200010024035FA8E3CCA
:101AD800012D7FF68FAA0025FFF763BA012F7FF645
:101AE80014AB1F46FFF7E8BA1BB207EE903A5FED5A
:101AF800096AB4F95E31154AF8EEE77A07EE103A4A
:101B080067EEA67AB4F96031CDED1A7A07EE903A0D
:101B1800B8EEC77AF8EEE77A002127EE267A67EE64
:101B2800A67A11701AA80A498DED1B7ACDED1C7A98
:101B380005F028FAFFF707BA012F7FF6E6AA054B4A
:101B4800002783F800A0FFF7BEBA00BF7C00002082
:101B580084120020FB2B0020874A2DE9F04F1368E0
:101B6800864C03F59C4320332DED028B2360A3881C
:101B78000133A380824B196889B011F4804F059214
:101B8800019305D10FF0C4FA10B9237B01332373F5
:101B980000277C4BDFF804821E78FDB2AE4230D9B4
:101BA800D8F800307748072D98BF595D764B88BF25
:101BB80029461B689847032D1ED8D8F8002005F140
:101BC8000E0302EB83039988DA88A8B14FF47A737D
:101BD800401A5843531A90FBF3F040F6C90300F536
:101BE8007A70984205DC40F2EE239842B8BF184656
:101BF80001E040F6CA0080B204EB45050137E881F0
:101C0800C7E70F23277B84F83230032594F8333055
:101C1800B7FBF5F505EB45057D1B029394F83430C9
:101C28000393D8F800A0DFF87CB1EBB20493002549
:101C3800B54255DA5549029B31F815904FEA4508E7
:101C480053B90FF065FA28B1039B002B08BF4FF07A
:101C5800000901E0DDF80890BAF81400484503D8F7
:101C6800BAF8160048450ED2E8B20FF027FA032D4D
:101C78008146DFBF94F832E00120A8402EEA000038
:101C8800D8BF84F832000FF043FA18B1404828F85A
:101C9800009021E0049B94F87E002BF8139028B95B
:101CA800022F15D93549012081F87E00BBF80210B2
:101CB800BBF800000844BBF804100844354980B25A
:101CC80028F8010000B2032190FBF1F080B200E097
:101CD80048462F4928F8010001350BF1060BA7E704
:101CE80094F83250254BA5F10F0EDEF1000545EBB7
:101CF8000E0584F898503DB19A8811B21429CCBFCA
:101D0800143A00229A800BE083F83350B54207DA80
:101D1800E8B20FF0D3F91E4B23F815000135F5E7AB
:101D2800019B1B68DF0405D51B4B1B68DE0701D42C
:101D38000EF023FE059B1968184B1868837A9BB32D
:101D4800013B134D027B35F813301AB1C3F53B63E1
:101D580008339BB21BB2A3F57A73B3F57A7FA8BF99
:101D68004FF47A7323EAE37307EE903A9FED0C7A07
:101D7800F8EEE77A51E000BFDC2B0020000E0020CF
:101D8800E81F002048120020180000200E0E002036
:101D980024200020800E0020E40F0020C42B002007
:101DA80000007A44360E0020019A1268150440D5C6
:101DB800D4F89C20AD4E8A1A002A3ADB01F59C42E1
:101DC8002032C6F89C20AA4AC07A5579A94A32F826
:101DD800152096F8A050013592B292FBF0F205F06A
:101DE8000F0086F8A000304480F8A1201A46A248C7
:101DF800185C01330244102B92B2F8D112B292FB54
:101E0800F3F31BB2642BA8BF642323EAE37307EE42
:101E1800903A9FED9A7AF8EEE77AC7EE877A984A71
:101E28009FED987A67EE877AFCEEE77A17EE903A9C
:101E38001380019B944D1B68DFF8708213F4807F38
:101E48007AD0924B994204D9237A13B9874B01224D
:101E58001A72B4F904E098F80060844BBEF1140FCC
:101E6800CCBF4FF0000E4FF0010EC6F38006BEF156
:101E7800000F03D000279F725F7200E00327A07A4B
:101E8800D4F8B4B0D4F8B8C0B4F90490617AE3884F
:101E98002A88032848D8DFE800F0020E1B35BEF177
:101EA800000F02D02A8000222AE0002E40F0688627
:101EB8002A80A6723AE09CF8000000EB8000814579
:101EC80002DC2A8001221BE001206EB300F0BCBEB8
:101ED8003EB1BBF80E206A80AA80BCF80200E880F8
:101EE80002279CF800A09CF80100504400EB8000F9
:101EF800814500F34886002E00F045862A8002229C
:101F0800A27213E02A800322A2726172E3807EB17A
:101F180098F8003043F0020388F80030534B002251
:101F28005A720EF02AFD03E02A80A0726172E380E3
:101F380017B1384609F034F9554EB6F852010DF08C
:101F4800C3FF834668B90EF085FB524BC3F800B057
:101F5800C3F804B0C3F808B04F4B00221A605A60A7
:101F68009A6098F800305A0736D5019B1B68DB0643
:101F780032D54A4B1B78DF062ED4494B1B7893B1D8
:101F880096F8DE31BBF1000F15D17BB1454B1A68CD
:101F9800D4F8BC309B1A002B08DA0EF0EEFC334B59
:101FA80083F8C0B018E0BBF1000F0DD1102009F084
:101FB800F7F801230EE03BB13A4A12684FF47A7100
:101FC80001FB0323C4F8BC3094F8C03023B109F0F6
:101FD800CFF8002384F8C030002396F8DCA196F8E7
:101FE800DD11B6F89A71B6F89CE1184635F9132058
:101FF8008008BA42C4BF60F07F00C0B201337245A6
:10200800B8BF40F04000042BF0D194F8C130174A13
:10201800834205D192F8C230F92B04D8013300E08D
:10202800002382F8C2301E4A84F8C10010780F4B92
:102038001D4F914600283ED13A68D00709D5BBF11B
:10204800000F38D198F80030D90734D50EF010FBBE
:1020580031E098F8002052072DD593F8332052B379
:102068005B7A43BB21B30EF088FC24E0000E00200D
:10207800A8120020B8120020A10E00200000C842BB
:102088003C10002000C07F4424200020404B4C001E
:1020980048200020B01300206C140020D410002029
:1020A800100000200C200020E40F0020FD2B002051
:1020B800BBF1000FD7D094F8C230B64ADFF800B3AE
:1020C800142B40F08C8099F800301AF1000A18BFE0
:1020D8004FF0010A7BB392F8C1305F2B12D198F808
:1020E800003003F0040303F0FF0113B10EF045FCC8
:1020F80008E00B200391029209F052F8029A039922
:1021080082F8C210BAF1000F15D094F8C1307D2BB7
:1021180011D198F8003003F0040303F0FF0213B163
:102128000EF02BFC07E00B20029209F039F8994BCE
:10213800029A83F8C22098F8003003F0040303F0F1
:10214800FF01002B4BD194F8C130924A572B11D183
:10215800914B4FF47A721A80019B1B681B0601D5BC
:102168000AF07AF88D4B1B6813F0080337D18C4AB4
:10217800138034E001980068400717D55A2B15D111
:1021880092F8C3302BB1012382F8C31082F8C4300F
:1021980025E092F8C53083F0010382F8C5300BB111
:1021A8000C2000E00D2008F0FBFF18E05D2B00F08C
:1021B80020855B2B00F01F855E2B00F01E85562BBB
:1021C80001D105F017FA99F80030002B00F0E484EB
:1021D80094F8C1306F2B40F0D9840EF049FA019B76
:1021E8001B68580737D594F8C5306A4A93B198F8F0
:1021F800003059070ED5B5F90610B6F89A3199424C
:1022080008DD3B6813F0010302BF3221A2F8C810B1
:1022180082F8C5303B68DA030DD594F8CA205D4BC7
:102228002AB993F8C32012B93222A3F8C82001238F
:1022380084F8CA300FE094F8C330564A5BB198F876
:10224800003003F0040303F0FF0123B9012382F8EF
:10225800C31082F8C430DBF8009000233B6009F11A
:102268007B0609F1CB0A3278737816F8010C9A428A
:102278000BD2314608F098FD38B116F8022C01232C
:1022880003FA02F23B6813433B6004365645EAD131
:10229800444B1B7843B1444D404F2B68434E13F0D9
:1022A800020F40F035832DE309F1CA0609F5897755
:1022B8003278737816F8010C9A4225D2314608F024
:1022C80073FD08B3B37896F804E0394A96F803909A
:1022D80030480C21013B01FB0E4103EB430313443F
:1022E800D1F8D0209A420FD0C1F8D030002390F80E
:1022F800FC20C1F8D430012303FA0EF322EA0303C9
:1023080081F8CC9080F8FC300636BE42D0D1294BFB
:10231800DFF8B0B01E68284B1B68039394F833307D
:10232800049300230293DBF80030002B00F0E182D5
:1023380093F80090B9F1000F00F0DB82DBF804207D
:1023480003998A1A002A0CDB01F5FA720299CBF874
:10235800042001228A4094F8FC1021EA020284F841
:10236800FC20049A002A00F0C4821BF8042C597837
:102378000432D2B2002940F07E8235F912100F4A99
:10238800044FB2F8982102F1C800814222DD93F887
:1023980002A035E0000E0020F42B0020D010002011
:1023A800B0100020012C0020E40F0020981100201C
:1023B8001C620108401000200C200020482000204A
:1023C80020100020D00E00200000C84200000000AD
:1023D80000007A44C83A914203DA9978C1F1000AB8
:1023E8000EE0029A0123934097F8FC2022EA0303A7
:1023F80087F8FC30039B03F5FA73CBF8043078E2D6
:1024080097F8FC30029A1341DB0700F17282BAF1A7
:10241800000FCCBF0220012008F0E8FE09F1FF33CD
:10242800132B00F25D82DFE813F0140021002F0067
:1024380043005C006300CA002D019401C401F4014B
:102448005B02430052006300CA002D019A00FF009E
:10245800640137785744FA2FA8BFFA2727EAE777A5
:102468003046377008F086FC01200BE07778574437
:10247800642FA8BF642727EAE7773046777008F00B
:1024880079FC02203946C1E196F80390D144B9F1AC
:10249800640FA8BF4FF0640929EAE97986F8039028
:1024A8003046D7F8001108F01BFC03204946ADE17F
:1024B800717951446429A8BF642121EAE1717171DD
:1024C8000D2008F0BDFCB9F10D0F00F0098231793B
:1024D80051446429A8BF642121EAE17131710E20B9
:1024E80094E1B179514481F30801B17105208DE17E
:1024F800D7F804311A78022A22D107EE90AAF8EE0A
:10250800E77AB2EE040A87EE800AD3ED097A30EE54
:10251800270AB5EEC00AF1EE10FA09D45FED567A33
:10252800B4EE670AF1EE10FAC8BFB0EE670A01E030
:102538001FED5A0A83ED090A0F2008F06CFC0AE027
:1025480099785144C829A8BFC82121EAE171997036
:102558000F2008F075FCB9F10F0F00F0C181D7F812
:1025680004311A78022A20D107EE90AAB8EEE78A39
:10257800B2EE040A88EE008A93ED080A38EE000AE3
:10258800B5EEC00AF1EE10FA09D45FED717AB4EE37
:10259800670AF1EE10FAC8BFB0EE670A01E01FED56
:1025A800750A83ED080A122058E159785144C82960
:1025B800A8BFC82121EAE1715970122026E1D7F895
:1025C80004311A78022A20D107EE90AAB8EEE70A59
:1025D8005FED837A93ED0C7A80EE270A30EE070AD6
:1025E800B5EEC00AF1EE10FA07D4B4EE670AF1EEC0
:1025F80010FAC8BFB0EE670A01E01FED8C0A83ED40
:102608000C0A102008F007FC0AE0197B5144C8297D
:10261800A8BFC82121EAE1711973102008F010FC45
:10262800B9F1100F00F05C81D7F804311A78022A4A
:102638001ED107EE90AAB8EEE78A5FED9D7A93ED7A
:102648000B0A88EE278A38EE000AB5EEC00AF1EECA
:1026580010FA07D4B4EE670AF1EE10FAC8BFB0EE6C
:10266800670A01E01FEDA70A83ED0B0A1320F5E0C6
:10267800D97A5144C829A8BFC82121EAE171D97281
:102688001320C3E0D7F804311A78022A22D107EEC2
:1026980090AA1FEDB10AF8EEE77A87EE800AD3ED2B
:1026A8000F7A30EE270AB5EEC00AF1EE10FA09D417
:1026B8005FEDBB7AB4EE670AF1EE10FAC8BFB0EE70
:1026C800670A01E01FEDBF0A83ED0F0A112008F029
:1026D800A2FB0AE0997D5144C829A8BFC82121EA74
:1026E800E1719975112008F0ABFBB9F1110F00F0F9
:1026F800F780D7F804311A78022A20D107EE90AA79
:102708001FEDCD0AB8EEE78A88EE008A93ED0E0A2F
:1027180038EE000AB5EEC00AF1EE10FA09D4DFED82
:10272800BC7AB4EE670AF1EE10FAC8BFB0EE670AD9
:1027380001E09FEDB80A83ED0E0A14208EE0597D62
:102748005144C829A8BFC82121EAE171597514204C
:102758005CE0D7F804311A78022A20D107EE90AA53
:10276800B8EEE78AB2EE040A88EE008A93ED0A0A08
:1027780038EE000AB5EEC00AF1EE10FA09D4DFED22
:10278800A47AB4EE670AF1EE10FAC8BFB0EE670A91
:1027980001E09FEDA00A83ED0A0A09205EE0D978DE
:1027A8005144C829A8BFC82121EAE171D97009207C
:1027B8002CE0D7F804311A78022A1ED107EE90AA25
:1027C800B8EEE78ADFED927A93ED0D0A88EE278A54
:1027D80038EE000AB5EEC00AF1EE10FA07D4B4EEEE
:1027E800670AF1EE10FAC8BFB0EE670A01E09FED84
:1027F800890A83ED0D0A0A2030E0597B5144C82923
:10280800A8BFC82121EAE17159730A2008F018FB12
:1028180066E0D7F804311A78022A22D107EE90AA86
:102828009FED7D0AB8EEE78A88EE008A93ED100ADC
:1028380038EE000AB5EEC00AF1EE10FA09D4DFED61
:10284800747AB4EE670AF1EE10FAC8BFB0EE670A00
:1028580001E09FED700A83ED100A0B2008F0DBFA07
:102868003EE0D97D5144C829A8BFC82121EAE171B9
:10287800D9750B20CAE7012932D1987835F9123079
:10288800B3F5617F05DB40F633029342A8BF1346D8
:1028980001E04FF46173B9F10C0F21D14FF4966246
:1028A80092FBF0F05D4AA3F5617393FBF0F3DFB29E
:1028B8001378BB4214D0042F34BF3B460223137055
:1028C800574A09FB0323574A0633136004F0DEFC1A
:1028D8004846394608F0B4FA781CC0B208F086FCBD
:1028E8005149029A0123934091F8FC20134381F83F
:1028F800FC30029B0133042B02930BF10C0B7FF489
:1029080012ADC8E4019B1B68D8050ED5637A63B184
:102918003B68990709D5338813F001090AD10DF0EE
:1029280099FE012004F0DAFB04E0012004F0C5FB65
:10293800012300E000232A6852070CD55BB101206F
:1029480004F0BBFB3388980708D40DF083FE0220FF
:1029580004F0C4FB02E0022004F0AFFB3388334AE2
:1029680013F0030F4FF4884114BF916111853A6841
:1029780012F00A0F23D02A68D10609D55A070AD4BB
:10298800042004F0ABFB2A4B1B88A4F8083102E0B2
:10299800042004F092FB2B689B0606D53388580662
:1029A80006D4402004F09AFB02E0402004F085FBA6
:1029B8002B68590642BF1E4B1B88A4F80A313B6896
:1029C8009A0608D42B681B0540F1A6804FF4807046
:1029D80004F084FBA4E0174B1B789F0768D5164BBF
:1029E8001B78042B64D92B680F4F13F4007927D078
:1029F8003388DC0650D4102004F070FB202004F04B
:102A08005CFB0E48011D09F07BFB022340E000BF80
:102A18000000C8420000000000007A44941F002013
:102A2800E827002040100020000E00200010004879
:102A3800B0100020D4100020DA1000204810002028
:102A4800348804F01004A4B22CB1102004F035FB33
:102A5800012487F80C912B68580512D5D7F8103146
:102A680089495A89B1F90030002BB8BF5B429342BB
:102A780007DAB1F90230002BB8BF5B429342C0F2CB
:102A8800E9803388990608D5202004F016FB002336
:102A980087F80C31012400E0002497F81431B3B909
:102AA8000E2008F07DFB794B012283F814210EE0FB
:102AB800338803F03003002B84D0102004F0FDFA93
:102AC800202004F0FAFA002384F80C3102E0002CEC
:102AD8003FF478AF6E4B002003F1280603F1500451
:102AE8006C4A002122F810106B4A596022F8101025
:102AF8000432716022F8101000221A609A60326065
:102B0800B26022606160A260143314361434002865
:102B18007FF458AF0120E3E74FF4807004F0CDFA5A
:102B28005E4B5A79082A1C4601D00E2A02D1402051
:102B380004F0C3FA019B1B685A0540F1A08094F881
:102B48000C3223B998F8003013F0040F02E02B6818
:102B580013F4002F0BD0524B00221A703C2003F0C4
:102B6800F7F9002800F08B800CF08CF8F6E70EF0EF
:102B780081FB09B0BDEC028BBDE8F04F03F0E9B86A
:102B88000120FFF786B90320FFF783B9BAF1000FD8
:102B980002D07E2B3FF421AB94F8C130972B06D19D
:102BA8003A4B4FF4C872A3F8C620FFF718BBA72BFF
:102BB80006D13C4A137843F004031370FFF70FBBA8
:102BC8000022BB2B079201D1022303E0B72B04D1CB
:102BD8004FF6FE73ADF81E301FE0BE2B01D1022365
:102BE80004E0BD2B7FF4FBAA4FF6FE73ADF81C3052
:102BF80013E0012002E0022000E003205FFA80F9E0
:102C080009F1FF3386F8A43704F0AAFA04F062FB4E
:102C1800484608F0EBFAFFF7E2BADBF80030BDF8F7
:102C28001C10B3F858200A44A3F85820BDF81E1009
:102C3800B3F85A200A44A3F85A2004F0DBFC002316
:102C480084F8C230FFF7CBBA013301469BB20220A9
:102C5800FFF71FB933889B063FF51FAF202004F00C
:102C68003DFA1148114B011D1A685B684360026008
:102C780009F046FA054B012483F80C410DE709B029
:102C8800BDEC028BBDE8F08FB4100020000E0020D0
:102C9800180F0020F62B0020900F0020482000205D
:102CA8004D120020D410002050100020DC1000200D
:102CB8002DE9F04FC14BB3F90610C14B2DED028B36
:102CC8001F687A8989B0914201930EDBB1F5FA6FDA
:102CD800FC79BDBF8B1A6343A2F5FA64C4F164049E
:102CE800BCBF93FBF4F4643400E06424B54AB64BEB
:102CF800B2F898A192F962211868049092B20592EC
:102D0800054600220293AD4B33F912300393CAEB08
:102D1800030303F2F31640F2E63086424FEA420B11
:102D280003D8002BB8BF5B4201E04FF4FA73022AC4
:102D3800049E4FF064002FD096F811E1BEF1000F09
:102D480004D07345CCBFCEEB03030023DFF8C0E209
:102D580093FBF0FC6FF063093EF81C809B4E09FB67
:102D68000C390CF1010C3EF91CE00FFA88FCCCEB95
:102D78000E0E0EFB09FE9EFBF0FEC64426F80BE085
:102D8800BE1836797343924E93FBF6F364339BB2C5
:102D9800634393FBF0F02EE096F812E1BEF1000FCA
:102DA80004D07345CCBFCEEB03030023DFF84C827D
:102DB80093FBF0F06FF0630C0CFB003938F910E06E
:102DC8000130002B38F91000CEEB000000FB09F9A8
:102DD800BDF8140099FBFCF9CEEB090919FB00F9C1
:102DE8007A48A0F80490B879B8BF5B424343784862
:102DF80093FBF0F064306B78764E4FF0640E4343EB
:102E080093FBFEF3B354744EEB7A434393FBFEF308
:102E1800B3546B7D6D4E5843704B90FBFEF0022A05
:102E280098546F4B0FD183F802E0039B53450EDB98
:102E3800644CB4F89A21914215DBB1F5FA6FA8BF3A
:102E48004FF4FA6110E09C54039B534504DA36F8BA
:102E58000B305B4226F80B300132032A05F10105DD
:102E68007FF451AFE4E71146891A4FF47A73DFF81B
:102E7800A4E1564D59436FF06303C2F5FA62642723
:102E8800B1FBF2F191FBF7F23EF8120003FB0211DD
:102E9800013203B23EF91220D21A514391FBF7F3E3
:102EA8000344F3804F4B1B88580635D54E4B4F4A89
:102EB8001B881288DFED4E7A9B1A1BB208EE103A77
:102EC800B8EEC88A28EE278AB0EE480A04F052F80D
:102ED800F0EE408AB0EE480A03F0E9FFB5F9023097
:102EE80006EE903AB5F90030F8EEE66A07EE903A49
:102EF80020EE667AF8EEE77AA7EEA87A67EE807A8F
:102F0800BDEEC77AE6EEA87A17EE103AFDEEE77A3C
:102F18002B8017EE903A6B80364D2B68990740F15D
:102F2800A180354B354F1A687B6945F20721D31AC2
:102F38008B4240F397807A6103F0CEFC304BDFF888
:102F4800D8901A78032A9846B9F8003022D10A2B6B
:102F58002AD90023282088F8003007F0ACFF03F0B6
:102F6800BBFC284B18880EF093F8274B1A68D378C7
:102F780090FBF3F001300828244BA8BF08201870F4
:102F8800537980B213FB00F33B83137913FB00F0F2
:102F9800788309E00A2B07D803231C4A88F80030F5
:102FA800002313703B837B8398F80030144A012B6D
:102FB8003DD033D3022B4CD054E000BF2420002056
:102FC800401000204820002020100020B4100020CD
:102FD8000CFEFFFF2C140020A60F00204414002034
:102FE8009013002098110020B01000200A0F002034
:102FF80035FA8E3CE81F0020DC2B0020980F0020BB
:1030080020110020C0120020BC1000201001002058
:10301800B21400209A140020C01000203A8BB9F88E
:1030280000309A421EDD012388F800300FE0B9F81D
:1030380000107B8B8B4202DD022313700FE09E4B46
:103048001B8B0133994202DD002313700AE008202C
:1030580006E07B8BB9F8002001339A42E3DC0720B5
:1030680008F09EF82D682A0576D5944B924F1A6879
:10307800FB69C3EB020845F2072398456CDD904BCA
:10308800B6F906B0D3F80090FA6199F80A30B4F8A6
:1030980052018C4E012B4FF47A71ABF57A7B98FB79
:1030A800F1F803D041D3022B20D040E0864B386A98
:1030B8005A7B864B33F812204FF0080E92B290FBE1
:1030C800FEF3C01A8318BA843B6240F6E44293FBCD
:1030D800FEF39BB25343B9F80820C2EB13335943AC
:1030E800B9F9063091FBF3F1316020E0784BB9F87B
:1030F80008A01B78C6F800A05B0718D50CF0E4FE02
:1031080020B915F0100F18BF4FF0000B32220BFB3F
:103118000BF393FBF2F3B9F906205B445A434FF4DF
:103128007A7392FBF3F3534400E000233360D7E94A
:103138000A013368674A03FB08F84FF47A7398FB6F
:10314800F3F810EB080041EBE8710023C7E90A0126
:103158000EF0AAF9604B1860604E3368D90427D581
:103168002A0622D55E4B1B789B071ED55D4B187827
:1031780004281AD900225C4BD7180521951C4FF05A
:103188000A0E122AD154E9B287F801E004D0B0EB54
:10319800510F2A46EFD800E014215A18322002F8BD
:1031A800010CFF225A540F2000E00A2007F0F8FF14
:1031B8004E4D2A68002A50D04D4B4E4F186839683A
:1031C8008142984649D84C4BDFF8389119785268B3
:1031D800E1B94FF0010A83F800A0B9F80030D35CD8
:1031E80023B3504607F0BEFF444B83F800A00DF010
:1031F8009BFFB9F80030CBB92B681B78053B5345CA
:1032080014D807F031FE3E4B18600FE04FF0000A6B
:1032180083F800A0B9F80030D35C3BB1504607F002
:10322800A1FF364B83F800A00DF07EFF2A68B9F89D
:10323800003052683348D25CFE2A01D100230BE0EB
:10324800FF2A02D107F094FF07E0D8F800500A21BE
:1032580011FB02523A60013303801D4D2B785F0742
:1032680004D5294B4FF488529A6163E03268D0073D
:103278005CBF43F001032B70194B1B7819075EBF25
:103288002B7823F001032B70D30242BF2B7823F055
:1032980001032B701D4B1A88184B1AB11C4A12686F
:1032A800970702D41B4A1288B2B302221A702B78ED
:1032B80023F001032B7034E0980F0020DC2B002052
:1032C800BC100020C8100020A8120020B81200204E
:1032D800FD2B0020407E0500CC100020E40F0020CC
:1032E800D4100020DA100020C01F00202C15002068
:1032F8000C2000202415002020150020C82B0020B9
:103308000C2A00202815002000100048C60E0020B6
:10331800D0100020F42B00202978CE0758BF0222B5
:103328001A7007F0A1FDB04B1B68C01A002801DB1A
:103338000DF0FAFEAD4F0DF09DFF3E78002E00F027
:10334800AB80AB4B1A689846002A00F01B87D8F868
:10335800000007F0A6FF002800F01487A44BA54C36
:10336800186807F09BFF092801D03F2852D14FF079
:10337800000A2668DFF8B492554636B19E48D9F857
:103388000010324611F0D2F810B9CA4605B94D46B8
:103398009A4B09F110099945EFD3EDB1D5F800C062
:1033A800DAF8009023681CF803E019F80300704568
:1033B80012D15A1C904958B92D2B09D8DFF834E29C
:1033C800CEF800204FF0200E01F803E0885403E007
:1033D80001F803E02260E5E723680BB1554510D0FA
:1033E80087480BF049FD554507D855F8100B0BF0E9
:1033F80043FD09200BF038FDF5E782480BF03CFD52
:10340800002623689E42A2D27B4B985D0BF02CFDD0
:103418000136F6E72368002B40F09986042840F02F
:10342800D686754809F0D4FC00F0ACBED8F8000088
:10343800DFF8DCA107F035FF20B3DAF8000007F069
:103448002DFFDBF8003093F848100246A1BB242872
:103458006BD1012283F84820DBF80030DFF8D0A1D7
:1034680093F84820062AE1D193F8490000F042FF7A
:10347800834600287BD00BF053FCD9F8003000229B
:1034880083F84820604B93F83530002B40F04D8688
:103498004C36982E00F076865C4BF21892F84A105B
:1034A8000129F5D1DFF88891F358C9F80020584A66
:1034B800CB4613609046B9E7012904D14D2814BFC3
:1034C80000220222C6E7022904D13C2814BF0022A8
:1034D8000322BFE703290CD140284FF0000102D98D
:1034E80083F84810B8E758711971D9719871042296
:1034F800B0E7042906D1997983F849004A409A71BE
:103508000522A7E70529A7D158791979884298791A
:1035180006D950409871481C18710B441A729BE7E1
:1035280090420CBF0622002294E72B78590793D4C7
:103538002328DAF800300DD1012139702C49039085
:103548000B60314933480B630BF096FC2D480BF0A8
:1035580093FC039A304B1B681B78934201BF2F4B97
:103568002F4A1A602F4B04BF2F4ADA6074E7DAF843
:10357800002092F849304C2B00F0888400F28580B6
:10358800332B00F0DB8421D8292B00F04B8409D899
:10359800252B00F02284272B00F02684232B40F0D3
:1035A800128609E22D2B00F04E8407D82B2B40F011
:1035B8000A860BF087FB607100F0B2BD2F2B00F07C
:1035C8002A85312B00F03C8500F0FDBD3E2B00F034
:1035D800E58044D8372B00F0E5842BD8352B00F054
:1035E800268200F0F0BD00BFCC2B0020012C00206B
:1035F800B01F0020141D0020E41C0020006C0108EE
:10360800B6810108BB810108980F0020AC11002089
:103618007C110020EB81010850120020FC9F002043
:10362800EFBEADDE00ED00E00400FA05406A0108D7
:1036380078110020392B00F0E4833C2B40F0C3853F
:10364800DFF84C84D8F800A00BF03CFB8AF80000A7
:10365800D8F80030187808F063F800F061BD432B03
:1036680000F07D8406D8412B40F0AD854FF000086E
:1036780000F069BC442B00F018854A2B40F0A38564
:103688000BF02AFBA08100F04BBDD12B00F0668324
:103698001FD8CC2B00F00C820ED8C82B61D004D8D0
:1036A8004E2B00F01D8400F08EBDC92B00F02F8337
:1036B800CA2B7DD000F087BDCE2B00F01B83C0F055
:1036C8001083CF2B00F04882D02B00F0FF8200F04F
:1036D8007ABDD82B00F001810BD8D32B3BD027D350
:1036E800D42B00F07D82D62B40F06D854FF000087A
:1036F8006BE2F22B00F0C28212D8EF2B40F0638508
:10370800DFF88C83D8F800A00BF0E6FAAAF85A0084
:10371800D8F800800BF0E0FAA8F8580000F000BDD7
:10372800F32B00F0C784FA2B00F0ED8200F04BBDBC
:103738002B7803F0040303F0FF08002B40F0F0841B
:103748000BF0C0FA022884F8A40740F2C582CC4BDB
:1037580083F8A487C0E20BF0BFFACA4B188000F0C8
:10376800DFBC92F805804FEA5808B8F1120F03D968
:1037780002F0EAFB00F0D4BC4FF0000AC24507D2C1
:103788000BF0AAFAC04B23F81A000AF1010AF5E770
:10379800BE4B012283F8342000F0C2BC0BF092FA31
:1037A80084F8DE010BF08EFA84F8DD0100F0B8BC75
:1037B800B74B1A681278022A4FF0000A984670D15F
:1037C800D8F800B00BF07EFA07EE900AF8EE677AA8
:1037D800B2EE048AC7EE887A0BEB8A0BCBED087A37
:1037E800D8F800B00BF06EFA07EE900A9FEDA97AB0
:1037F800F8EE677A0BEB8A0BC7EE877ACBED0B7A7C
:10380800D8F800B00BF05EFA07EE900A9FEDA27AA6
:10381800F8EE677A0BEB8A0BC7EE877A0AF1010A92
:10382800BAF1030FCBED0E7ACAD1BAF1070FD8F867
:1038380000B01CD10BF046FA07EE900AF8EE677A52
:10384800C7EE887ACBED117AD8F800B00BF03AFAC7
:1038580007EE900AF8EE677AC7EE887ACBED127A0F
:10386800D8F800B00BF02EFA8BF84C0012E00BF0F1
:1038780029FAD3448BF80100D8F800B00BF022FAEB
:10388800D3448BF80B00D8F800B00BF01BFAD344E4
:103898008BF815000AF1010ABAF10A0FC5D100F038
:1038A8003FBCD8F800B00BF00DFAD3448BF80100F8
:1038B800D8F800B00BF006FAD3448BF80B00D8F810
:1038C80000B00BF0FFF9D3440AF1010ABAF10A0F6C
:1038D8008BF81500E5D100F023BC8246DFF8B081F3
:1038E8009FED6D8AD8F800B00BF0F6F907EE900A54
:1038F800F8EE677A0BEB8A0BC7EE887ACBED087A7D
:10390800D8F800B00BF0E8F907EE900AF8EE677AFD
:103918000BEB8A0BC7EE887ACBED0B7AD8F800B0A0
:103928000BF0DAF907EE900AF8EE677A0BEB8A0BE0
:10393800C7EE887A0AF1010ABAF1030FCBED0E7AC5
:10394800CCD1BAF1070FD8F800B01CD10BF0C4F9EC
:1039580007EE900AF8EE677AC7EE887ACBED117A0F
:10396800D8F800B00BF0B8F907EE900AF8EE677ACD
:10397800C7EE887ACBED127AD8F800B00BF0ACF924
:103988008BF84C0012E00BF0A7F9D3448BF8010038
:10399800D8F800B00BF0A0F9D3448BF80B00D8F896
:1039A80000B00BF099F9D3448BF815000AF1010A1D
:1039B800BAF10A0FC5D1B3E30BF084F91328834693
:1039C8003FF6D6AEDFF8C8A0DAF800800BF07AF937
:1039D8000023324A0C2101FB0322117A814222D1B1
:1039E8000FFA8BFB08EB8B08137888F879300BF00B
:1039F80069F988F87A000BF065F988F87B000BF014
:103A080061F9274B274A1A6088F87C00264BDAF8B8
:103A1800000018600021793007F0ECF9234B80F0A2
:103A2800010018707CE301331B2BD2D1A0E60BF008
:103A380049F90B2882463FF69BAE154BD3F8008018
:103A48000BF040F903283FF693AE062303FB0A88E0
:103A580088F8CE000BF036F988F8C9000BF032F977
:103A680088F8CA000BF02EF988F8CB000BF02AF979
:103A780088F8CC000BF026F988F8CD0050E300BF99
:103A880048200020080F002024200020980F002044
:103A9800201000200000C84200007A448862010813
:103AA800000F00208C210020040F002010000020AF
:103AB8005379092B7FF65CAE019BD3F800800BF09D
:103AC80001F9019B88F80000D3F800800BF0FAF8A0
:103AD80088F801000BF0F6F8019B64281B68A8BF62
:103AE800642018710BF0EEF8019B64281B68A8BFCE
:103AF800642058710BF0E6F8019BFF281B68A8BFEB
:103B0800FF2098710BF0DEF8019B6428D3F8008041
:103B180028BF642088F807000BF0D4F8019B88F8C8
:103B28000200D3F800800BF0CDF8019B88F8030061
:103B3800D3F800800BF0D0F8DAF80030A8F80A00C3
:103B48005B790A2B40F2EC82D74BD3F800800BF05C
:103B5800B9F888F80800E3E20BF0BEF86FF4AF623A
:103B680083189BB2C62B98BFA4F898010BF0B4F841
:103B7800A4F844010BF0B0F8A4F846010BF0ACF837
:103B8800A4F848010BF0A8F8A4F8DA010BF09AF8A9
:103B980084F8EB010BF096F80BF094F884F8EC013C
:103BA8000BF090F884F887010BF08CF884F89401F6
:103BB8000BF088F8BD4BD3F800800BF08DF800EBC4
:103BC80080004000A8F856001BE10BF085F8B84BC0
:103BD80023F8180008F10108B8F1080FF5D19FE2A1
:103BE80053790F2B7FF4C4AD0BF06CF8072880468F
:103BF8003FF6BEAD029BD3F800A00BF06DF80E2384
:103C080003FB08F8C244029BAAF81901D3F800A0E4
:103C18000BF062F8C244029BAAF81B01D3F800A07B
:103C28000BF05AF8C244029BAAF81D01D3F800A071
:103C38000BF048F8C244029B8AF81F01D3F800A091
:103C48000BF040F8C244029B8AF82001D3F800A088
:103C58000BF038F8C244029B8AF82101D3F800A07F
:103C68000BF030F8C244029B8AF82201D3F800A076
:103C78000BF03CF8D044C8F8230151E20BF022F8CD
:103C88000F2880463FF674AD0BF01CF8C8EBC80847
:103C9800A04488F8D4000BF015F888F8D5000BF08C
:103CA80011F888F8D6000BF00DF888F8D7000BF05B
:103CB80009F888F8D8000BF005F888F8D9000BF057
:103CC80001F888F8DA0007F08FFC29E22B785B0707
:103CD80000F126820BF0D6FA03F042FA03F0FAFA62
:103CE8001EE22B78580700F11B82724B4FF4C87202
:103CF8001A8015E22B78590700F112826E4A137860
:103D080043F0040328E02B785A07E5D55BE20AF074
:103D1800D9FF694B1A7810B142F0020201E022F093
:103D280002021A700AF0CEFF644BDFF8B0811870F7
:103D38000AF0DCFFC8F800000AF0D8FFC8F8040051
:103D48000AF0CAFF5E4B18800AF0C6FF5D4B5E4A58
:103D58001880137843F002031370E1E10AF0B2FF10
:103D680003900AF0C3FF83460AF0C0FF82460AF0B8
:103D7800BDFF80460AF0B0FF0AF0AEFF0AF0A2FFCE
:103D8800039BA3B9514B1020C3F800B0C3F804A09B
:103D980003F093F9484A137843F001031370B8F11C
:103DA800000F00F0BD814A4BC3F80080B8E1102B2A
:103DB80040F0B681474BC3F800B0C3F804A0B8F18F
:103DC800000F02D0424BC3F800804248424B022207
:103DD800011D1A7008F094F9A2E1A0600AF086FFAC
:103DE800A3681843A0609BE10AF076FFA4F85C0181
:103DF8000AF072FFA4F85E010AF06EFFA4F86001F1
:103E08008EE10AF05FFF84F87C010AF05BFF84F81A
:103E180080010AF057FF84F87F010AF053FF84F805
:103E280081017DE10AF058FFA4F882010AF054FFED
:103E3800A4F884010AF046FF84F886010AF04CFFD2
:103E4800A4F888016CE10AF03DFF84F892010AF0B9
:103E580043FFA4F89C010AF03FFFA4F898010AF078
:103E68003BFFA4F89A010AF02DFFDAF8003084F835
:103E780093015B79082B40F253810AF02DFFA4F8D7
:103E88009E010AF029FFA4F8A00149E10AF01AFFEF
:103E980084F8D8010AF016FF84F8D9010AF01CFF4B
:103EA800A4F8DA013CE100BF4010002020100020F7
:103EB800961F0020C60E0020D4100020DA10002023
:103EC800D8100020D61000204610002048100020EE
:103ED80058100020501000200C0F0020DC1000208B
:103EE80092F805800323B8FBF3F8B8F1120F3FF6F8
:103EF8003FACDFF8FCA34FF0000BC34580F0108106
:103F08000AF0E0FE8AF8A2010AF0E6FE40F2ED238C
:103F1800984205DD40F6CA039842A8BF184601E05A
:103F280040F2EE20A0F2EE2019230BF1010B90FBDA
:103F3800F3F00AF1020A8AF8A101DEE70AF0C2FEEC
:103F480084F89401ECE00AF0BDFE04EB080308F1E4
:103F58000108B8F1080F83F88A01F4D1E0E00AF00B
:103F6800B1FEC4F808B060710AF0C0FEA368184337
:103F7800A0600AF0A7FE84F892010AF0ADFEA4F84A
:103F88005C010AF0A9FEA4F85E010AF0A5FEA4F8F7
:103F980060010AF0A1FEA4F882010AF09DFEA4F8CF
:103FA8008401BDE053794FF0070AB3FBFAF2C2EB84
:103FB800C2029A1A12F0FF0F7FF4DAABB3FBFAFAD7
:103FC8000AF1FF3A5FFA8AFABAF1FF0F00F0A88007
:103FD8000AF078FE5FFA80FB4FFA8BF006F03AFEA3
:103FE800804600283FF4C4AB80F800B00AF074FEA5
:103FF800A8F802000AF066FE88F804000AF062FEDB
:1040080088F805000AF05EFE88F807000AF05AFEF4
:1040180088F80600D4E7DFF8D88208F1400A0AF0E9
:104028005BFEA8F89C020AF04DFE88F89E020AF092
:1040380049FE08F1040888F89B02D045EFD16FE0EB
:104048000AF040FE1F2880463FF692ABD9F80030B0
:104058005B79082B7FF48CAB0AF03EFE08F18608EA
:1040680004EB880800F03F00A8F806000AF034FEC8
:10407800B8F80630800100F4FE501843A8F806008E
:104088000AF020FE000188F804000AF01BFE98F8E8
:10409800043000F00F00184388F804000AF012FEFC
:1040A80088F805000AF01AF93AE07D4B012283F8F6
:1040B800352035E00AF006FEFF2882461BD1002392
:1040C8008DF81F309DF81F30052B29D89DF81F004B
:1040D800744A9DF81F3052F8300002EBC3030121E7
:1040E8005B68994089B2042204F018FD9DF81F30DE
:1040F8000133DBB2E4E705283FF63AAB00200AF0CB
:1041080033FE0AF00DFED8F8000007F0C1F818B920
:10411800322006F0D0FEF6E74FFA8AF004F00CFDE4
:1041280000200AF021FEFFF7A6B95F4B985907F067
:10413800AFF818B9322006F0BEFEF6E707F014FA19
:1041480002F0E4FF594B5A4ADA60FFF7A1B90C288C
:104158003FD00A2841D1574D57480AF08DFE2846CE
:10416800232110F0CCF908B1401B20602368002BF4
:1041780036D1504823600021302210F08AF93B786C
:10418800002B60D14D4B1B689B0615D54C4B444901
:104198001B688A6B9A1A002A0EDB4A4A1278042A8C
:1041A8000AD9494A03F5123303F5F8738B63938AE6
:1041B8009BB283F488439382444B9B68002B69D05D
:1041C8004348984766E001F0BFFEFFF754B90C2852
:1041D80047D140480AF050FE35E00D2835D1BAE7FE
:1041E8005A1EA95C202901D11346C0E7314A236031
:1041F8000021D154384B394DD3F800A0D5F800B080
:10420800DFF8B090584610F088F90646324648461E
:10421800594610F08BF9324A28B919F80630534438
:104228005B78580703D010359542E7D306E09542EE
:1042380004D2701CEB684844984702E029480AF009
:104248001BFE002395E7284807E07F280DD1013B96
:10425800184A264823600021D1540AF00DFEFFF7C2
:1042680076B87F2804D1FFF772B82F2B3FF66FA8D6
:10427800A0F12002D2B25E2A3FF669A813B920281D
:104288003FF465A85A1C22600A4AD0540AF0ECFD93
:10429800FFF75DB809B0BDEC028BBDE8F08F00BF39
:1042A800980F00208C850108AC11002000ED00E07B
:1042B8000400FA05E41C0020538F0108D0100020E8
:1042C800DC2B0020DA100020001000483C280020D9
:1042D800B2100020C081010820010020406A0108B6
:1042E800006C0108CB810108BB810108E781010846
:1042F800482000202DE9F0474D282DED028B04467B
:1043080000F0598600F2B980302800F0C08651D8F4
:10431800222800F0978423D8032800F0018214D8BB
:10432800012800F0F181022840F0FF8604200AF0FD
:104338001BFD43200AF0E3FC4C200AF0E0FC462079
:104348000AF0DDFC4C2000F05CBE042800F0F1818E
:10435800052840F0EA861A200AF006FD0024F8E154
:10436800282800F0E78515D8242800F0CE852628CF
:1043780040F0DB86D84C06200AF0F6FCB4F85C0165
:104388000AF0F5FCB4F85E010AF0F1FCB4F860013B
:1043980000F0B8BD2C2800F0E0852E2800F06186DA
:1043A8002A2840F0C28601200AF0DEFCCA4B587960
:1043B80000F027BE3D2800F0F5821ED8362800F010
:1043C80031860BD8322800F01686342840F0AD86A6
:1043D80048200AF0C9FC002500F056BC3A2800F035
:1043E800B7823B2800F02784382840F09E860420B6
:1043F8000AF0BAFCB84C00F08EBD452800F0828661
:1044080027D8402800F00086422840F08E86B24C1B
:1044180010200AF0A9FC60790AF071FCA0680AF083
:10442800AFFC94F892010AF06AFCB4F85C010AF057
:104438009EFCB4F85E010AF09AFCB4F860010AF038
:1044480096FCB4F882010AF092FCB4F8840100F0FA
:1044580059BD492800F0B1824B2800F09D854628B7
:1044680040F063860D200AF07FFC00200AF047FC2C
:1044780000200AF085FC00F050BE702800F0F082A1
:1044880000F2DD80692800F0438200F2AF806628E0
:1044980000F09D8100F29F80642800F073816528F8
:1044A80040F043868D4C0B200AF05EFC20880AF011
:1044B8005EFC62688A4B9A420CBF2089608980B290
:1044C8000AF055FC874B1B68C3F3C000C3F3800296
:1044D800800040EA4200C3F340021043C3F3401295
:1044E80040EAC20003F0100318430AF040FC7E4B78
:1044F8001A88E36812F0010F14BF4FF0020C4FF056
:10450800000C12F0020F02F0080814BF4FF0040E5E
:104518004FF0000E03F4475912F0040F14BF102790
:10452800002749EA080912F0400F03F4804814BF35
:104538002026002649EA080912F0100F03F4004863
:1045480014BF4FF40075002549EA080912F0200F3E
:1045580003F4803814BF4FF48060002049EA08094A
:1045680012F4807F03F4003814BF4FF40061002177
:1045780049EA080912F4007F03F480285B4A49EAF3
:10458800080903F4002849EA0809127803F4801896
:1045980049EA080903F0007349EA0303C2F38002F9
:1045A80043EA020343EA0C0343EA0E0E4EEA070706
:1045B80046EA070645EA060540EA050041EA000121
:1045C80014BF4FF400184FF00008002041EA080813
:1045D8000346217CE6E0672800F02181682840F046
:1045E800A48510200AF0C0FB002488E16C2800F0A4
:1045F800A28117D86A2800F00B846B2840F09585B3
:1046080005200AF0B1FB3A4B18880AF0B0FB394B89
:1046180018880AF0ACFB314B93F86E0000F00100EB
:1046280000F0EFBC6E2800F0978100F2CC810620E4
:104638000AF09AFB00200AF0A3FB00F062BC78287D
:1046480000F0FA8018D8742800F03F830AD872283E
:1046580000F09E83732840F0688508200AF084FBE8
:104668000124CEE3762800F0F38300F267832F203D
:104678000AF07AFB204CD6E2A42800F00F8414D864
:104688007B2800F07682A02840F04F850C200AF0A5
:104698006BFB1A4B18680AF073FB194B18680AF081
:1046A8006FFB184B186800F03CBDF12800F0008142
:1046B800FE2800F01A84F02840F03785074C0420C3
:1046C8000AF052FBA36CB3F85A000AF050FBA36C33
:1046D800B3F8580000F016BC48200020D80F00207E
:1046E80000540040D010002098110020FD2B00201D
:1046F8004E1100205011002057620108ACF7FF1F2F
:10470800B0F7FF1FB4F7FF1F03200AF02DFB0020AE
:104718000AF0F5FA20460AF0F2FA0C2000F071BC13
:104728000AF022FB01200AF0EAFA0A200AF0E7FA66
:10473800B2E306200AF018FB53200AF0E0FA4420FE
:104748000AF0DDFA46200AF0DAFA33200AF0D7FA3E
:10475800D7E3B24B185D01340AF0D1FA0B2CF8D12B
:104768000024AF4B185D01340AF0C9FA082CF8D1BF
:104778000024AC4B185D01340AF0C1FA072CF8D1BB
:1047880000F0D1BC07200AF0EFFAE7200AF0B7FAE8
:10479800A54B58790AF0B3FA00200AF0B0FA0420C1
:1047A80000F0BFBC8B420BD2A04A9C5C012202FAEB
:1047B80004F414EA080F1CBF9A4010430133F1E7D0
:1047C8000AF0DEFA984B93F8A40700F01ABC1220FE
:1047D8000AF0CAFA964B1B88B3F5806F8CBF082580
:1047E80001250024934B33F9140090FBF5F00134B4
:1047F80080B20AF0BCFA032CF4D18F4CA08D0AF0D9
:10480800B6FAE08D0AF0B3FA208E0AF0B0FA608E9C
:104818000AF0ADFAA08E0AF0AAFAE08E72E3102030
:104828000AF0A2FA0024854B185D01340AF067FAF1
:10483800102CF8D100F077BC70200AF095FA002609
:104848007D4D0E24AB6C744323440136B3F8190133
:104858000AF08DFAAB6C2344B3F81B010AF087FA0F
:10486800AB6C2344B3F81D010AF081FAAB6C234406
:1048780093F81F010AF043FAAB6C234493F8200124
:104888000AF03DFAAB6C234493F821010AF037FA99
:10489800AB6C234493F822010AF031FAAB6C1C4448
:1048A800D4F823010AF06CFA082EC9D100F03BBCF9
:1048B80070205D4C0AF058FA04F1700594F8D400A1
:1048C8000AF01DFA94F8D5000AF019FA94F8D600FF
:1048D8000AF015FA94F8D7000AF011FA94F8D800FB
:1048E8000AF00DFA94F8D9000AF009FA073494F896
:1048F800D3000AF004FAAC42E0D100F014BC504BEB
:10490800185D01340AF0FBF9102CF8D100F00BBC4B
:104918004C4D2878400000F0FE000AF025FA0024EB
:104928002B789C4280F0FF83474B33F814000AF041
:104938001EFA0134F4E7454C06200AF015FA2088DF
:104948000AF015FA60880AF012FA414B1888D9E281
:1049580004200AF009FAE3E307200AF005FA3D4BC0
:104968001888FF28A8BFFF20C0B20AF0C8F93A4B40
:10497800186880F3100080B20AF0F9F92E4BB3F8EA
:1049880064000AF0F4F9284B93F88721334B186830
:1049980022B10A23584380F3100001E000F30F000E
:1049A80080B2AFE2204C02200AF0DEF994F8DE0172
:1049B8000AF0A5F994F8DD0123E302200AF0D4F9FE
:1049C800194B98899EE21C4C0B200AF0CDF9A36E76
:1049D80018780AF094F9A36E58780AF090F900262E
:1049E8002546AB6E144C3344013618790AF087F922
:1049F800032EF6D1A36ED8790AF081F9A36E9878C0
:104A08000AF07DF9A36ED8780AF079F9A36E58896F
:104A18000AF0ADF9A36E187AF3E200BFF87E010838
:104A2800047F0108D97E010848200020E90F0020F2
:104A380012000020AA100020D80F0020101000201B
:104A4800241000204812002024200020E01F00200D
:104A5800B0100020C0100020CC100020C81000208A
:104A6800C64C1E200AF080F9A36C1B78022B4FF06D
:104A780000056BD1A36C03EB850393ED080AB2EE36
:104A8800048A20EE080A0FF013FF80F30800C0B272
:104A98000AF035F9A36CDFEDBA7A03EB850393EDE1
:104AA8000B0A20EE270A0FF003FF80F30800C0B2BC
:104AB8000AF025F9A36CDFEDB37A03EB850393EDD8
:104AC8000E0A20EE270A0FF0F3FE80F30800C0B2AA
:104AD80001350AF014F9032DCCD1072DA36C23D18D
:104AE80093ED110A20EE080A0FF0E2FE80F30800A9
:104AF800C0B20AF004F9A36C93ED120A20EE080A7A
:104B08000FF0D6FE80F30800C0B20AF0F8F8A36CE4
:104B180093F84C3000EE103AB8EE400A0FF0C8FE99
:104B280080F30800C0B20BE02B4458780AF0E7F88D
:104B3800A36C2B44D87A0AF0E2F8A36C2B44587D76
:104B480001350AF0DCF80A2DC7D1ECE2A36C2B443E
:104B580058780AF0D4F8A36C2B44D87A0AF0CFF826
:104B6800A36C2B440135587D0AF0C9F80A2DEDD104
:104B7800D9E23C200AF0F8F80024804D9FED818AA4
:104B8800AB6C03EB840393ED080A20EE080A0FF0E0
:104B98008FFE80B20AF0EBF8AB6C03EB840393ED65
:104BA8000B0A20EE080A0FF083FE80B20AF0DFF845
:104BB800AB6C03EB840393ED0E0A20EE080A0FF0AA
:104BC80077FE013480B20AF0D2F8032CD5D1072C35
:104BD800AB6C16D193ED110A20EE080A0FF068FEAF
:104BE80080B20AF0C4F8AB6C93ED120A20EE080A02
:104BF8000FF05EFE80B20AF0BAF8AB6C93F84C0086
:104C08000BE0234458780AF0B2F8AB6C2344D87A06
:104C18000AF0ADF8AB6C2344587D01340AF0A7F8CC
:104C28000A2CD4D17FE214F8010F002800F07B820F
:104C38000AF065F8F7E701200AF096F84F4B9B6CED
:104C48001878DEE150200AF08FF800254B4B9C6C59
:104C58004D4B04EB85040C2194F8792001FB0233B9
:104C6800013593F838000AF04AF894F87A000AF007
:104C780046F894F87B000AF042F894F87C000AF0B1
:104C88003EF8142DE2D14EE23C4B9C6C062303FB0C
:104C98000544013594F8CE000AF031F894F8C900BB
:104CA8000AF02DF894F8CA000AF029F894F8CB0015
:104CB8000AF025F894F8CC000AF021F894F8CD0011
:104CC8000AF01DF80C2DDFD12DE24FF00008012667
:104CD80000272A4B1A7C974227DA11330024FA5C02
:104CE800294D0C2305F130016343595C914207D1EA
:104CF8002B44586B0FF011FC82462EB9B14605E0E3
:104D080001341B2CECD10EE080440CE0D1450ADACA
:104D18000C2303FB04535B6B13F8090009F0EFFF46
:104D280009F10109F2E70137D3E7002E00F0FB8112
:104D38005FFA88F00AF018F80026C9E70F4D287CBA
:104D48000AF012F800242B7C9C4280F0EC810F4B77
:104D5800E65C00210C480C2200F1300702FB01F34D
:104D6800DA5DB24205D1034493F8380009F0C7FF71
:104D780002E001311B29EDD10134E4E7D80F00200E
:104D88000000C84200007A4458620108E90F002078
:104D9800D14C162009F0E8FFB4F8980109F0E7FFB4
:104DA800B4F8440109F0E3FFB4F8460109F0DFFF65
:104DB800B4F8480109F0DBFFB4F8DA0109F0D7FFCD
:104DC80094F8EB0109F09BFF002009F098FF94F894
:104DD800EC0109F094FF94F8870109F090FF94F82A
:104DE800940109F08CFF002009F089FFBB4B9B6CF4
:104DF8000A20B3F9563093FBF0F080B209F0B7FF00
:104E080089E0E0B2013409F07AFF092CF9D18AE18E
:104E1800102009F0A9FFB24BB24C187800F002003C
:104E280009F06DFFB04B187809F069FF206809F0A8
:104E3800A7FF606809F0A4FFAC4B188809F097FF3A
:104E4800AB4B188809F093FFA44BB3F86C0059E0FA
:104E580009F038FF0746122009F086FF9F4C17B962
:104E6800266F656F05E0102F13BF0025A66FE56F4D
:104E78002E46384609F043FF304609F081FF2846A0
:104E880009F07EFFD4F8800009F07AFF002009F0CD
:104E98006EFF002009F06BFF0020B2E08F4D95F8FF
:104EA800840080000130C0B209F05EFF95F88400EC
:104EB80009F025FF00242E4696F884309C4280F0A5
:104EC80032818C4D285D09F01AFF05F11003185D39
:104ED80009F015FF05F120033035185D09F00FFFC3
:104EE800285D09F00CFF0134E6E7082009F03CFFD3
:104EF800002009F03CFF002009F039FF002009F0EC
:104F080036FF002009F033FF0DE1042009F02CFFE3
:104F1800714B986805E194F87C0109F0F0FE94F86B
:104F2800800109F0ECFE94F87F0109F0E8FE94F89E
:104F3800810166E0684C072009F016FFB4F8820189
:104F480009F015FFB4F8840109F011FF94F88601FF
:104F580009F0D5FEB4F88801D4E75F4C0C2009F0BD
:104F680003FF94F8920109F0CAFEB4F89C0109F015
:104F7800FEFEB4F8980109F0FAFEB4F89A0109F0B7
:104F8800F6FE94F8930109F0BAFEB4F89E0109F010
:104F9800EEFEB4F8A001B5E74F4C042009F0E4FE9A
:104FA80094F8D80109F0ABFE94F8D90109F0A7FEEE
:104FB800B4F8DA01A6E7504C504D207800EB4000D9
:104FC800C0B209F0D1FE002623789E4205F1020501
:104FD80080F0A98015F8020C09F091FE15F8010C73
:104FE80000EB800000EB800000F2EE2080B209F0B8
:104FF800BEFE0136E8E7012009F0B6FE364B93F80D
:10500800940109F07CFE8EE0082009F0ADFE002432
:10501800314B2344013493F88A0109F070FE082CBF
:10502800F6D180E02D4B2C4C93F8C500C0EBC000A6
:10503800C0B209F099FE04F11805314A94F8F2015A
:1050480092F9001043B2994271D092F90C1099422A
:105058006DD092F918209A4269D00834AC42ECD14C
:1050680061E040201C4C09F07FFE04F14005B4F8D3
:105078009C0209F07CFE94F89E0209F040FE04347C
:1050880094F89B0209F03BFEAC42F0D14BE0E020E3
:10509800114C09F069FE04F18005B4F81E0200F015
:1050A8003F0009F064FEB4F81E02C0F3861009F050
:1050B8005EFE94F81C02000909F021FE94F81C0217
:1050C80000F00F0009F01BFE043494F8190209F0EF
:1050D80016FEAC42E1D126E048200020D80F00207F
:1050E800D4100020DC100020DA100020D810002096
:1050F800D61000205D10002048120020EA21002070
:1051080054120020132009F02FFE0024154B185DBF
:10511800013409F0F4FD0B2CF8D1002009F030FE21
:10512800002009F02DFE012018E0002016E009F00B
:10513800E6FDB4F8F40109F01AFE94F8F60109F056
:10514800DEFD94F8F70109F0DAFD94F8F90109F0A9
:10515800D6FD94F8F80109F0D2FD7EE7BDEC028B8C
:10516800BDE8F087F87E01082DE9F047B94CBA4E42
:10517800237886B00746002B00F0F2813268636816
:10518800D31A7C2B40F2EC81237A626001332372BC
:10519800002505F12400DFF8BC82C0B20CF05AF8F3
:1051A80008F10A0333F9153007EE903AAB4B1B8828
:1051B800B8EEE77A07EE903AF8EEE77A0135C7EEEF
:1051C800277A9FEDA77A67EE877AFDEEE77ACDED2D
:1051D800037ABDF90C000CF02BF8032DD9D130203F
:1051E8000CF038F800200CF023F80CF02BF898F8A5
:1051F800085015F0030520D1D8F8042041F288336F
:105208009A420BD910200CF025F828460CF010F81B
:1052180021200CF01FF828460CF00AF814200CF096
:1052280019F8B4F910000CF003F81C200CF012F86F
:1052380000200BF0FDFF0CF005F8237ADFF814824C
:105248005B0740F06A8102200CF004F80A23B8F9E1
:10525800120090FBF3F00BF0EBFF0320B8F91A50A3
:10526800DFF810920BF0F6FF7E4B1B7813F0040F5B
:105278004FF0050A95FBFAF5ADB20BD038460AF0A7
:1052880023FE28B9D9F8003013F0100F18BF0025F5
:1052980028B205E0D8F81C309889B0FBFAF000B2C3
:1052A8000BF0C6FFD9F800309F0740F18180DFF886
:1052B800C891678C99F80030228C664D3F014FF0F9
:1052C8006408BFB208FB02325B00B2FBF3F347EAA3
:1052D8000327BFB2C3F303231F4306200BF0BAFF13
:1052E80038B20BF0A5FF638C99F8001001339BB21C
:1052F80093FBF1F201FB12336384636A9B7B012BFE
:1053080005D139200BF0A6FFB5F9200019E02D8C46
:105318006E233A205D4315270BF09CFF95FBF7F5AC
:10532800AFB2B7FBF8F528B20BF082FF08FB157592
:105338003B200BF08FFFA8B2451D0A2095FBF0F02B
:1053480000B20BF075FF28200BF084FFA36A414DD3
:105358000A2093FBF0F000B20BF06AFF04200BF078
:1053680079FFE369E86A9A894FF6FF739842A8BF04
:105378001846C2B10028ACBF131A134607EE903A7C
:105388009FED397AF8EEE77A67EE877A07EE102A0A
:10539800B8EEC77AC7EE877AFDEEE77A17EE900A7D
:1053A8006428A8BF642020EAE07000B20BF040FF38
:1053B800236B284F9D0640F1A58097F83430980755
:1053C8001BD511200BF046FFF88E284B4FF4F365E0
:1053D800684390FBF3F000B20BF02AFF19200BF0A2
:1053E80039FFF88E4543642095FBF0F595FBF0F303
:1053F80000FB135000B20BF01BFF94F83430258FDC
:1054080013F0020F08BF002501200BF023FF28B27C
:105418000BF00EFF09200BF01DFF00200BF008FF1A
:10542800134B94F83A501A88B2F5967F0AD9094B6B
:105438001B7A03F00F03072B04D842F20F7595422D
:1054480028BF154605200BF005FF636A5B7BBBB9D7
:1054580028B232E0A01000200C200020120000200A
:1054680000007A44FD2B00200000C842A0860100FD
:1054780012010020E81F0020100100206666E63FA8
:10548800A5F1200307EE903A1FED047AF8EEE77ACB
:10549800F6EE006AC7EE877ABEEE007AF5EEC07ABD
:1054A800F1EE10FA58BFB0EE667A77EE877AFDEE25
:1054B800E77ACDED037ABDF90C000BF0B9FE94F84C
:1054C8003420C34B910703D493F83B20012A04D11D
:1054D800012384F83B30BF481BE05B6ADFEDBE6AFE
:1054E80093ED017AD3ED027A27EE267A67EEA67A53
:1054F800BDEEC77AFDEEE77A8DED047ACDED057A3B
:1055080004A806E0B54A92E8030004AB83E8030068
:10551800184602F0B5FD0BF095FE237A282B1FD113
:10552800AB4B00221A723C2733684FF47A70B3FBF6
:10553800F0F817200BF08EFEB8FBF7F5B5FBF7F087
:1055480007FB1050000200B20BF072FE18200BF09F
:1055580081FE07FB158000B20BF06AFE0BF072FEAD
:1055680094F844309A4D002B00F0578105F07CFCEC
:10557800AB6C9B4AC31A9342074640F2BC80002397
:1055880085F84E3085F850302B8CDAB21B0A85F836
:105598006A2085F86B3085F8602085F86130AA6F3D
:1055A80033689A1AEB6FD97B4FF47A734B439A425C
:1055B8000DD38C4B1B68AB6795F88030013B012BF2
:1055C8009FBF102385F84E30022385F850300A20FB
:1055D800A26A92FBF0F284F86820121284F869201B
:1055E80094F83420E36A93FBF0F384F86C301B12D0
:1055F80084F86D30920794F83A30754984F89B30F6
:1056080003D42D2381F89C3074E0042BD4F83C900B
:10561800266CDFF8E081744A8CBF3323322381F88B
:105628009C304FF0060C714B99FBF3F096FBF3F3AB
:1056380008FB009108FB036803EB83030CFB01F1F3
:1056480003EB830391FBF2FE642502FB1E119B0012
:1056580091FBF5F184F88D1009120CFB08FC84F815
:105668008E109CFBF2F143FA81F39BB202FB11C24C
:1056780092FBF5F284F89220121284F8903084F8A4
:1056880093201B0AE28E84F891302423534393FB22
:10569800F5F5B4F8AE3084F8943000EB80001B0ABE
:1056A80000EB8000800084F895300A22238FB3FB3A
:1056B800F2F303F5FA739BB240FA8EF080B284F8E5
:1056C80096301B0A4FEAD97984F88B00F60F000A46
:1056D80084F8885084F89730C5F30725B4F8B030BB
:1056E80084F88A9084F88C0084F88F6084F8895054
:1056F80084F89D30A76494F8B280354DB8F1000F56
:105708000DD1D5F8B80005F0CCFD012807D902283D
:10571800374E00F0458202F0A5FC0123B370D4F89F
:10572800BC202B4D002A78D095F8B2603EB1D5F850
:10573800C43040F6B731FB1A8B4219D86DE001230B
:10574800D5F8B80085F8B23003F08DFAD5F8C8302E
:1057580093F9000002238DE84800082132464FF4EF
:10576800964305F0B2FB85F8CC60C5F8B80052E066
:1057780095F8C060CEB9D5F8B800C5F8BC6085F812
:10578800B26003F070FAD5F8C83093F9000001232D
:105798008DE84800082132464FF4964305F095FB02
:1057A800C5F8B80002F05EFC35E0013EF6B285F8B7
:1057B800C06095F8CC1095F8CD30EEB94A1C01338D
:1057C80085F8CC2085F8CD30D5F8B80021E000BFA9
:1057D800A0100020DC1000208096184BD863010828
:1057E8003F0D03000C20002040420F0080969800D7
:1057F80012000020806967FF12F8016BC5F8BC2011
:10580800701885F8CC000133D5F8B80085F8CD308C
:10581800314605F049FDC4F8C47094F8CE30954D72
:10582800DBB1D5F8D030C3B1D5F8D430ABB1C5F8B9
:10583800D8301B68904AC5F8DC30D5F8E0301344FE
:10584800187AFEF757FD09F06BFAD5F8E030013306
:10585800092B88BF0023C5F8E030884D94F8E42070
:105868002E68844B002A00F0D581D3F8E820002A5E
:1058780000F0D08193F8EC30013B012B00F2CA8193
:10588800D4F8E8007B4F05F00CFDE0B1D7F8E8004C
:1058980005F004FD97F8ED30D5F800907E2B804692
:1058A8000ED102231B2887F8EC3009D1D7F8E8007D
:1058B80005F0F7FC20B90123C7F8F09087F8F43019
:1058C80084F8ED80DCE7D7F8F0202B689B1A41F6C6
:1058D800583293421DD9032387F8EC309AE1684A7D
:1058E80032F8130010B903464FF403600133B0F5E2
:1058F800C06FDBB269D01DD9B0F5006F6ED030D95A
:10590800B0F5036F3BD184F8F530236B594F9A06F5
:105918003CD494F8F41094F8F530002900F03D8157
:105928002A68921B012ADAD984F8F530002384F812
:10593800F4306FE1B0F5007F3ED006D8B0F5807F37
:105948007CD0B0F5887F79D0E7E7B0F5806F00F0BC
:105958009B80B0F5826F00F0E080B0F5047FDCD169
:1059680020E0B0F5E26F78D0B0F5E46F7AD0B0F50A
:10597800E06FD2D184F8F530B4F90A1076E0B0F5CA
:10598800046F63D0B0F5026FC7D1F1E097F83430F7
:105998009B07BED5F98E24234B431233642193FB16
:1059A800F1F1F4E084F8F530364B324F1B68990773
:1059B800AFD53B8C0A21E9E084F8F530314B2D4F07
:1059C8001B681A05A5D5B96AE1E084F8F5302D4BB6
:1059D800284F1B681B059CD5F96AD8E0216B254A1E
:1059E80084F8F530880694D592F83410890790D554
:1059F800DB0711D5136C83EAE371002BA1EBE3718C
:105A080001EB51014FF01902B1FBF2F1ACBF41F0CB
:105A1800004141F040410EE0D36B83EAE371A1EB12
:105A2800E371002B01EB51014FF01902B1FBF2F1C8
:105A3800B8BF41F080414FF4006088E084F8F53049
:105A4800236B5F077FF565AF00215FE0B4F91010A5
:105A580084F8F5306423594379E084F8F530B4F9D3
:105A68000C1003E0B4F90E1084F8F5302C2391FBE8
:105A7800F3F16CE0A0100020D86301080C2000208E
:105A8800FE820108E81F002084F8F53094F8F6300B
:105A9800624A0133DBB2032B88BF012382F8F63058
:105AA80094F8F61042F2107359435D4B1B78D807EF
:105AB80048BF01319A0748BF02315F07B4F8F83090
:105AC80048BF0431D80748BF0A319A0748BF143184
:105AD8001F0648BF2831D80548BF28315A0748BF94
:105AE80064311F0748BFC831980548BF01F5C87120
:105AF8009A0648BF01F57A71DF0648BF01F5FA61D9
:105B0800580648BF01F57A614FF4806002F076FAD2
:105B1800424B002283F8F420FBE6216BDFF8FC807F
:105B280084F8F53011F0200717D098F8342012F0D7
:105B3800020F14BF4FF47A71002112F0010F14BF45
:105B48004FF4FA6300230B4494F83A10194402F016
:105B580055FA002384F8F430DBE6324B1B6819064B
:105B68007FF5D7AE394602F049FA88F8F470D0E6E6
:105B780084F8F530236B294F9A067FF5CAAE97F85B
:105B880034309B077FF5C5AE3B8F6421594302F043
:105B980035FA002387F8F430BBE684F8F53039E0AD
:105BA800B37823B1C5F8B47086F80280B7E5D5F8A4
:105BB800B430FB1AB3F57A6FFFF4B1AD0123D5F811
:105BC800B800B37005F06AFB0646D5F8B80005F0D2
:105BD80065FB76067FF4A3AD8A2802D08E280CD008
:105BE8009DE52B6B99067FF59AAD95F8B230002BA1
:105BF8007FF495AD05F1810306E095F8B230002BEE
:105C08007FF48DAD05F14C03C5F8BC302D2385F824
:105C1800C03084E506B0BDE8F08700BFA0100020C2
:105C2800FD2B0020E81F0020704708B51F4A18B94F
:105C3800536802221A8208BD0020516810800B7830
:105C480013F07F030DD14B7A990644BF02211170DE
:105C580013F0400F137814BF43F0010323F001033E
:105C680015E0012B1FD0022B1ED14B7913F0800FAA
:105C780003F00F034FEA830303F1804303F5B843AE
:105C88001B6806D003F03003102B07D101231370D3
:105C980004E003F44053B3F5805FF6E793681B69AB
:105CA8009847024808BD104608BD00BFA011002053
:105CB80010B5064C18B9636801221A8210BDA36892
:105CC8009B68984760680C3010BD00BFA011002089
:105CD80010B5064C18B9636801221A8210BDA36872
:105CE8001B68984760680A3010BD00BFA0110020EB
:105CF800084BDA68D10709D4DA68D20608D4DB6819
:105D080013F0040F14BF03200420704701207047CC
:105D1800022070470020024010B50446B0F9000088
:105D280009F02FFEB4F9020009F02BFEB4F90400C3
:105D3800BDE8104009F025BE10B50446006809F01A
:105D480020FE606809F01DFEA068BDE8104009F05B
:105D580018BE2DE9F74F012004F0BCFF002488B3DA
:105D6800012C2FD8194E4FF04C0909FB04FA06EB09
:105D78000A0808F15407BD7815B10134E4B2EEE71A
:105D880090F9003090F804E01846114B03228DE892
:105D9800240001212A4653F82E3005F096F8834650
:105DA80060B106F10C00504429464A460EF071FBDA
:105DB80001231C44C8F80CB0BB70E4B2012004F005
:105DC8006FFFCCE703B0BDE8F08F00BFA011002043
:105DD800F063010810B5184C002120461A220EF075
:105DE80058FBA4F5F870142380F8F231052300223B
:105DF800042180F8F63180F8F83180F8FE3180F817
:105E0800003280F8063280F808325223012480F8E4
:105E1800F71180F8F92180F8FF1180F8012280F845
:105E2800071280F8092280F8F03180F8FA2180F80A
:105E38000242A0F8F44110BD3822002010B5FFF747
:105E480057FF4FF43024012806D11CB1FFF750FF4B
:105E5800013CF8E7052010BD002C08BF052010BD47
:105E680070B50646441E14F8011F89B1094D28462D
:105E78000EF045FB0028F6D005F1080398423FBF15
:105E8800054B401BC018A31B38BF80F88A31EAE7CE
:105E980070BD00BF1E83010848200020031EB8BF44
:105EA8002D2210B5B8BF58420C46B8BF01F8012BD7
:105EB8000A2200F0CDFE00230370204610BD07B56E
:105EC8001C4B03F1A802C3F8A4201B4A92F89221A4
:105ED8005AB1012A14D1032183F8AA10072183F8A3
:105EE800AC2083F8AB100C2208E0022183F8AA103A
:105EF800032183F8AC2083F8AB10072283F8A8208D
:105F08000E4B0F4A1A60402004F0E4FE70B10122E3
:105F1800002390F9000040218DE80C00094A4FF455
:105F2800E13304F0D2FF003018BF012003B05DF860
:105F380004FB00BFA011002048200020180000200A
:105F4800750D0108050F01080120002108F0EEBEBB
:105F5800F0B51C4A92F8AD30D2F8B05092F8B4704F
:105F680092F8C06092F8CCE0022B0ED805EBC3047F
:105F7800591CA31CC9B206D02346A48814F0010FEB
:105F880001D0204205D10B46EEE782F8AD30002063
:105F9800F0BD93F902307CB29C4201D1002307E0A6
:105FA80074B29C420CD04FFA8EF49C42EBD102237F
:105FB80082F8AD100C2101FB0322D2F8B800F0BD25
:105FC8000123F5E7A011002030B5002202F180532B
:105FD80003F5B8539B0042F400441D6840F60F7166
:105FE80044F08004294001322143042A1960EDD18C
:105FF800024B40F08000186030BD00BF4C5C004090
:106008002DE9F843324D6E68328A377ABAB9042FCF
:1060180015D130480378012B0CD12F4B19682F4B21
:1060280089B20B445B0019681A603023A5F8D83090
:10603800027049E01023A5F8D830072744E0B48A55
:10604800B369A24294BF04270227944228BF14468A
:106058001FFA84F8404698471F4A13689BB203F119
:10606800005303F540535B0004F1010E1B689BB21B
:1060780003F1005303F540534FEA6E0E5B00002115
:10608800714500F1020009D010F8019C10F802CC0B
:106098004CEA092C23F821C00131F1E712680F4BB3
:1060A80092B213445B001A681C60338AC8EB03037E
:1060B8003382738A98443023A5F8D8304FF440537C
:1060C800A6F81280A5F8DA306B681F72BDE8F8836D
:1060D800A0110020FE2B0020505C00400230002060
:1060E8000E4B0F4A1B689BB203EBC00002443E29CB
:1060F8004FEA420209D94B09C80604BF03F1FF332E
:106108009BB29B0243F4004304E04B08C90748BF15
:1061180001339B0211681360704700BF505C004058
:106128000630002008B50B4B002093F83010FFF71D
:10613800D7FF094B5A68107A082801BF4FF48052DC
:10614800A3F8DA201022A3F8D820A0F109035842B6
:10615800584108BD18000020A011002038B5444D52
:106168006A68107810F07F0004D1537A23F0200376
:10617800537238BD022879D15388002B77D113790F
:10618800002B74D1537923F08000840004F18041FE
:1061980001F5B84113F0800F096814BF01F0300110
:1061A80001F44051032861D800295FD0927A002A6F
:1061B8005CD004F1804404F5B8441906226825D55A
:1061C80002F03002102A4CD103F07F039B0003F148
:1061D800804303F5B8431A68510641BF196840F671
:1061E8000F720A4042F4004244BF42F0C0021A60F3
:1061F8001A6822F4E04222F0400292B282F03002A1
:1062080042F4004242F080021A602AE002F440524E
:10621800B2F5805F25D128B9164B93F83010FFF7F7
:106228005FFF11E09B0003F1804303F5B8431A6850
:10623800520441BF196840F60F720A4042F44042C6
:1062480044BF42F080021A60236823F4804323F09D
:1062580070039BB283F4405343F4004343F080033C
:106268002360AB685B699847002038BD022038BDC1
:10627800A011002018000020002303604360836001
:106288008381036143618361C36103624362836203
:1062980070478A68036810B50C6A14430A69144386
:1062A8004A6914438A691443CA6914434A6A1443FD
:1062B8008A6A23F4FF4323F07003224313430360E5
:1062C8008B8943600B6883604B68C36010BD0268AC
:1062D8004FF6FE731340036000230360436083603E
:1062E800C360294B984201D1284A27E0284B98429D
:1062F80001D1264A2AE0274B984201D1234A2DE0B2
:10630800254B984201D1214A30E0244B984201D1D3
:106318001E4A33E0224B984204D11C4A536843F486
:1063280070032EE01F4B984204D1184A536843F07B
:10633800706326E01C4B984204D11C4A536843F012
:106348000F031EE01A4B984204D1184A536843F0D1
:10635800F00316E0174B984204D1144A536843F4EB
:1063680070630EE0144B984204D1104A536843F40A
:10637800704306E0114B984204D10C4A536843F429
:1063880070235360704700BF0800024000000240BD
:106398001C00024030000240440002405800024005
:1063A8006C000240800002400804024000040240E1
:1063B8001C040240300402404404024058040240D5
:1063C800036A23F001030362036A70B544688269B3
:1063D8000D6822F4803222F0730215438A8923F073
:1063E800020313438A881343134A90420FD002F5DD
:1063F800006290420BD002F54062904207D002F54D
:106408008062904203D002F5806290420DD1CA8921
:10641800CE8823F0080313430A8A24F440741443F3
:106428004A8A23F00403334314438A68446085612D
:106438004263036270BD00BF002C01409D4A53684F
:1064480003F00C03042B2DE9F04105D0082B06D0EE
:1064580099490160B3B916E0974B036012E053689D
:106468005468C3F38343991CE30349BFD36A934B2E
:10647800914C03F00F0344BF0133B4FBF3F34B43D8
:10648800036000E0002351688D4FC1F303113944C4
:1064980091F834500168EDB221FA05F44460566869
:1064A800C6F302263E4496F8346024FA06FEC0F885
:1064B80008E05668C6F3C2263E4496F83460F6B241
:1064C800F440C460D2F82C80C8F3041808F00F0C0C
:1064D80007EB4C0C18F0100FBCF844C01FFA8CFCEA
:1064E80007D0BCF1000F04D0B3FBFCFCC0F810C00F
:1064F80000E00161D2F82CC0CCF3442C0CF00F085A
:1065080007EB48071CF0100FB7F84470BFB204D06F
:106518001FB1B3FBF7F7476100E04161176BFF0656
:106528005ABF654F87618161176BBF065ABF624FBB
:10653800C761C161176B7F065ABF5F4F076201626F
:10654800176BFF0506D5994204D1AE4202D14F0020
:10655800476200E04462176BFF0406D5994204D1F4
:10656800AE4202D14F00876200E08462176BBF051C
:1065780006D5994204D1AE4202D14F00C76200E06D
:10658800C462176B7F0506D5994204D1AE4202D189
:106598004F00476400E04464176B3F0506D59942F5
:1065A80004D1AE4202D14F00876400E08464176BC7
:1065B800BF0406D5994204D1AE4202D14B00C36450
:1065C80000E08464156B3B4BAD0701D1046315E013
:1065D8001C6B04F00304012C01D101630EE01C6B59
:1065E80004F00304022C02D14FF4004305E01B6BB6
:1065F80003F00303032B01D12F4B0363146B2D4BC3
:1066080014F4403F02D1C0F834E018E01C6B04F4E5
:106618004034B4F5803F01D1416310E01C6B04F4B1
:106628004034B4F5003F02D14FF4004306E01B6B41
:1066380003F44033B3F5403F01D11F4B4363146B60
:106648001C4B14F4402F02D1C0F838E018E01C6B42
:1066580004F44024B4F5802F01D1816310E01C6B51
:1066680004F44024B4F5002F02D14FF4004306E0AF
:106678001B6B03F44023B3F5402F01D10E4B83630A
:10668800146B0C4B14F4401F02D1C0F83CE021E01D
:106698001C6B04F44014B4F5801F01D1C16319E0E8
:1066A8001C6B04F44014B4F5001F0BD14FF40043E5
:1066B8000FE000BF0010024000127A0000093D0000
:1066C800180000201B6B03F44013B3F5401F01D1E1
:1066D800134BC363126B134B12F4400F03D1C0F872
:1066E80040E0BDE8F0811A6B02F44002B2F5800F79
:1066F80002D10164BDE8F0811A6B02F44002B2F5E0
:10670800000F02D14FF4004306E01B6B03F4400373
:10671800B3F5400F01D1024B0364BDE8F08100BF1F
:1067280000127A0000100240F0B500230E681C46E3
:106738000125A54005EA060EAE452BD10F797A1E34
:10674800012A15D8856803229A4025EA0202826048
:106758004D7982689D4015438560828892B222EA0D
:106768000E0282808A798588A2402A4392B282806A
:10677800032205689A40D2431540056005689F408A
:106788002F430760C7681740CA7902FA03F547EA3A
:106798000502C2600134102C03F10203C8D1F0BD18
:1067A80038B52DED048B4A4C0368C4F8DC30838877
:1067B800A4F8E030013A0D46072A42D8DFE802F093
:1067C800040A101822292F35B4F8DC300B80B4F8ED
:1067D800DE3013E0B4F8DE300B80B4F8DC3005E0CE
:1067E800B4F8DC305B420B80B4F8DE305B4205E085
:1067F800B4F8DE305B420B80B4F8DC306B80B4F860
:10680800E0301DE0B4F8DC305B420B80B4F8DE30D9
:1068180012E0B4F8DE300B80B4F8DC300CE0B4F8E9
:10682800DC300B80B4F8DE3005E0B4F8DE305B42D3
:106838000B80B4F8DC305B426B80B4F8E0305B422C
:10684800AB80244B93F86430002B3ED1B5F900306F
:1068580094ED3C0AD4ED397A09EE103AB5F90230D4
:1068680008EE103AB8EEC88AB5F90430B8EEC99AFD
:1068780028EE000A08EE903AA7EE890AF8EEE88AB0
:10688800D4ED3F7AA7EEA80A0EF012F894ED3D0A6F
:10689800D4ED3A7A288028EE000AA7EE890AD4EDCA
:1068A800407AA7EEA80A0EF003F894ED3E0AD4ED5C
:1068B8003B7A688028EE000AA7EE890AD4ED417A6F
:1068C800A7EEA80A0DF0F4FFA880BDEC048B38BD34
:1068D800A01100201800002008B50A4890F80931D6
:1068E80000EB43030A22B3F8181189B2A0F820116B
:1068F80000F5947004F0DBFC80B20AF0C9FB024B8F
:10690800188008BDA0110020C0100020F0B5012497
:10691800B0FBF4F58D4201D34C43F9E70026D4B11E
:10692800B0FBF4F504FB1500B4FBF1F41EB9002D1F
:1069380001DC002CF3D1092D03F1010EEFB204DDC7
:10694800002A14BF3725572500E030253D441D7027
:1069580001367346E3E71C70F0BDF0B50124B0FBC7
:10696800F4F58D4201D34C43F9E70026D4B1B0FBCE
:10697800F4F504FB1500B4FBF1F41EB9002D01DC9D
:10698800002CF3D1092D03F1010EEFB204DD002A2A
:1069980014BF3725572500E030253D441D700136CA
:1069A8007346E3E71C70F0BD03685A1C0260197057
:1069B80070472DE9F843089E002B07468846144681
:1069C80014BF4FF030094FF02009334613F8012B5C
:1069D8000AB9254603E0002CFBDD013CF6E7002D53
:1069E80004DD38464946C047013DF8E724EAE47427
:1069F8003546A01B284415F8011B11B13846C0477D
:106A0800F7E7BDE8F883024B186804F04DBC00BFF7
:106A1800C80F002090ED017A07EE901AB5EE407A83
:106A2800F1EE10FA01BFF8EEE77A9FED0E7A67EE05
:106A3800877AB7EE007A04BFC7EE277AC0ED017AED
:106A480090ED017AD0ED007A30EE877A30EE670A61
:106A5800C0EE870AE0EE807AB0EE670AC0ED007AF1
:106A6800704700BFDB0FC94010B50278202A0346E3
:106A780000F10100F9D0092AF7D02D2A03D10346E5
:106A8800BFEE000A04E02B2A08BF0346B7EE000A4F
:106A9800DFED387A1A46134612F8010BA0F13001DF
:106AA800CCB2092C0AD807EE101AB8EEC77AF2EE63
:106AB800046AA7EEA67AF0EE477AECE72E2816D1FC
:106AC800F2EE046A1146B0EE666A0B4611F8012B25
:106AD800303AD0B209280AD807EE102AB8EEC77A99
:106AE80087EE267A66EE866A77EE877AEDE71A7879
:106AF80002F0DF02452A35D15A782D2A02D1023315
:106B0800012004E02B2A14BF013302330020013B8B
:106B1800002213F8011F3039CCB2092C03D80A24FB
:106B280004FB0212F5E7B2F59A7F28BF4FF49A7278
:106B38001346B7EE007A072B05D9DFED0F6A083B3D
:106B480027EE267AF7E702F007032BB1F2EE046A84
:106B580027EE267A013BF8E7F0EE476A20B1C7EE48
:106B6800877A03E0F7EE006A67EEA67A20EE270A36
:106B780010BD00BF0000000020BCBE4C30B52DED9C
:106B8800028B87B0B0EE408A0C220021054603A88C
:106B98000DF07FFCB5EEC08ADFED2A7AF1EE10FA2F
:106BA800CCBF38EE278A38EE678ADFED277A28EEE1
:106BB800278A6946FDEEC87A17EE904A84EAE4709F
:106BC800A0EBE470FFF76AF9002CACBF20232D235B
:106BD80068468DF80C300DF0A0FC012807D1302351
:106BE8008DF80D308DF80E308DF80F300CE002283E
:106BF80005D130238DF80D308DF80E3004E00328D0
:106C080004BF30238DF80D30694603A80DF068FCE9
:106C180003A80DF082FC0338C4B2224603A9284613
:106C28000DF0A8FC00232B55284608490DF058FC08
:106C380003AB284619190DF053FC284607B0BDECE4
:106C4800028B30BD6F12033A00007A443383010887
:106C580070B5064615460846B6FBF2F414B1204650
:106C6800FFF7F6FF05FB1464024B1B5D00F8013BC0
:106C780070BD00BF358301082DE9F04F814689B00A
:106C88008A4616461C4600253178002900F0DD802A
:106C9800252902D00136484675E07278302A08BFA7
:106CA800B278A2F1300319BFB71C4FF0000BF71CE4
:106CB8004FF0010B092B4FF0000819D8A2F130034F
:106CC800D9B2092905D80A2202FB083817F8012B7E
:106CD800F4E7A2F16103052B02D8A2F1570305E0FE
:106CE800A2F14103052B03D8A2F137030A2BEADDF1
:106CF8006C2A31D13A78642A07F1010600F08380C2
:106D08000BD8252A3DD003D8002A00F09E80BBE787
:106D1800582A0CD0632A19D0B6E7732A22D002D891
:106D28006E2A37D0B0E7752A5CD0782AACD1271DF7
:106D38002068A2F1580462424FF01001624155E008
:106D48002CD9582A32D0632A2AD13E46484621787F
:106D5800271DD04701350FE0642A64D00ED9732A65
:106D680014D13E46236800934846514642460023C4
:106D7800FFF71FFE271D05443C4685E7252ADFD17E
:106D88003E4648462521D04701357DE70AD86E2A78
:106D980006D13E46236804341D6075E7002A54D0A6
:106DA8003E4671E7752A26D0782AF9D1A2F1580310
:106DB80004F1040C5A422068CDF80CC04FF01001C1
:106DC8005A4105ABFFF7A2FDDDF80CC03E4664460C
:106DD80005AB00934846514642465B46FFF7E9FD3E
:106DE800054451E72068271D0A21002205ABFFF75B
:106DF800B4FD3C46ECE704F1040CCDF80CC0206867
:106E08000A210022DDE72068002804F1040708DAD7
:106E18002D238DF8143040420DF115030A2100226C
:106E2800E5E705ABFAE72068002804F1040C0ADA64
:106E38002D238DF8143040420DF11503CDF80CC008
:106E48000A210022BEE705ABF8E7284609B0BDE8ED
:106E5800F08F0FB413B50B4904AB08680A4953F80F
:106E6800042B09680193FFF707FF0446074B1868CE
:106E780004F00EFA0028F9D0204602B0BDE8104010
:106E880004B070479401002090010020C80F002032
:106E980080EAE073A3EBE0738B4206DB002801DD98
:106EA800401A704702D00844704700207047FDEE32
:106EB800C07A17EE903A2033402B43D8DFED237A7F
:106EC800B4EEE70AF1EE10FA04DDDFED217A30EED8
:106ED800670AF3E7DFED1F7AB4EEE70AF1EE10FA7E
:106EE80004D5DFED1B7A30EE270AF3E7DFED1A7AD7
:106EF800B4EEE70AF1EE10FA04DD30EE670A37EE79
:106F0800C00A0AE09FED157AB4EEC70AF1EE10FA4E
:106F180044BF30EE270A37EE400A60EE007ADFED14
:106F2800106A9FED107AA7EEA67ADFED0F6AE7EEFA
:106F3800876A9FED0E7AA7EEA67A20EE276AA6EE5C
:106F4800070A70479FED0A0A704700BFDB0F4940E8
:106F5800DB0FC940DB0F49C0DB0FC93FDB0FC9BFDF
:106F68009A7C2E36FAAF4FB93587083CA4AA2ABEB8
:106F780000000000DFED027A30EE270A97E700BF35
:106F8800DB0FC93F38B52DED068B90ED008AB0EECA
:106F9800480A0C460546FFF7EDFFB0EE40AAB0EEF2
:106FA800480AFFF784FFD5ED018AB0EE409AB0EEAB
:106FB800680AFFF7DFFFB0EE408AB0EE680AFFF715
:106FC80076FFD5ED02AAF0EE408AB0EE6A0AFFF726
:106FD800D1FFF0EE409AB0EE6A0AFFF768FF60EE64
:106FE8000A6A69EE297AF0EE665AE7EEA85A29EE9F
:106FF8008A6A29EE007A69EE889A29EE489A28EE7C
:10700800400A28EE0A8AC4ED035AF0EE465AE7EE23
:10701800685AE6EEA87AA6EE687AC4ED009AC4ED3E
:10702800028A84ED059A84ED088ABDEC068B84ED0E
:10703800010AC4ED045A84ED067AC4ED077A38BD16
:1070480010B52DED048B8AB090ED009AD0ED028A30
:1070580090ED018A0446084601A9FFF793FFDDED8C
:10706800047A9DED017A68EE277AE9EE077A9DEDBC
:10707800077AE8EE877A9DED027AC4ED007ADDEDB5
:10708800057A68EE277AE9EE077A9DED087AE8EE48
:10709800877AC4ED017ADDED067A28EE278ADDEDE0
:1070A800037AA9EE278ADDED097AA8EEA78A84ED8E
:1070B800028A0AB0BDEC048B10BD074B1A8822EA7D
:1070C8000000904210B518801C4602D0012004F040
:1070D8008DF8208810BD00BF98110020064B1A8833
:1070E8001043904210B518801C4602D0012004F0CD
:1070F8007DF8208810BD00BF98110020024A9368CF
:1071080023EA0000906070474820002008B5104B23
:107118001A780023D9B2914207D20E4951F82310A8
:107128000968002008600133F4E7322003F0C3FE49
:10713800094B1B685A0309D5084B9B685B0305D4A8
:1071480040F2DC50BDE8084003F0B5BE08BD00BF02
:107158006015002030150020E81F0020482000207E
:10716800454A69232DE9F34113704FF4FA635380BC
:10717800BE231371EF2382F8CD37002382F8CE3770
:1071880019461646F25C0133B3F5FA6F81EA02013B
:10719800F8D1394B83F8CE17384B1A69120604D543
:1071A800374A5A6002F188325A6004270020013FAA
:1071B80017F0FF074FD0314B3422DA60002444B176
:1071C800002356F804800193FEF738FE0428EED118
:1071D80017E0FEF733FE0428E9D1284D2B6943F068
:1071E80002032B61274B6B612B6943F040032B6132
:1071F800FEF724FE2B69042823F002032B61DFD05D
:10720800D5E71E4D2B6943F001032B6104F10063A0
:1072180003F57E331FFA88F21A80FEF70FFE042862
:1072280010D1194B23440193019B4FEA1848A3F846
:107238000080FEF703FE2B69042823F001032B616D
:1072480005D0B4E72B6923F001032B61AFE70434C1
:10725800B4F5FA6FB3D1094A1369042843F08003DF
:10726800136102D107F0ECFF10B90A2003F0D6FF32
:1072780002B0BDE8F08100BF482000200020024095
:107288002301674500F8030802F8030810B50E4CFF
:10729800206803F06FFD2068047A002202FB02F3E5
:1072A800193B634303F6C4135343192193FBF1F3CA
:1072B800064921F812300132072AEFD10449BDE806
:1072C800104003F00DBD00BF40100020980F0020B3
:1072D8008C2100202DE9F04107F0B2FF10B90A20F7
:1072E80003F09CFFA34CA449A44D4FF4FA62204636
:1072F8000DF0C4F894F8A437022B84BF002384F857
:10730800A43794F8A4274FF4CC7101FB02F3E018DA
:10731800234400F53770286093F8300303F54A7367
:10732800022801FB024284BF0020187292F8303311
:10733800934A13700C2202FB0343924A03F2A6738A
:107348001360A36846F209021A401AB9894A43F43D
:1073580000539360A368D80703D54FF40050FFF794
:10736800CDFEA368590409D50820FFF7C7FE4FF4DE
:107378000050FFF7C3FE0120FFF7C0FEA3681A07FD
:1073880006D54FF40050FFF7B9FE0120FFF7B6FE0F
:10739800A3689B0406D54FF48030FFF7AFFE40206A
:1073A800FFF7ACFE94F8DC21724B2AB193F8E02188
:1073B80012B1002283F8E021734B744E1E604FF027
:1073C800000C674604EB0C03B3F8F4E14FEA5E01E6
:1073D80001F077314FEA9E0303F03333C1EB0E001F
:1073E800C11A4FEADE0303F01133CB1A03EB231360
:1073F8001EF0010803F00F324FF0FF0392FBF3F386
:10740800C3EB032318BF0137A2EB030318BFFFB276
:10741800012B0ADD022B40F0AA80B8F1000F00F022
:10742800A6801EF0BC0F00F0A2800CF1080CBCF185
:10743800180FC7D1013F012F00F29980FFF726FFEF
:10744800302200215248534F0DF023F8524BD5F803
:1074580000801F60514B002108F17900C3F80080BB
:1074680003F0C8FC4E4B80F0010018704D4B07F13B
:1074780026021A604C4B07F1C8021A6098F80000FF
:1074880004F04EF92868494B00F5C5721A6004F0FB
:1074980081FE474BDFED476A07F194021A60464BBD
:1074A80000221A809A71454B07F12C021A602B684A
:1074B800434A93ED187A03F219111160414A03F215
:1074C80089111160404A07F1080111603F4A1760AD
:1074D8003F4A07F19C0111603E4A07F1A60111607D
:1074E8003D4953610E6067EE266AB4F866119361F0
:1074F800B6EE007A07EE901A87EE267AB4F868118D
:107508005762101DF8EE677AC2ED027A07EE901AFC
:1075180093F85C10117193F87810517194F8DF1199
:107528001174F8EE677AB3F81611C2ED037A07EE14
:10753800901A2A4908602A4903F164000860294919
:10754800F8EEE77A81ED007A9FED277A2749C7EEB2
:10755800277A9FED277A67EE877AC1ED007A03F1E3
:10756800680103F21113D1611362BDE8F081FEF7DF
:1075780031FC63E74820002000F8030820100020B1
:10758800941F002040100020C42B0020D22100208E
:10759800CC0E00208C210020000F0020040F0020BA
:1075A80010000020D40600205C060020100F0020E8
:1075B800B80E0020DB0F4940040E00202C070020E5
:1075C8001C1D0020340900207C1600208016002095
:1075D80048080020501300200C0900205C070020F8
:1075E8009407002090070020000061444408002010
:1075F8004C3D0F4408B5FFF7B3FDFFF76BFE0120C4
:10760800BDE8084003F0F2BD2D4B2E4A1B681268F6
:1076180010B51A602C4A1168596051689268DA608E
:107628002A4A996011681961516892689A61284AD2
:1076380059611168D961516892685A62254A19627C
:1076480011881985518859859188D288DA85224A06
:107658009985118819865188598692889A861F4A71
:107668001188D986518819871946928821F83A2FA6
:107678001B4A10780022824206DA1A4C34F812406B
:1076880021F8024F0132F6E7174A1288A3F864205E
:10769800164A1288A3F86620154A1188A3F86810BC
:1076A80051889288A3F86C20124AA3F86A101288AD
:1076B800A3F86E20104A5289A3F85E2010BD00BFBF
:1076C80098280020DC2B0020001400200C14002037
:1076D80018140020B410002004100020AA10002064
:1076E8006015002024100020C0120020BC0F0020CC
:1076F8000A1000203C100020101000202DE9F8434B
:107708000E4B93E8800305460E460024B44213DA74
:107718007B1933F9140008EB050333F9142009EB3E
:10772800050333F914301344022293FBF2F3C01A11
:1077380008F027F90134E9E7BDE8F8839828002024
:1077480070B5472008F06CF8174B1B681B0307D56A
:10775800164B174A5B6810681B68C01A08F002F9D4
:10776800144E154C154D307808F0FCF8236828683D
:10777800C01A08F006F963686868C01A08F001F9C9
:107788000F4B188808F0EEF80E4B188808F0EAF846
:107798000D4B188808F0E6F8337823742B68A3603B
:1077A8006B68E36070BD00BFF829002098280020AE
:1077B800DC2B0020DA10002084280020DC100020B8
:1077C800D8100020D6100020441000207FB5254C8A
:1077D800254E264D2649274A274B20B127480088A1
:1077E800B0F5805F30D23088ADF8040028781D4DA0
:1077F800897912788DF806008DF807108DF8082021
:107808001B788DF8093001A8294606220CF026FEBF
:1078180028B30198BDF808302860AB80532007F0E2
:10782800FFFF208808F09EF8A07808F09BF8E3781E
:1078380001932379029301A86379039307F0F8FF72
:107848000E4B00221A800AE0308820808979287837
:1078580012781B78A070E17022716371DEE704B0C2
:1078680070BD00BF7813002098110020D4100020AC
:10787800040E0020330E0020980E0020182A002045
:10788800A0F17D03012B70B504460D460A4E05D8BC
:1078980030687D2103F008FD84F02004306821461B
:1078A80003F002FD35B12B881C4404EB142404F0CA
:1078B800FF042C8070BD00BF881100200A4A13887D
:1078C80001331380094A136801331360084A138887
:1078D80001339BB2202B01BF00231380054A138874
:1078E80008BF013313807047182A0020002A00209F
:1078F800042A0020062A002038B53A4B1B78083B9A
:10790800012B05460C466BD8452007F089FF284611
:1079180007F086FF0C2D23D004D80A2D0AD014D8DE
:1079280035B138BD0E2D4BD02ED3FF2D50D038BDDC
:10793800206849E0207807F073FF62796378002AAD
:1079480014BF80200020184300E0207807F068FF6B
:10795800A07807F065FFE07807F062FF20793BE048
:10796800B4F9000007F0F4FFA07807F059FFE078B9
:1079780007F056FFB4F9040007F0EAFFB4F906006F
:10798800BDE8384007F0E4BF637820788BB180F019
:10799800800007F045FFA468E0B207F041FFC4F398
:1079A800072007F03DFFC4F3074007F039FF200E1A
:1079B80012E007F035FF6068BDE8384007F0E1BF26
:1079C800206807F0CFFF6068BDE8384007F0CABFFD
:1079D800054807F003FF0020BDE8384007F020BF46
:1079E80038BD00BF742800205A8301082DE9F04FE4
:1079F800B84BB94F1A888BB00193002A40F09D808C
:107A0800B7F8CA07B54E42F20103C41A6042604192
:107A1800FFF7DCFEFFF7F8FD3468492007F000FFA8
:107A2800AF4B2546186807F09DFF55F8040B07F083
:107A380099FF2846FEF780F904F11000FEF77CF95B
:107A480004F11C094FF01008A64D01232A6803FA17
:107A580008F3134203D0D9F8000007F092FF08F1A9
:107A68000108B8F1130F09F10409EDD104F1280058
:107A7800FEF752F9B7F84431B4F92E00C01A07F0EE
:107A880071FF2B68D90408D5974BB4F864001B889C
:107A9800181AC0F30D0007F065FF2B689A0403D588
:107AA800B4F8660007F05EFF2B685B0503D504F1A8
:107AB8006800FEF731F92B68180403D5B4F86E0096
:107AC80007F050FF04F13000A046FEF725F904F155
:107AD8003600FEF721F9B7F8443138F93C0FC01ADF
:107AE80007F040FF0127814B1B789F4208DA38F9DD
:107AF800020FB4F93C30C01A07F043FF0137F2E730
:107B08002B68990505D5B4F95E00A0F2DC5007F0A2
:107B180038FF326876487260B260121A1111754ADD
:107B28004A43531C032293FBF2F202EB42029A1AD5
:107B3800702303FB02033360C0E16F4B6F4A1B687D
:107B480011688B4206D00AA9002041F8203D136035
:107B5800FFF7D2FE019B97F8CA171B8897F8CB0747
:107B68000B44013BB3FBF0F200FB12338B4280F075
:107B780070815A4F0120FFF729FEFFF745FD50207D
:107B88003E687D6807F04CFEBA683B6810681B6861
:107B98007A6803441068A3EB400007F0F2FE6A68B5
:107BA80073689B1A0293AA68B3689B1A0393EA68DE
:107BB800F36802A89B1A0493FEF7BEF82A69336992
:107BC8009B1A02936A6973699B1A0393B369AA693A
:107BD80002A89B1A049307F02BFE06F11C0B05F173
:107BE8001C0810243F4901220B68A2401A428A4609
:107BF80006D0DBF80000D8F80030C01A07F0C1FE44
:107C08000134132C0BF1040B08F10408EAD106F136
:107C1800260005F12601002331F9024F30F9022F21
:107C2800121B02AC44F823200133042BF4D10321A6
:107C38004FF000094FEA89035FFA83F902AB53F862
:107C480021206AB102F108000F2802D849F0010981
:107C580006E08032FF2A94BF49F0020949F003097F
:107C680011F1FF31E6D2484607F0DAFD00240DF1A4
:107C7800080BA04609F00302022A16D0032A1DD0D9
:107C8800012A4ED1B8F1000F05D1DBF800402401DC
:107C9800E4B2904645E0DBF8000000F00F00204316
:107CA80007F0BEFD4FF000083BE0B8F1000F0CD024
:107CB800DBF80000C0F3031020432CE0B8F1000FFC
:107CC8001ED19BF8010007F0ABFD9BF8000007F000
:107CD800A7FD26E0042A002048200020982800203C
:107CE800002A0020F8290020F4290020601500202F
:107CF800A4280020B76DDBB60C2A0020082A002033
:107D0800DBF80000C0F30330204307F089FDDBF8FF
:107D18000000C0F3071007F083FDDBF800402401E2
:107D2800E4B20BF1040B06AB9B454FEA9909A1D1CC
:107D3800B8F1010F02D1204607F072FDDAF8001001
:107D480011F480541FBFB6F86430B5F864209B1A4C
:107D5800029318BF01248A040AD50AAB03EB8402F4
:107D6800B5F86600B6F866301B1A42F8203C0134B4
:107D78004B0513D502AB03EB840C06F1660E05F137
:107D8800660000233EF9022F30F9028FC8EB020289
:107D98004CF823200133032BF4D1033408040BD50A
:107DA8000AAB03EB8402B5F86E10B6F86E305B1AB6
:107DB80042F8203C013400E0FCB1012C03D10298C8
:107DC80007F0DFFD19E0631E002002AA400052F808
:107DD8002320C0B20AB140F00100013BF5D507F0FD
:107DE8001FFD4FF0000802AB53F8280008B107F058
:107DF800C8FD08F10108A045F5DB30200321FFF795
:107E08007DFC36200321FFF779FC2F4B3C201978A5
:107E1800FFF774FCDAF80030990506D5B6F95E006C
:107E2800B5F95E30C01A07F0ACFD3A6827487B68A0
:107E38007A60121A1111264ABB604A43531C032266
:107E480093FBF2F202EB42029A1A702303FB02033D
:107E58003B60204B1B681A0630D51F4C1F4D22680B
:107E68002B689A420BD162686B689A4207D1019BD2
:107E78001B88102B11D11A4B1B885B060DD148208B
:107E880007F0CEFC206807F07CFD606807F079FDFC
:107E980023682B6063686B600EE0124A0F4B117801
:107EA8002A7C914208D1104A99681068884203D107
:107EB8005268DB689A4201D0FFF742FC07F080FC69
:107EC8000BB0BDE8F08F00BF60150020A42800208B
:107ED800B76DDBB6E81F002048100020842800207A
:107EE800062A0020DA100020DC1000202DE9F84FC7
:107EF8000C9E3A4CC2EB030B0B9BF61A63680029E5
:107F080014BF4FF0060A4FF0040A013305469046A5
:107F180013D1236853455ED2314A324852F82320A0
:107F2800032B98BF294607F069FC63680133636037
:107F38002D4B002205469A7113E0002511E02B4ACB
:107F48001278954240DA0B9BE3B109FB06F2995C83
:107F580001228A40264909680A4213D1636801331D
:107F68006360D4F804900A9B1C4F9945E7DB2BD13A
:107F78000A2007F055FC3B6801333B604FF0FF33A4
:107F88007B6021E0184A917921B12C2007F048FC48
:107F9800013501E001219171226809FB0BF308EB1F
:107FA800030752B958F8030007F018FC97F90410B2
:107FB8004B1C0544D2D00F4802E03A440E481179D0
:107FC80007F01CFC0544C9E7206850452CBF002079
:107FD8000120BDE8F88F0020BDE8F88F102A0020A6
:107FE8001464010865830108781300201C0100202F
:107FF800F8290020748301080F8E010830B585B078
:1080080004AC002524F8025D0091ADF80600214675
:108018001020FFF735FC9DF806002146FFF730FCDD
:108028009DF807002146FFF72BFC9DF8000021462C
:10803800FFF726FC9DF801002146FFF721FC9DF87B
:1080480002002146FFF71CFC9DF803002146FFF7BC
:1080580017FC9DF80E00C043C0B22946FFF710FC7C
:1080680005B030BD10B5054C206803F01AF918B1F9
:10807800206803F013F9F6E710BD00BF581100207F
:1080880013B5044601A9006809F0A8F8132009F0FF
:10809800E1F8BDF9040009F0CBF81B2009F0DAF883
:1080A800BDF9060009F0C4F8232009F0D3F82368C5
:1080B800002BB4BF53204E2009F0BAF801A960681C
:1080C80009F08CF8122009F0C5F8BDF9040009F090
:1080D800AFF81A2009F0BEF8BDF9060009F0A8F8B3
:1080E800222009F0B7F86368002BB4BF5720452059
:1080F80009F09EF802B010BDF8B504460E461746C2
:108108000025204620210CF0FAF90446D0B10134AC
:1081180020460CF059FAB0F5617F05DB40F63403D0
:108128009842A8BF184601E04FF46170A0F561704D
:10813800192390FBF3F00DB9307000E070703B78B4
:1081480001333B700DB90125DBE72046F8BD30B59A
:1081580005460C461346294622460248BDE83040EB
:10816800FEF777BE688401087FB504780646E4B94F
:10817800354B1B6803EB8403192193F87B0093F8B4
:108188007C6093F8792093F87A304FF4617511FB8D
:10819800005011FB0651009001912C4821460134F2
:1081A800FEF757FE142CE3D14BE00CF00DFA132820
:1081B800054641DC244B701C1C68202100238DF8E7
:1081C8000F300CF09CF91E35064670B1013630466A
:1081D8000CF0FAF919289FBF04EB850358709DF835
:1081E8000F30013398BF8DF80F30304620210CF046
:1081F80086F9064670B1013630460CF0E5F90D28CF
:108208009FBF04EB850398709DF80F30013398BF2A
:108218008DF80F3004EB85043046E11C0DF10F0298
:10822800FFF76AFF9DF80F30042B0AD0601C00216D
:1082380004220CF02EF904E0054800211322FFF770
:1082480086FF04B070BD00BF20100020878401089D
:108258009C840108014806F00FBE00BFA2840108F3
:108268002DE9F04304788FB00546002C59D17B4B9B
:108278000021142209A807AED3F800800CF009F9F0
:108288000722304600210CF004F905A80023A700B6
:10829800059308EB070583801A467149B5F802E093
:1082A80031F813C01CEA0E0F0AD00DF1380C0E314C
:1082B80002F1010E6244595C02F81C1C5FFA8EF24E
:1082C8000133072BE9D100210B46664AB5F802E0D5
:1082D80011F802C01CEA0E0F0AD00DF1380C063254
:1082E80003F1010E63448A5C03F8242C5FFA8EF3D1
:1082F80001310629E9D118F807305B498DE84100BA
:108308006A78029209A81A0903F00F0307F0C6FD5C
:108318002146564809AA0134FEF79BFD202CA6D118
:1083280098E00CF051F91F28044600F3868028468F
:108338002021E4B20CF0E3F81F2C02D9FFF78AFFE2
:1083480088E0464B1B6803EB8404451C002120464B
:1083580004220CF09EF80027454B09AE3046002158
:108368000A2217F803905FFA87F80CF092F80023B6
:1083780015F8012B32B10A2B04D04A4502D0F25429
:108388000133F5E74A455ED108F1FF33032B09D8DD
:10839800DFE803F01005023F0DF1230134E00DF191
:1083A80023011EE030460CF00FF92378C0B243EAEF
:1083B800001006E030460CF007F9237800F00F00B3
:1083C8001843207031E00133062B0AD0244800F10D
:1083D8001B069E5D9642F6D103445A7D638813437B
:1083E800638011F8012F02B30023EFE70133072B55
:1083F8000AD01B4800F10E069E5D9642F6D130F871
:10840800132063881343638011F8012F6AB1002396
:10841800EFE730460CF0D8F80F2804DC30460CF0B3
:10842800D3F8607001E0002363700137052F93D102
:10843800012405F053FF6CB980E70E4800211F2284
:10844800FFF785FE06E02046002104220CF021F803
:108458000024EEE70FB0BDE8F08300BF80130020D2
:108468002C64010841640108B0840108BF84010834
:108478004D6401089C840108F8B50478064674B96F
:10848800304DB5F8C621B5F8C8312F48214601341A
:10849800FEF7DFFC042C05F10405F2D1F8BD2B49E9
:1084A8000CF000F8A8B9274B4FF47A714FF4FA6230
:1084B800A3F8C611A3F8C821A3F8CA11A3F8CC21C0
:1084C800A3F8CE11A3F8D021A3F8D211A3F8D42190
:1084D800F8BD30460CF078F8032805462BD830460E
:1084E80020210CF00CF8044630B1013420460CF081
:1084F8006BF80126074600E00646204620210BF0CF
:10850800FEFF10B9BDE8F840A4E601300CF05CF8B5
:10851800012EF7D1A7F2EE2240F2DC539A42F1D8AD
:10852800A0F2EE229A42EDD8064B703503EB850394
:10853800DF801881F8BD064800210322BDE8F84015
:1085480005E600BF48200020CB840108DE8401082E
:10855800A19001082DE9FF4104780546002C39D186
:108568007348744D06F088FCD5ED057AF5EE407A2F
:10857800F1EE10FA00F0D88021466F48FEF769FC4A
:1085880095ED050A6846FEF7F9FA01466B48FEF7CD
:1085980060FC95ED060A6846FEF7F0FA0146674862
:1085A800FEF757FC95ED070A6846FEF7E7FA01461D
:1085B8006248FEF74EFC95ED080A6846FEF7DEFABB
:1085C800013401465E48FEF744FC0C2C05F1100509
:1085D800CAD1A9E05B4905220BF0A8FF40B9554B69
:1085E80003F1C0020021596110339342FAD19BE094
:1085F8002846554904220BF099FF04462846002CCA
:1086080040D120210BF07BFF002800F08D80451C15
:1086180028460BF082FF07464C4B53F824601EB9DE
:108628004B4806F029FC7FE028463146FAB20BF0A9
:108638007DFF01340028EFD13E4B03F1C0029E4676
:108648000021596110339342FAD1424B03EBC40223
:108658009846D2F804C0BCF1000F04D131463E4818
:10866800FEF7F7FB57E0002718F834309F42F5DA99
:108678003B010EEB030563440FCB143585E80F006F
:108688000137F1E70BF0A0FF0B28064647DC284628
:1086980020210BF034FF054650B101352846FEF77E
:1086A800E3F9244B03EB061383ED050A012400E0EC
:1086B8000446284620210BF022FF054648B1013523
:1086C8002846FEF7D1F91B4B03EB061383ED060A88
:1086D8000134284620210BF012FF054648B1013528
:1086E8002846FEF7C1F9134B03EB061383ED070A7F
:1086F8000134284620210BF002FF10B9FFF7AAFD2C
:1087080012E00130FEF7B0F90A4B032C03EB061612
:1087180086ED080AF2D11148FFF71CFF04E0104863
:1087280001210C22FFF713FD04B0BDE8F08100BF62
:10873800E484010848200020FF8401080585010819
:10874800F78D0108DE84010809850108006C01081D
:108758000E850108988301081D850108EA81010832
:108768009C840108F0B5047887B006461CBB514BC1
:108778001968062303FB0411192091F8CA5091F8CF
:10878800CB7091F8CE2091F8C9304FF4617610FB88
:10879800056510FB07600095019091F8CC000290E8
:1087A800C83145484979039121460134FEF751FB08
:1087B8000C2CDCD17CE00BF007FF0B28044672DCA4
:1087C8003C4B701C1D68202100238DF817300BF0DE
:1087D80096FE064680B1013630460BF0F5FE0328BA
:1087E8009FBF062303FB045383F8CE009DF8173080
:1087F8009CBF01338DF81730304620210BF07FFEE7
:10880800074680B1013738460BF0DEFE0D289FBFC2
:10881800062303FB045383F8C9009DF817309CBF57
:1088280001338DF8173006266643A9193846CA3130
:108838000DF11702FFF760FC20210BF060FE0746E0
:1088480070B1013738460BF0BFFE14289FBF9DF862
:1088580017307619013386F8CC0098BF8DF8173099
:10886800384620210BF04BFE78B101300BF0ACFEFE
:108878000D289FBF062303FB045383F8CD009DF802
:1088880017309CBF01338DF817309DF81730062B31
:108898000ED0062202FB04500021C9300BF0F9FD6E
:1088A800FFF7D8FC04E0054800210B22FFF74FFC36
:1088B80007B0F0BD20100020298501089C8401081C
:1088C800F0B5027887B0AAB94C4C04F118064C4BA5
:1088D80094F9F21193F900208A4272D093F90C208E
:1088E8008A426ED093F918308B426AD00834B44269
:1088F800EDD180E0002204920592451C0BF064FE45
:10890800C4B260B202F0A6F9074618B18DF810405B
:10891800012400E00446284620210BF0F0FD05461E
:1089280038B1013528460BF04FFE0134ADF812007E
:10893800E4B20026284620210BF0E1FDB0B3451C27
:1089480028460BF041FE00222E4951F8223083427E
:108958005FFA82FE04D00132082AF5D1002300E034
:10896800734651F82320824220D1022E0FD0032EC5
:1089780012D05A1E012ED2B204D0042A13D88DF870
:1089880014300EE0042A0ED88DF8153009E0052BB6
:1089980009D88DF8173004E09A1E052A03D88DF8F7
:1089A80016300134E4B20136042EC3D1052C03D8A5
:1089B80007B0BDE8F0404DE404AB03CB3860796004
:1089C80019E094F8F7010F4B94F8F65153F820008A
:1089D800B4F8F421009094F8F90153F820000190BC
:1089E80094F8F80153F82000029053F8253006480F
:1089F800FEF72FFA7AE707B0F0BD00BF4820002045
:108A080054120020F0630108498501082DE9F3415B
:108A1800047880464CB9204601A9FDF73FFA013495
:108A2800FFF7F4FF122CF6D16BE00BF0CDFDC6B2C8
:108A3800112E61D8344C06F1D00704EB470308F136
:108A4800010020219D780BF05AFD18B9AA1E554245
:108A5800554139E04378682B06D0732B07D0612B3A
:108A680013D14FF0000804E04FF0010801E04FF087
:108A78000208A8F102035D4200F101004FF0200155
:108A88005D410BF03CFDD8B115B9FFF7E3FB38E0C9
:108A980001300BF099FD40F2ED2380B2984205DDDC
:108AA80040F6CA039842A8BF184601E040F2EE20FB
:108AB80004EB4703A0F2EE20192290FBF2F0D870E5
:108AC80004EB470383F8028004EB47040F4AA378BA
:108AD800134493F8262055B1E3780D4840F2EE246C
:108AE8001925314605FB0343FEF7B3F909E0314682
:108AF8000848FEF7AEF904E0074800211122FFF705
:108B080026FB02B0BDE8F081482000202C64010853
:108B1800688501087A850108A190010807B5012335
:108B2800ADF8041001A98DF806208DF8073004F07F
:108B3800EBFE03B05DF804FB2DE9F843404B414CD4
:108B48009A6A42F400129A629A6A22F400129A62AD
:108B58005A6942F400125A6106464FF4A061204651
:108B68000122FFF7DBFF4FF4A063238572B6364D71
:108B780002214FF00809298528460422A5F82890E3
:108B8800FFF7CCFF284601224946FFF7C7FF2F48C9
:108B980050F8364000EBC6002368426801265700AB
:108BA80006FA07F848EA030396402360A661C5F869
:108BB80018902B8A9B07FCD4236848EA0303236098
:108BC800214B0822B1B221851A854FF48072A3F88F
:108BD80028284FF48062C3F8182840F605531A482D
:108BE800028A950711D4013BF9D122680323BB40BF
:108BF80022EA0303236008210222FFF78FFF62B6EF
:108C08003220BDE8F84302F056B90422A661204696
:108C1800FFF784FF0B4B4FF480621A850A4B1A8AC0
:108C28009207C9D5228A92B21642064A4FF0080026
:108C38004FF4807115BF9861188511859161EDE732
:108C48000010024000100048000800488C85010808
:108C580010B50446204602F01BFB18B90A2002F0A2
:108C68002AF9F7E710BD0C4B5A6882421A4607D01A
:108C78001B69834206D0D36983420BD1022302E0E9
:108C8800002300E001230021C1620C2000FB032324
:108C980019725960704700BF5412002013B506229C
:108CA80004466B4603211E2004F044FF9DF8002073
:108CB8009DF801309DF8021043EA02231BB21B4ABB
:108CC80007EE903A92ED007AF8EEE77A67EE877A47
:108CD80092ED027AFDEEE77A17EE903A23809DF83E
:108CE800033043EA01231BB207EE903AF8EEE77A25
:108CF8009DF8041067EE877A92ED017AFDEEE77A27
:108D080017EE903AA3809DF8053043EA01231BB281
:108D180007EE903AF8EEE77A67EE877AFDEEE77AA3
:108D280017EE903A638002B010BD00BF80000020AB
:108D380013B506220446A82119206B4604F0FAFE52
:108D4800F0B19DF800309DF8012043EA022202218B
:108D58009DF8033012B292FBF1F222809DF80220B6
:108D680042EA032212B29DF8053092FBF1F26280CA
:108D78009DF8042042EA03231BB293FBF1F3A3807E
:108D880002B010BD08B524218022192004F04EFF3E
:108D9800642002F090F820219722192004F046FF61
:108DA8000A2002F088F810222321192004F03EFF3F
:108DB800642002F080F8024B4FF480521A8008BDFC
:108DC800120000202DE9FF41634B1B6893B11A681C
:108DD8001AB16249486902434A619A88ADF8042089
:108DE80002228DF807209868002201A98DF8062034
:108DF80004F08AFD322002F05EF8002111221E20C4
:108E080004F014FF012160221E2004F00FFF6420EB
:108E180002F051F802A8FFF741FF00240A2726466E
:108E28002546022101221E2004F000FF322002F014
:108E380042F802A8FFF732FFBDF90820BDF90A1071
:108E4800BDF90C308A421444A8BF0A4693421D4417
:108E5800A8BF134613F5805F0E440ADD404A938A83
:108E68009BB283F48843013F9382DAD14FF0010823
:108E780001E04FF000081E200021122204F0D6FE67
:108E88000A27022101221E2004F0D0FE322002F01F
:108E980012F802A8FFF702FFBDF90820BDF90A1071
:108EA800BDF90C308A42A4EB0204A8BF0A469342DB
:108EB800A5EB0305A8BF134613F5805FA6EB0106D3
:108EC80008DD274A938A9BB283F48843013F938243
:108ED800D7D101E04FF0000807EE904A9FED217AC4
:108EE800214FF8EEE77A0021C7EE277A70221E207C
:108EF800F0EEE77AC7ED007A07EE906AF8EEE77AC7
:108F0800C7EE277A9FED197AF0EEE77AC7ED017A76
:108F180007EE905AF8EEE77AC7EE277AF0EEE77A8E
:108F2800C7ED027A04F082FE012120221E2004F0FF
:108F38007DFE1E200221002204F078FE642001F04C
:108F4800BAFFB8F1000F04D14FF07E533B607B604D
:108F5800BB6004B0BDE8F0810C03002000100240A3
:108F68000010004800406F468000002001C05E46A7
:108F7800154B37B5082205461A85E82006F008FD86
:108F88000024002006F004FD0DF804000134062C2E
:108F9800F7D10D4B08229A619DF800209DF8013009
:108FA80043EA02232B809DF802209DF8033043EA10
:108FB80002236B809DF804209DF8053043EA0223C4
:108FC800AB8003B030BD00BF001000482DE9F04F62
:108FD800944D954C2B68954E9BB2238022883188FE
:108FE8000A40900585B007D54FF6FF53904A2B608D
:108FF80013780133DBB2137023880B40190440F156
:1090080043830023ADF80A302B6887499AB21804C5
:10901800228040F139830B8803F00F038B70002BFB
:1090280040F00483834A844F136884489BB23B8092
:109038003B8803F0300303803B8803F440533B80B4
:10904800D2F800E04BF6BF730EEA030383F4005333
:1090580083F0200343F4004343F0800313600B883C
:1090680013F0100F804626D1116848F60F730B4095
:10907800734913600B681A7A022A894601D0042AB8
:1090880005D1FCF7BDFFD9F800301B7A3FE1062A6D
:109098006ED15A78052A09D11A78520606D1D8789D
:1090A800FCF792FF674B1B681B6A9847664B1B6867
:1090B8009B6898475CE013689BB2ADF80A30BDF82E
:1090C8000A301B0540F1F38111685D4840F68F7343
:1090D8000B405E4913600A685D4B92B213445B0013
:1090E80081461A68036893F808E0BEF1090F8A46BA
:1090F80017D092B2520002F1804202F5C0421178B4
:109108001970517859709188C8B2090A41EA00214A
:1091180059801189C8B2090A41EA002199809289C7
:10912800DA8001221A72DA8893F801B0002A40F036
:10913800F1801A7812F07F0250D1BBF1090F10D1DB
:10914800DA78012A00F2CA809978002940F0C680AE
:109158009988002940F0C2809A723A4B1B685B6874
:10916800BAE0BBF1050F10D193F90320002A01DA08
:109178000823CCE09A78002AFAD19A88002AF7D1F5
:109188009B7A002B00F0B480F2E7BBF1030F0FD1FC
:10919800DA78012A40F0A2809A88002A40F09E805E
:1091A8005A7A42F020025A72264B1B68DB6993E018
:1091B800BBF1010F40F09280DA78012A40F08E80EE
:1091C8009A88002A40F08A805B7A980640F1868067
:1091D800FCF7C4FF002800F08B807FE0012A39D11A
:1091E800BBF10B0F7AD1184A58791268D97892696D
:1091F8009047D9F800309A7A002A6FD000286DD1AC
:109208001A79002A6AD19B78002B67D10D4B1B680D
:10921800DB6898470A4B1B685A79DA72DA781A734E
:1092280066E000BF445C0040841300201C2A002034
:10923800FF2B0020005C00407A12002078120020EA
:10924800A4110020A811002018150020505C00402F
:1092580004300020022A41D1BBF1010FB8D0BBF184
:10926800030F3BD1587920F0800E4FEA8E0202F1AD
:10927800804101F5B84110F0800F096814BF01F072
:10928800300101F44051BEF1030F27D8B3F802E0D2
:10929800BEF1000F22D109B39B7AFBB102F18042E3
:1092A80002F5B842010613684BBF23F4E04323F4E8
:1092B800804323F0400323F070034BBF9BB29BB263
:1092C80083F0100383F4805343F4004343F0800396
:1092D8001360A94B1B689B69984709E0A74B1B685B
:1092E80058465B699847032810D000287FF440AFA0
:1092F800DAF80020A24B92B213445B001A680022ED
:109308001A603023A8F80030062300E00923D9F8B2
:10931800002065E1BBF1060F13D11A7850067DD104
:109328009A78964B012A02D11B68DB696AE0022A07
:1093380002D11B681B6A65E0032A6FD11B685B6A50
:1093480060E0BBF1000F3AD15988002966D15A680C
:1093580022F47F42B2F5003F60D11A7812F07F0202
:1093680004D19B88002B00F0F48157E0012A0AD130
:10937800824A587912689269904700284ED1D9F8E4
:1093880000309B7A17E0022A48D15A7902F00F017F
:109398000BB29B0003F1804303F5B84312F0800F32
:1093A8001B6814BF03F0300303F44053032935D876
:1093B80012F0700F32D1002B40F0CB812EE0BBF1C0
:1093C800080F04D11B78590600F0C58126E0BBF1CF
:1093D8000A0F23D11A7802F07F02012A1ED19A7A45
:1093E800E2B15988D1B95A6822F47F42B2F5803F78
:1093F80014D1624A5879126892699047002800F09F
:10940800AC810BE053B1D9F800204FF0000AA2F864
:1094180012A093615046984750460BE0574BD9F835
:1094280000201B6850781B699847032802D1554BC8
:109438001B6806E0D9F800301A8A4FF6FF718A4295
:1094480001D1092203E0022800D012B908221A72B9
:10945800C7E093F90010002923DAD988039103980B
:10946800DFF818E1824202D9039A1A8211E08A428F
:109478000FD2DEF8001091F82C00824201D20021B0
:1094880005E092FBF0F100FB112212B901213E4ADE
:109498001170DEF8002092F82C209A82FCF7B0FDBB
:1094A8009FE003221A724FF440533B8099E0BDF8C5
:1094B8000A301BB2002BBFF6A7AD116840F68F73B8
:1094C8000B4013602F4AD2F8009099F80830022B0D
:1094D800934600F08280042B7FD0032B01D0052B0C
:1094E80075D1D9F81830B9F810209BB9B9F81020FF
:1094F800002A4FD04FF440533B80244B1968204B2F
:1095080089B20B445B001968002119603023A8F860
:1095180000303FE0002AE9D0B9F814A0924528BFEE
:1095280092461FFA8AF2104601929847019AB9F8B2
:1095380010309B1AA9F81030B9F812301344A9F862
:109548001230124B1A68124B92B213445B000AF1A4
:10955800010A1B689BB203F1005303F540534FEA1D
:109568006A0A5B0000215145C0D053F8212020F839
:1095780011200131F7E700BFA811002018150020BD
:1095880002300020A4110020FE2B0020505C004077
:1095980004300020B9F814309342DBF8003001D8C9
:1095A800032201E012B105221A720CE00621197299
:1095B8006C4B19686C4B89B20B445B0019681A60D4
:1095C8003023A8F80030DBF800301B7A06E0072BC0
:1095D80003D1664B1B68DB6898470823DBF800203B
:1095E8001372FCF79FFD624B1A684BF6BF7313406A
:1095F8003A88D2043A8848BF83F480539004B8F874
:10960800002048BF83F40053D106B8F8002048BFB3
:1096180083F01003920648BF83F0200343F400430D
:1096280043F08003524A9BB213602DE09A0002F186
:10963800804202F5B842116889B2ADF80A10BDF847
:109648000A1009B2002909DA106840F68F71014042
:109658001160013B474A52F823309847BDF80A3059
:109668001F067FF5D1ACA1788B0003F1804303F589
:10967800B84348F60F72186802401A603D4B03EB76
:1096880081039B699847BFE42288338813405905B2
:1096980005D54FF6FF332B60374B5B689847228818
:1096A80031880A40920444BF4DF6FF732B6023882B
:1096B800324A0B40DB0452D54EF6FF732B60002371
:1096C800D370D378052B41D8DFE803F0030D1418C5
:1096D800222DA368294D1BB902F03CFE062300E0A9
:1096E8000523EB703BE002F035FE0423E370012311
:1096F800A36034E002232371032328E02379013B8C
:10970800DBB22371237953BB1C4B0422DA7026E0A9
:109718001B4A13689BB243F0100313600523E370E0
:109728000A2323711BE02379144A013BDBB223711E
:10973800237903F0FF0093B911490C684FF6EF73D2
:1097480023400B600623D370906008E00623E37083
:1097580005E00C4B57E60C4B55E60C4B53E605B0B1
:10976800BDE8F08F505C0040023000201815002042
:10977800005C0040186901081C00002084130020C8
:10978800405C0040335C0008D95C0008B95C000804
:10979800704770477047FEE7FEE7FEE7704730B551
:1097A8000024E3B293420DD2030F092B94BF303348
:1097B800373301F8143001EB4403002500015D70D4
:1097C8000134EEE730BD00BF2DE9F04F2DED028BDF
:1097D80085B007460293A04B1B889807934636D559
:1097E800109B9E48DC89B0F900301B1B03F2F3156F
:1097F80040F2E632954203D8002BB8BF5B4201E045
:109808004FF4FA73B0F90220121B02F2F31440F27B
:10981800E630844203D8002AB8BF524201E04FF430
:10982800FA729342B8BF1346C3F5FA73052293FB45
:10983800F2F30A22643B53433A7FD2105343642223
:1098480093FBF2F3134423EAE373DBB200E06423EF
:109858000093CB1C0193B8460024019BDFF824A297
:1098680013F8016F0193022C4FEA440905D1BAF9A4
:1098780004301B365E43761146E079493AF81420E5
:1098880031F91410022012FB0011CBF100029142B1
:1098980003DB59450A46A8BF5A467249029B31F96B
:1098A8000950551B33F91420154406F027FB88B1DD
:1098B80007EE905A6C4AB8EEE70AB2EE048A105DD9
:1098C80080EE080A06F0D6F820EE080AFDEEC07A07
:1098D80017EE905A604A1288D10712D43AF9093023
:1098E8001B365E4393074FEA26160DD5BB7C5D43B6
:1098F8009DF900305D43642395FBF3F506EB2516CF
:1099080002E03E7A75432E11584B042533F909308D
:1099180093FBF5F5564BE25C924698F80120751BCF
:1099280051466A434A43642192FBF1F297F8511079
:10993800D21108EE102AA9B1022CB8EEC80A08D133
:109948004A0803D09142A8BF114600E001214948C6
:1099580002E0181D00EBC400D3ED070AFDF75AF822
:10996800BDEEC08ADFF808E1434B98F80B60188811
:109978000EF1200300FB05F253F82410D21206FB67
:109988000216B6F5001F3D4AA8BF4FF400169642CE
:10999800B8BF16460EF12C0243F8246052F8243062
:1099A80042F82450EB1A0EF138014FF6FF72000905
:1099B800B2FBF0F043430EF1440051F8245050F844
:1099C800242040F824509B112A4441F8243097F869
:1099D80050101A444FEA840C761300EE102A79B11D
:1099E8000EF15000B8EEC00A00EBC400DEED070A25
:1099F800CDF80CC0FDF70EF8DDF80CC0BDEEC00ABE
:109A080098F8153010EE102A18EE101A5A435346DB
:109A180053431A463144642392FBF3F3184A1B124A
:109A2800194422F8091018EE100A02F1080101344D
:109A38004CF8010002F114012032032C4CF80160AB
:109A48004CF8023008F101087FF407AF05B0BDEC0F
:109A5800028BBDE8F08F00BF981100202420002061
:109A6800F62B0020E01F0020506901080410002098
:109A780090130020A4130020D80F00200000E0FF5E
:109A8800F8130020B41000202DE9F04F2DED028BC3
:109A980087B000260593C54B0491B3F90280B3F94A
:109AA80000300392B8F1000FB8BFC8F10008002BCE
:109AB800B8BF5B429845B8BF9846B8F5FA7F0746E5
:109AC800A8BF4FF4FA780090B1460196B3463446E1
:109AD800B74D2B88990758D0B44BB64A33F8143091
:109AE80032F91420022013FB0022039B5B429A42A6
:109AF8004FEA440103DB039B9342A8BF1346AE4AD7
:109B080031F902A0059A32F91420CAEB030303EBDA
:109B1800020A06F0F3F988B107EE90AAA74BB8EE4F
:109B2800E70AB2EE048A185D80EE080A05F0A2FF83
:109B380020EE080AFDEEC07A17EE90AA3B7A64225E
:109B480003FB0AF393FBF2F33A7F6FF0040101FB86
:109B580002FB5B4505DB02EB82029342A8BF13467A
:109B68009B46974A52F824100AEB010342F21071FF
:109B78008B42A8BF0B4693498B42B8BF0B4642F8AD
:109B88002430BA7C53431B1301932D8805F003033B
:109B9800012B38D0854B8C4933F91490009B51F830
:109BA80024E093F801C0894B33F9140080EAE0738C
:109BB800A3EBE073B3F5206F4FEA840616DC09EBDC
:109BC80089031A0192FBFCF3042290FBF2F0181AA5
:109BD8008644BEF57A5FA8BF4FF47A5E7C4B9E45FB
:109BE800ACBF41F824E041F8243002E0002341F8FA
:109BF80024308B597D2693FBF6F6009BDB7A734362
:109C0800402693FBF6F6AA0711D5019BC8F5FA7210
:109C180008FB09F008FB06F54FF4FA7102FB0B008C
:109C280002FB035590FBF1F095FBF1F505E0EB071E
:109C38004DBF019D354648465846644B33F91420BC
:109C4800042392FBF3F3634A02F19C014FEA440AAE
:109C5800615C4B436FF04F0193FBF1F397F85110A0
:109C6800C31808EE103A51B1101DB8EEC80A00EB3F
:109C7800C400D2ED070AFCF7CDFEBDEEC08ADFF8BE
:109C880054E1524B0EF1A0013AF803003AF90130C1
:109C98002AF8010002B20EF1A4010EF1AC00D31AA9
:109CA800042293FBF2F2A30051F824C0029350F867
:109CB800243041F82420634497F8501040F824C019
:109CC800134400EE103A59B10EF15000B8EEC00A34
:109CD80000EBC400DEED070AFCF79CFEBDEEC00AEF
:109CE8003C4A02F1B40110EE103A095D01FB03FE93
:109CF80018EE101A02F1680029444FF0200C9EFB60
:109D0800FCF3C91A2AF80010029902F1700E0846ED
:109D180018EE101A40F80E1002F17C015B42455013
:109D280002F188014350009B013300930CB90124D0
:109D3800CEE61E4B946AB3F90410049B9B790F334B
:109D48005B004B435B112149002BB1F904104FF024
:109D5800040091FBF0F0A3EB0000B8BF5B42322B8C
:109D6800797B0BDC1C4B01FB00418B42A8BF0B46E7
:109D78001A498B42ACBF9362916201E0002393625F
:109D8800F97801FB00F31649097803294FEAA31370
:109D980029D9B7F84E10B1F5FA7F24D24842834248
:109DA80020DB8B42A8BF0B461DE000BFB41000208B
:109DB80098110020F62B0020E01F002050690108B0
:109DC80024140020F0D8FFFFB01300200410002056
:109DD80080C1FFFF90130020FEFFFF0F020000F07C
:109DE800601500200346916A936741F34F31B1F53E
:109DF800807FA8BF4FF480716FF0FF008142B8BF29
:109E0800014658180023A2F86C00C2F88410C2F862
:109E1800903007B0BDEC028BBDE8F08F2DE9F04F14
:109E28002DED028B85B080460393BC4B02911C88B4
:109E3800019204F00204A4B294B1B94BB3F9024000
:109E4800B3F90030002CB8BF6442002BB8BF5B42A6
:109E58009C42B8BF1C46B4F5007FA8BF4FF40074FD
:109E6800C2460025AF4AAE4B32F9152033F815101B
:109E7800AD4882EAE27EAEEBE27E0BB2BEF5206F21
:109E88004FEA45094FEA43034FEA850750F8256032
:109E980012DC4FF0040E92FBFEF29A1A1644B6F545
:109EA8007A5FA8BF4FF47A56A04A9642ACBF40F8F2
:109EB800256040F8252002E0002240F82520C659F8
:109EC8009AF80B20F61156439AF801205343934A07
:109ED80012884FEAA31B93074FEAA61654D0944A58
:109EE800019B32F90920022011FB00215A429142BC
:109EF80003DB8B42A8BF0B461A468E49039B39F9F0
:109F08000110511A33F915208B1808EE103A05F094
:109F1800F5FF68B1B8EEC80A874AB2EE048A80EE47
:109F2800080A505D05F0A6FD20EE080ABDEEC08ABD
:109F3800824883493A5818EE103A42F2107E1A4481
:109F48007245A8BF72468A42B8BF0A463A5098F886
:109F5800081098F81C00594300EB8000C911C0F1A3
:109F6800000E714503DB8142A8BF01468E4698F872
:109F780012104A431213CEEB0B03B61A664363431F
:109F880002EB66260EEB632B664A39F902100422AF
:109F980091FBF2F16B4A02F19C00405D4143ABEB4F
:109FA800A11398F8511008EE103A51B1101DB8EEEF
:109FB800C80A00EBC500D2ED070AFCF72BFDBDEE81
:109FC800C08ADFF880E1574B0EF1B80139F8030079
:109FD80039F9012029F801000FFA80FC0EF1BC01C3
:109FE8000EF1C400C2EB0C023B584FF0040C92FB7C
:109FF800FCF257F801C07A50634498F8501047F8BB
:10A0080000C0134400EE103A59B10EF15000B8EEFA
:10A01800C00A00EBC500DEED070AFCF7FBFCBDEE4D
:10A02800C00A484901F1B40210EE103A525D534398
:10A038005A1118EE103A01F1680E9819801A01F1B8
:10A04800700329F80E0018EE100AF85001F17C038D
:10A058005242FE5001F188030AF1010AFA500B46F8
:10A068000DB90125FEE62E4A9C6AB2F90410029A3F
:10A0780092790F3252004A4352112A49002AB1F903
:10A0880004104FF0040091FBF0F0A2EB0000B8BF01
:10A098005242322A98F80D100BDC2B4A01FB004182
:10A0A8008A42A8BF0A4629498A42ACBF9A62996285
:10A0B80001E000229A6298F8031001FB00F224499B
:10A0C800097803294FEAA2120CD9B8F84E10B1F555
:10A0D800FA7F07D24842824203DB8A42A8BF0A4677
:10A0E80000E00246996A9A6741F34F31B1F5807FE3
:10A0F800A8BF4FF480716FF0FF008142B8BF0146DE
:10A1080050180022A3F86C00C3F88410C3F89020FC
:10A1180005B0BDEC028BBDE8F08F00BF98110020A0
:10A12800B410002004100020B013002080C1FFFFED
:10A13800F62B0020E01F002050690108241400209D
:10A14800F0D8FFFF90130020FEFFFF0F020000F081
:10A15800601500202DE9F04F2DED0A8B85B0834660
:10A16800039390F85030029101921BB1322BA8BF93
:10A17800322300E0012307EE903AF8EEE7BADFED6C
:10A18800DE7ADE4B9FEDDECA1B88C7EEABBA002B2A
:10A1980008BF012307EE903AB8EEE7AAD94B2AEE9A
:10A1A8000CCA1B887BEE8CBA9807CCEE2BBA27D545
:10A1B800D54AB2F90030B2F9022083EAE37182EAA3
:10A1C800E270A1EBE371A0EBE27088420446B8BFED
:10A1D8000C46B4F5E17F16DA88429FEDCCBA05DD6E
:10A1E800002AD8BF524207EE902A04E0002BD8BFBD
:10A1F8005B4207EE903AF8EEE77A87EE8BBA04E016
:10A208009FEDC3BA01E0B7EE00BAC24EDFEDC09AC7
:10A21800CDF800B006F1080806F1100906F11C0592
:10A228000024F0EE69AABC49DFF8D8A231F914304D
:10A23800B54909EE103AB8EEC99AF5EE047A29EE56
:10A24800279A31F91430BAF80010BDEEC99A08EE11
:10A25800103AF8EEC97A9FEDB19A89074FEA440798
:10A2680027EE899AB8EEC88A00F08180AC4931F9A6
:10A27800143007EE903AF8EEE77AB0EE007AE8EE9E
:10A28800077A019B5842FDEEE77A17EE901A814251
:10A2980003DB8B42A8BF0B461846A249039B795E95
:10A2A800401A33F91410084407EE900AF8EEE78ACA
:10A2B80005F024FE48B19C49F2EE049A88EEA90AFA
:10A2C800085D05F0D7FB60EE298A9BF81C30DFEDAE
:10A2D800976A0AEE903A9BF8083007EE903AF8EE43
:10A2E800677AF8EE6AAA68EEA77AB1EE047A67EEA2
:10A2F800A67A2AEE877AFDEEE77A17EE901AF1EE43
:10A30800477AFDEEE7AA1AEE903A994208DBFDEE8D
:10A31800C7AA1AEE903A8B42A8BF0B460AEE903AAB
:10A32800D5ED007AE8EE8C7ABBEE0E7AF4EEC77AB9
:10A33800F1EE10FAF8EEEAAA09D4B3EE0E7AF4EECA
:10A34800477AF1EE10FAC8BFF0EE477A01E0F0EE76
:10A35800477AC5ED007A9BF8123009EE903AF8EE8C
:10A36800699A67EEA97ADFED729A67EEA99ABAF848
:10A378000010CA0753D46848385E0028B8BF404266
:10A38800B0F5206F03DD0020C9F8000026E0009B2F
:10A398009FED687A5B7868EE077A07EE103AB8EEB8
:10A3A800477A87EE877AD9ED007A37EE497AE7EE71
:10A3B8000C7A9FED617AF4EEC77AF1EE10FA09D4BF
:10A3C8009FED5E7AF4EE477AF1EE10FAC8BFF0EE30
:10A3D800477A01E0F0EE477AC9ED007A009BD9EDA3
:10A3E800007ADB7A08EE903AF8EE688A8B0768EE16
:10A3F800A77ADFED538A67EEA88A14D538EE6A8A01
:10A40800F0EE6A7AEBEE087A78EEE98AB0EE678ABF
:10A41800F0EE697AEBEE287AF0EE678A03E0F0EE68
:10A42800698AB0EE6A8A474B9FED477A03F19C012F
:10A43800625C9BF8511007EE902AF8EEE77A67EE17
:10A44800C97AA7EE878A51B1181DB0EE480A00EB09
:10A45800C400D3ED070AFCF7DDFAB0EE408A96EDAA
:10A46800007ADFF8E0A0D8ED007AA6EC019A39EE80
:10A47800477A0AF1B40187EE0C7A635C09F10409A2
:10A48800043509EE103A37EE677AB8EEC99AEBEE62
:10A49800877A38EE280AE8EC017A67EE897A9FED28
:10A4A8002B9A27EE899A30EE490A0AF001FA0AF146
:10A4B8006801BDEEC88AC85318EE103A0AF1700157
:10A4C800FDEEE88AB1EE499A41F82430BDEEC99A0A
:10A4D8000AF17C0118EE903A41F8243019EE103A4E
:10A4E8000AF18801574641F82430009B0133009354
:10A4F80074BB012497E600BF83F9223ED80F0020E1
:10A50800BD37863598110020B41000200000E143C3
:10A51800000000005C14002004100020CDCC4C404A
:10A52800F62B0020E01F0020506901086F12033C41
:10A538000AD7A33D0000A043000040C300004043E9
:10A548000AD7233C90130020A69B443BF7CC9238B3
:10A55800029A584B9479B3F90430640028345C4368
:10A56800554BB3F9043000EE103ABAEECF0A0AF0B0
:10A578009FF96411201A002C07EE900AB8BF6442B4
:10A58800322CF8EEE76A03DD0023CAF8283029E008
:10A59800BDEECAAA1AEE103A23F0030307EE903A6A
:10A5A800B8EEE7AADFED457A9BF80D30CAEE277AB8
:10A5B80007EE103AB8EE477ADAF8283026EE877AAE
:10A5C80067EE277AFDEEE77A17EE902A13443C4AA5
:10A5D8009342A8BF13463B4A9342ACBFCAF82830FF
:10A5E800CAF82820BB6A5B13B3F5807FA8BF4FF475
:10A5F80080736FF0FF029342B8BF134607EE903A9C
:10A60800F8EEE78AFDEEE67A9BF8032017EE903A1B
:10A6180053439B1107EE903A2B4B1B78032BB8EE54
:10A62800E78A14D9BBF84E20B2F5FA7F0FD2FDEEB7
:10A63800C87A534217EE901A994204DB914217EEFA
:10A64800903AA8BF134607EE903AB8EEE78A9BF80F
:10A65800511079B14B0803D09942A8BF194600E0C0
:10A668000121B0EE480A1948D7ED070AFCF7D2F9DC
:10A67800B0EE408A38EE280ABDEEC00A8DED000A19
:10A68800BDF9003000EE103AB8EEC00A0AF010F931
:10A69800BDEEC88AFDEEE88A0023A7F86C0087EDB6
:10A6A8001E8AC7ED218AC7F8903005B0BDEC0A8B29
:10A6B800BDE8F08FB41000200410002000803B4556
:10A6C800FEFFFF0F020000F060150020A413002019
:10A6D8002DE9F74FA44C00F0C7FB26686568A7680A
:10A6E800861BF643451BC71BED43FF43F60F804609
:10A6F800ED0FFF0F2EB93FB9002D00F07E82B9464D
:10A708002CE04FF0000929E0B14627E003EB8A0B63
:10A71800BBF8023019050ED413F4805F1DBF934AAD
:10A728009BF801101268924A924B14BF52F82120EC
:10A73800126843F82A20BBF80230DA0516D49B05C4
:10A748000AD58D4B1B7813F0040F0CBF8B4A8C4A2B
:10A75800884B126843F82A2009F10109207B8949AE
:10A768005FFA89FA82450B68D0D320E050465946F3
:10A77800854A03F043FD854B1B88580603D5504690
:10A788005946834A10E0590703D550465946814A2D
:10A798000AE09A0703D5504659467F4A04E0DB078A
:10A7A800DAD57E4A5046594603F028FDD4E7DFF84B
:10A7B80004E20093BEF906307822A3F57A73534376
:10A7C8004FF47A7293FBF2F303F22B1301930022F6
:10A7D800F3465FFA82FE864517D2009B03EB820E92
:10A7E800BEF802E01EF4806F0DD0DFF88891019B5F
:10A7F80039F822E040F2671A9E449EFBFAFC0AFBF5
:10A808001CEE29F822E00132E3E74DB308F5C33323
:10A81800A0336360637B544A13BB9373604B1B681C
:10A8280013F0020F0AD0DFF890E19EF800E0BEF1C5
:10A83800000F03D04FF0010E82F80EE0DA0506D5BE
:10A84800584B5B791BB1A37B43F00203A3734A4BBC
:10A858001B7813F0050F02BFA37B43F00403A37317
:10A8680094F80EE0BEF1000F03D13F4B5B7B002B49
:10A878004FD094F80DC01CF0010FACF10C031DD1A2
:10A88800BCF1030F07D8DFF8E8903C4A1EF0040F2C
:10A8980008BF4A4600E0364AACF1040CBCF1070F89
:10A8A80005D8DFF818C11EF0010F18BF6246DBB2E9
:10A8B800032B0ED81EF0020F3B4B06E0DBB2032B36
:10A8C80006D82F4B2A4A1EF0020F18BF1A4600E07E
:10A8D800274A4FF0000C5FFA8CF383420DD20B68C5
:10A8E80003EB8C035B881B0642BF224BD2F8009017
:10A8F80043F82C900CF1010CEDE785B1BEF1000F87
:10A9080008D0637B184A0133DBB2142B06D100232D
:10A9180004E025B1637B002BF3D100E05373002ED4
:10A9280050D0224AB2F90250B2F90020002DB8BF27
:10A938006D42002A4FF03203B8BF524295FBF3F53F
:10A9480092FBF3F2EDB2D3B2AB4238BF2B46184AB2
:10A9580013B192FBF3F300E0134643442360E37B17
:10A96800014A6BBB01232CE080140020181D002035
:10A97800A07E01087A0D0020FD2B0020A87D01088B
:10A98800987D010880130020526901089811002061
:10A99800586901085E690108646901086A69010863
:10A9A800E81F0020040E0020B07D0108B41000202C
:10A9B800400D03002420002020110020B87D01084C
:10A9C8000023D3738E4D8F4B2D78E27BADB9002FCA
:10A9D80000F00E818C4B267B1A788C4B8C4D93F8AB
:10A9E80000C08C4BD3F800E00B6802F00402002191
:10A9F800D2B203EB86060F46B5E01AB9864A1A6149
:10AA0800002508E0854AFAE70A68AB00D618768878
:10AA1800760604D40135EBB28342F5D3D7E7804EEE
:10AA2800B6F90060192E25DD12F803E094F814C079
:10AA380026690EF00F09E1450CDCDFF8C8C19CF867
:10AA480015C0BCEB1E1FDEBFDFF8D8E1D6F800C08A
:10AA580043F80EC012F803E094F816C00EF00F0980
:10AA6800E14533DBDFF89CC19CF815C0BCEB1E1F29
:10AA78002CDC26E0193629DA12F803E094F814C021
:10AA880026690EF00F09E1450CDCDFF878C19CF867
:10AA980017C0BCEB1E1FA2BFDFF888E1D6F800C0C4
:10AAA80043F80EC012F803E094F816C00EF00F0930
:10AAB800E1450BDBDFF84CC19CF817C0BCEB1E1F4F
:10AAC80004DBD6F800E0574E43F806E0544EB6F9DA
:10AAD8000260192E1BDD12F803C094F814E02669F1
:10AAE8000CF00F09F1450CDCDFF8189199F8159076
:10AAF800B9EB1C1FDEBFDFF82CC1D6F8009043F875
:10AB08000C90D25C02F00F0CF4451EDD82E719367A
:10AB180080DA12F803C094F816E026690CF00F09E1
:10AB2800F1450CDBDFF8DC9099F81590B9EB1C1FA8
:10AB3800DEBFDFF8F0C0D6F8009043F80C90D25C86
:10AB480002F00F0CF445FFF665AF94F817E0BEEB82
:10AB5800121FA2BF334A36689E505BE7588800052B
:10AB680004D404330435B342F8D122E04AB101EBEE
:10AB78000C0A06209AFBF0F900FB19A001280DDC4D
:10AB880001E057B9012793F801900EEB89003EF8D0
:10AB980029A090F80290C07803E01746002081466B
:10ABA8008246013125F802AC85F800906870C9B278
:10ABB800D7E7164A1378013B13F0FF0308BF0623B3
:10ABC8001370114B1B785B0741BFBBF90630A3F527
:10ABD8007A7303EBC3034FF47A7243BF93FBF2F328
:10ABE8000133DBB20123104A92FBF3F34344A36021
:10ABF80003B0BDE8F04F02F0A9BD03B0BDE8F08F87
:10AC0800330E002080140020FD2B00208C00002033
:10AC18007C0D0020181D0020B47D0108A07E0108CD
:10AC2800B41000207A0D0020400D0300034B4FF4B0
:10AC3800085208B19A6170471A8570470010004899
:10AC4800034B4FF4085208B11A8570479A61704750
:10AC5800001000480C4B1B6893F90220824209D06F
:10AC680093F90A20824207D093F91220824208D130
:10AC7800022002E0002000E0012003EBC0000230C7
:10AC880070470020704700BF5012002038B1438839
:10AC980011EA030003D08B420CBF01200220704749
:10ACA80030B50A4B0A491C680A78022A0AD81346A2
:10ACB80004EBC303551CEAB29D882842F5D00A70FC
:10ACC800981C30BD0A70002030BD00BF5012002013
:10ACD80098140020014B00221A70E1E79814002014
:10ACE8002DE9F047877890F803C0214DBBB2C7F132
:10ACF800640E03EB83065C42C3F178005FFA8EFEB4
:10AD08007600CCF16408A4B280B2A3B20FFA83F93A
:10AD1800B9F1000F05DC002B14BFBA464FF0010A49
:10AD280000E0F24613FB03F303FB0CF21AFB0AF3F1
:10AD380092FBF3F3434403FB09F30A2293FBF2F378
:10AD480033449BB225F8023FB1F800904A880A3490
:10AD5800C9EB020AA4B21AB202FB0AF24FF47A73E0
:10AD6800844292FBF3F34B442B80CED1BDE8F087AD
:10AD78009814002010B544780078002202FB02F3F2
:10AD8800193B634303F6C413534340F6C4114343CA
:10AD980093FBF1F3034921F812300132072AEDD170
:10ADA80010BD00BFB21400200430114B33F910005D
:10ADB800B0F5617F10B506DB40F6330398420246D2
:10ADC800A8BF1A4601E04FF461720C78192340F2CB
:10ADD800833013FB0404944207DA497813FB010318
:10ADE8009342B4BF0020012010BD002010BD00BF59
:10ADF8002420002010B500F1500302788A4203D1C4
:10AE08008478C278944204D304309842F5D1002063
:10AE180010BD012010BD1FB5084B1B681B030AD5C8
:10AE28008DF8040001230D2001A98DED030A8DF88A
:10AE38000530FCF761FD05B05DF804FBE81F002054
:10AE48001FB5084B1B681B0309D58DF80400029138
:10AE580000230D2001A98DF80530FCF74DFD05B044
:10AE68005DF804FBE81F002010B50A4A0A4B116878
:10AE78009B6800BF12689142F7D1084A946A4FF460
:10AE88007A7000FB04F2D31AB3FBF4F300FB013031
:10AE980010BD00BF0C20002010E000E09814002036
:10AEA80038B50446FFF7E0FF0546FFF7DDFF401B16
:10AEB800A042FAD338BD10B504462CB14FF47A70CD
:10AEC800FFF7EEFF013CF8E710BD2DE9F04F06460D
:10AED8008A4890F9004087B0B44288469DF84450AB
:10AEE80011461A469DF8403009D090F90C40B442FA
:10AEF80007D090F91840B44209D1022702E0002790
:10AF080000E001270C2404FB0700047A0CB10020A0
:10AF1800F0E0012E00F0DD80142E05D0002E40F068
:10AF2800E88000957648D6E0DFF814A2DAF8183001
:10AF380043F00103CAF81830DAF814304FF090459E
:10AF480043F40033CAF814304FF0010903224FF4D8
:10AF5800805B04A94FF090408DF815200392CDF83E
:10AF680010B08DF814908DF816908DF81740FBF7F7
:10AF7800DBFBA5F828B0C820FFF79DFFC5F818B07F
:10AF8800DAF81430039A43F40033CAF81430284628
:10AF98004FF4C0534FF0020B04A904938DF8152009
:10AFA8008DF814B08DF816408DF81740FBF7BCFBF0
:10AFB8006B6A23F470436B626B6A43F460436B62A1
:10AFC8006B6A23F470236B626B6A43F460236B62D1
:10AFD8004C4B4D4D4FF480221A6002F18042A2F58D
:10AFE8003F321223EB65082385F86130136885F832
:10AFF800629023F480231360536823F48023536002
:10B0080095F8603003F1804303F582331A6842F4FF
:10B0180080221A60EA6D3D4B22F01F0002F01F02E9
:10B02800C15809FA02F221EA0202C250EA6D38490F
:10B0380022F01F0002F01F0250F801E009FA02F2A4
:10B048002EEA02024250EA6D22F01F0102F01F02AE
:10B05800C85809FA02F20243CA502E4B2E4A1C6005
:10B06800DAF81C3043F40003CAF81C302B4B04A850
:10B07800DA608DF810608DF811B08DF812408DF8F7
:10B08800139004F0ADFC2A238DF810309DF813308E
:10B098008DF811908DF812401BB104A804F0A0FCA3
:10B0A80004E01F4B4FF48062C3F884201D4B1E4CF4
:10B0B8001C60022385F86C301C4A1D4B1D49C5F8DD
:10B0C800803011601B6898471B4BEB62A4F1380075
:10B0D80006E01A48009501F091FA00283FF417AFEE
:10B0E800064B06710C2202FB073787F80880786048
:10B0F80000E0204607B0BDE8F08F00BF54120020E2
:10B10800003801401404014098140020080401404C
:10B118000C040140D80042420005FA0500ED00E0A9
:10B1280000E100E0A4110020FC140020A811002078
:10B138001C000020900000207069010800440040B5
:10B1480000100240024A136801331360704700BFC1
:10B158000C200020024BD3F8843003B11847704705
:10B1680098140020014B1B68184700BFE02B0020F3
:10B1780010B50020FFF7F6FF074B00241C7005F000
:10B18800D3FF064B83F88840C3F88C40A3F890405F
:10B19800C3F8944010BD00BFC82B002098140020AD
:10B1A80010B510B9BDE81040E2E700230C225A435D
:10B1B8000C4C1119125D824203D00133102BF5D1CA
:10B1C80010BD094BD3F8940018B14A7840788242F0
:10B1D80006D20022C3F89410A3F89020C3F88C205C
:10B1E80010BD00BF506E01089814002010B5400033
:10B1F8001428A8BF14200023074A022199540B449D
:10B2080099181424834201F8014CF5DBFF21D1542D
:10B218000F20BDE81040C3E7C01F002038B5174B0A
:10B228004FF4884240F2DB159A6168434FF4885224
:10B238001A85851E0B24013C14F0FF0417D00F4A11
:10B24800938A9BB283F488439382938A9BB283F454
:10B25800885393822846FFF72EFE0120FFF782FFCE
:10B268001920FFF728FE0020FFF77CFFE3E7044BD7
:10B27800044A1A60044B054ADA6038BD00100048D9
:10B28800FC9F0020EFBEADDE00ED00E00400FA05F3
:10B2980003681B6918470368DB68184703689B68DD
:10B2A800184703685B68184703681B6818472DE947
:10B2B800F84FB0F90230934218BF00232DED028BEE
:10B2C80018BF0370057804460E469146002D40F0DD
:10B2D8008B8007EE902A9FED770AF8EEE77AB6EEB4
:10B2E800008A27EE800ADFED747A20EE270AA0464E
:10B2F80020EE080A09F052FBDFED706A60EE266A5C
:10B30800B7EE006AB0EE667AA0EE007A40F2DC533F
:10B318006365D0EE006A1023A4F8523037EE067A3F
:10B3280076EE866AC6EE077A1823A4F850302746C8
:10B3380084ED046A27EE807A27EE007A77EE075AC2
:10B3480084ED017AC4ED025A70EE005A84ED037A56
:10B35800B8EE007AA5EE807A27EE877A67EEA67AAD
:10B3680084ED057AC4ED067ADFED557A98ED047A16
:10B3780027EE277AF0EE678AB5EEC07AF1EE10FA7A
:10B388004CBF77EE487A77EE087A013517EE900AC7
:10B3980006F0A6F8D8ED017A67EEA87AC7E90E019B
:10B3A800F5EEC07AF1EE10FA4CBF77EEC87A77EE78
:10B3B800887A08F1040817EE900A06F091F8032D30
:10B3C800C7E9080107F10807CED1A6F2DC531B0430
:10B3D8002367E3676367C4F88030A367C4F88430E1
:10B3E8000123A4F802902370D4F85490B4F9528041
:10B3F800636A276A206FE26FD4F840C0D4F88010DF
:10B40800C4F88020C9EB060606FA08F64FEAE67B80
:10B41800734307FB0B332667A7FB06671F44636C60
:10B42800656F60674FEAE27B53430CFB0B3EACFB56
:10B4380002237344B61A67EB0307E36AA26AC4F8E7
:10B4480084104FEAE07B434302FB0B3EA2FB002340
:10B458007344B6185F41E36CA06CB4F95020A5673B
:10B468004FEAE17B4B4300FB0B33A0FB010119447E
:10B47800636B361A206B4FEAE57B05FB03F300FB91
:10B488000B3367EB0107A0FB0501194480197941CB
:10B4980005F0FCFF08F1FF3201239340E067C01874
:10B4A80041EBE371424605F0F1FFBDEC028B4844E5
:10B4B800BDE8F88F6F12833ADB0F4940F404B53FBB
:10B4C8000000804B2DE9F8430024244B93F8C86012
:10B4D800E0B2B0420DD203EB8003214AD3F8983092
:10B4E80032F810101BB10B2801D8DB6898470134DB
:10B4F800EBE71C4B1B685B032DD500242346E2B207
:10B50800B24228D2DFF8549009F198074FEA84082C
:10B5180057F8242055689D4215D0284602F0BEFDF4
:10B52800EFF31283502282F3128828216A6A01FB02
:10B5380000900132C0F8F0206A6942F001026A61A5
:10B54800DBB283F3118857F808301B6800221A60B1
:10B5580001342B46D3E7BDE8F88300BF98140020D8
:10B5680024100020E81F002008B50E4B1B6813F4B8
:10B57800805F0D4B14BFD3F8E421D3F8E82193F88A
:10B58800C81092880023D8B2884204D2074820F80D
:10B5980013200133F7E7FFF795FF3220BDE8084095
:10B5A80089E400BFE81F0020981400202410002020
:10B5B8000A4B1A680A4B30B502F48052D3F8E441BA
:10B5C800D3F8E85100230AB1A18800E0A98805480A
:10B5D80020F8131001330C2BF5D130BDE81F0020E3
:10B5E80098140020961F002070B5124D00242146A3
:10B5F80005F2ED10702285F8EC4108F04AFF21466B
:10B60800D5F860320B4A0B4493F9020080B102F27C
:10B61800ED141E680E5108199C8884809B798371EB
:10B6280092F8EC3107310133702982F8EC31E7D117
:10B6380070BD00BF98140020094B1A680E2303FB45
:10B648000020437AFF2B07D0064A12789A4203D982
:10B65800054A32F8130000E0808800B2704700BF46
:10B668001C1D0020481200202420002038B5294C39
:10B678002DED048B94ED998AB0EE480A0546FBF748
:10B6880079FCF0EE408AB0EE480AFBF710FC94ED26
:10B698009A9AB0EE408AB0EE490AFBF76BFCF0EEDE
:10B6A800409AB0EE490AFBF702FC95ED017AD5ED18
:10B6B800027A95ED006A68EE676A27EE088AE7EE77
:10B6C800286A68EE000A67EE807AE6EE290AB0EE8C
:10B6D800660AE7EEA80A09F0EDF9DFED0F7A20EE29
:10B6E800270ADFED0E7A80EE270AD4ED9B7A30EE3A
:10B6F800270AF2EE047A80EE270A09F0D9F8BDECA1
:10B70800048B83B21A0444BF00F5B47083B218B234
:10B7180038BD00BF981400200000E144DB0F494009
:10B7280001380A4B042804D8DFE800F00507090BA4
:10B738000D00074A08E0074A06E0074A04E0074AFE
:10B7480002E0074A00E0074A1A6070471401002027
:10B7580029FF0008D197000855020108259E000816
:10B76800919A00085DA1000882B01B4B1B4A8DF816
:10B7780007101968106860B31268052A29D1184A99
:10B78800106810BB9DF808109DF8073043EA0123A4
:10B7980014490B80144B1968144B89B20B445B0095
:10B7A80019680121196013680B441360104A136863
:10B7B80023F4E04323F040039BB283F0300343F4C7
:10B7C800004343F08003136003E01A68521A312AD9
:10B7D800D5D902B0704700BF0C200020E42B002010
:10B7E8000817002080610040505C00400A300020AB
:10B7F800045C0040014B5868C0B27047081700202D
:10B80800012070477047704720B9034B1B68082216
:10B818001A82704701487047A4110020B400002024
:10B8280020B9034B1B6808221A82704701487047E9
:10B83800A4110020B400002021B901288CBF0220E7
:10B84800002070470220704710B5094B1A68D3785A
:10B85800042B0BD8074C518ADB00234418B99B8969
:10B868005B1A138210BD9B68581810BD002010BDCC
:10B87800A4110020B4000020054B1968054B4A8A22
:10B8880018B99B8D9B1A0B827047986A10447047B1
:10B89800A4110020B4000020054B1968054B4A8A02
:10B8A80018B99B8E9B1A0B827047186B104470470F
:10B8B800A4110020B4000020074B1B681B7803F07C
:10B8C8007F03212B06D100F0DF00022814BF0220DD
:10B8D8000020704702207047A4110020212810B5CD
:10B8E80008D1114B1B681B7803F07F03212B10D064
:10B8F800022010BD2028FBD10B4B0C4A1B681B787B
:10B90800107003F07F03212B094B18BF00230BB9DC
:10B91800EEE7084B044A12680024936154822046DB
:10B928009847204610BD00BFA4110020002C00201D
:10B9380011B8000829B80008704707EE900AF8EE19
:10B94800E77ADFED0C6A9FED0C0AF5EEC07AF1EEAE
:10B9580010FAD4BFB1EE677AC7EEA67A08B5D8BF99
:10B96800C7EE267A27EE800AFBF704FB034B83ED2C
:10B97800000A08BD8096184B35FA8E3C0801002055
:10B98800F7B51C4B5A681D460AB95C6800E00124EB
:10B99800187A0021CAB2A24201F1010107D202AE0F
:10B9A8002F1816443A44527A06F8042CF2E75A68DB
:10B9B800121B5A601A7A5D6822441A729DB90320D4
:10B9C8004021FAF78DFB0C4A136823F4804323F0D7
:10B9D80070039BB283F4405343F4004343F0800365
:10B9E8001360044B1D72002CCBD09DF8040003B0EB
:10B9F800F0BD00BF081700200C5C0040F8B5A84B4C
:10BA08001B680546187818B1012800F0838106E301
:10BA1800242DA44C0CD006D80A2D00F0EC800D2D56
:10BA280000F0E9805CE12A2D09D02C2D07D057E1E0
:10BA380084F8490084F84A0084F84B0066E19A4B80
:10BA480094F84A1094F84970964A0020585447BB15
:10BA5800197882F84C70472923D15978502920D178
:10BA68009978472908D1D978472905D119794129E1
:10BA780002D1012182F84C1099788B4A522903D1BE
:10BA8800D1784D2900F0CD829978874A472908D185
:10BA9800D178532905D11279562A04BF032284F894
:10BAA8004C2094F84C207F4E022A3BD0032A50D0D9
:10BAB800012A40F08A80BA1E072A00F28680DFE851
:10BAC80002F004080F131A25842B04F061F920658D
:10BAD8007BE01B78532B78D1236D5B42236574E0A0
:10BAE80004F056F9606570E01B78572B6DD1636DD3
:10BAF8005B42636569E01B78302B6C4B1A788CBF0E
:10BB080042F0020222F002021A705EE0002004F005
:10BB18009FF984F8580058E0002004F099F9A4F837
:10BB28005A0052E0072F07D0082F4ED1012004F009
:10BB38008FF9A6F85E0048E0012004F089F941F287
:10BB4800184358434FF47A73B0FBF3F0A6F85C003F
:10BB58003BE0022F07D0032F0BD1002004F078F927
:10BB6800534B187031E0002004F072F986F8600039
:10BB78002BE02AD93A1F921096F860300132D2B2DF
:10BB8800013B02EB8303DBB2102B1ED8F91EC2F176
:10BB9800010201EB8202D2B2012A0BD0042A11D190
:10BBA80000205E1E04F054F9424B9855424B002287
:10BBB8009A5507E05E1E414A0020935504F048F963
:10BBC8003F4B9855636E01336366364B2A2D18BF79
:10BBD80093F84B2007F101074FF000000CBF01223A
:10BBE800554084F8497084F84A000CBF83F86820EF
:10BBF80083F84B508AE094F8680000284CD0314B09
:10BC080013F8012D30495A708B42F9D1264A254D37
:10BC180013785278402B85BF373B1B011B01DBB2E1
:10BC280098BF03F0F003402A8CBF373A303AD2B2BB
:10BC3800134494F84B20DBB29A422AD121230B708B
:10BC480095F84C00EB6E204A01330128EB660CD0C6
:10BC5800022820D1722313701C4BB5F85C201A807F
:10BC68001B4BB5F85E201A8015E0672313700F4B45
:10BC78001B789F0710D5174B2A6D1A606A6D5A609A
:10BC8800154B95F858201A70144BB5F85A201A809D
:10BC980002E03F230B700020002384F8683035E071
:10BCA800CC0600200817002014200020D410002003
:10BCB8005C1000208D1000207D1000205D100020F9
:10BCC8006D100020300300201C030020D610002037
:10BCD80044100020DC100020DA100020D8100020CA
:10BCE80094F84A3094F868000E2B9FBFB14A591C4B
:10BCF80082F84A10B04A98BFD554AE4A28B992F88B
:10BD08004B305D4082F84B5000E00020003018BFF7
:10BD18000120F8BDA74B93F870100022082900F203
:10BD28007E81DFE801F0050C101A2B3C63828F003E
:10BD3800B52D40F0748183F87120012253E0622D03
:10BD480008BF02224FE0032283F8702083F8725064
:10BD580083F8735083F8745061E1042283F87020EB
:10BD680093F8732093F8741083F875502A44D2B26C
:10BD780083F873200A4483F8742050E1052283F87D
:10BD8800702093F8732093F87410A3F876502A441F
:10BD9800D2B283F873200A4483F874203FE1062264
:10BDA80083F8702093F8732093F874102A44D2B261
:10BDB80083F873200A4483F87420B3F8762002EBE2
:10BDC8000525ADB2B5F5AC7F88BF7A4AA3F87650A1
:10BDD80084BF012182F871100022A3F87820002D79
:10BDE80040F01D81072283F8702018E193F8732032
:10BDF80093F874102A44D2B283F873200A4483F863
:10BE08007420B3F87820B2F5AC7F3CBF6949891833
:10BE180002F1010238BF81F87C50B3F8761092B273
:10BE28009142A3F87820DDD9F9E0082283F8702040
:10BE380093F87330AB4200F0F2805E4B012283F836
:10BE480071200FE05D4C83F8702014F8012D6270AA
:10BE58005B4A9442F9D193F87410564AA94206D025
:10BE68003F232370574A536801335360D7E0D16E9C
:10BE780092F871000131D16610B13E232370CEE0F3
:10BE88002121217092F87510062944D004D802297E
:10BE980007D0032926D0F8BD12295CD030296CD0F0
:10BEA800F8BD502121704849D2F880404C60D2F842
:10BEB80084400C60D2F88C104FF47A7491FBF4F142
:10BEC800424C218092F8D411414A19B1117841F0BD
:10BED800020102E0117821F002011170012283F8B9
:10BEE800D5218EE05321217092F88110CE0705D517
:10BEF80092F88020D51E6A426A4100E0024602F0AC
:10BF0800010183F8D411002A7BD131490A7822F043
:10BF180002020A7075E04F21217092F88710CC0751
:10BF280005D592F88620D11E4A424A4100E00246D1
:10BF380002F0010183F8D41122B925490A7822F0C8
:10BF480002020A70234A93F8AB101170224AB3F820
:10BF5800A810118055E0562121702049D2F8904050
:10BF68000C8042F21074D2F8941091FBF4F11C4C3E
:10BF78002180012182F8D61143E04921217092F8ED
:10BF88008010184A102988BF10211170164914789A
:10BF98000022A24232D2154D0E7A5655144D4E7AD1
:10BFA8005655144DCE7A5655134D11F80C6F5655FB
:10BFB8000132EEE70817002014200020300300208B
:10BFC8001C030020AC060020DC100020D810002044
:10BFD800D4100020DA10002012010020D610002012
:10BFE800441000205C100020841700205D10002001
:10BFF8006D1000207D1000208D1000205A6E013237
:10C008005A6693F8D5310B4A9BB192F8D63183B171
:10C01800002182F8D51182F8D6111846F8BD002003
:10C02800F8BD1279432A7FF42FAD022284F84C2000
:10C038002AE5F8BD081700200449054B096818705F
:10C0480000225A6199611A77704700BF0C200020BE
:10C05800AC06002010B5121A07EE902A5B1A2DEDD7
:10C06800028BF8EEE78A07EE903A184B059CB8EE7B
:10C07800E78AD3ED007A28EE278A28EE080AA8EE88
:10C08800A80A08F019FDDFED127A049B20EE270AB2
:10C09800F0EE480ABCEEC00A83ED000AB1EE680A69
:10C0A80008F008FDDFED0B7A9FED0B7AE0EE077ADA
:10C0B800BDEC028BFDEEE77A17EE903A002BBCBF81
:10C0C80003F50C43A033236010BD00BF0801002016
:10C0D8002C7D8E3F00A00C46A00CB34544F2506363
:10C0E800984203DDA0F50C40A0387047034B9842F6
:10C0F800BCBF00F50C40A030704700BFB0B9FFFFCF
:10C1080073B51A4C036823600B686360184D0068A8
:10C11800184EFFF712FC184B009395E8030094E8BB
:10C128000C000196FFF796FF144B32681A60686896
:10C13800636813491B1A07EE903A124B286893ED6F
:10C14800007A23681B1A0B600F4BF8EEE77A1A6027
:10C158000E4B67EE877A1B68FDEEE77ADA880C4BA0
:10C16800C1ED017A1A8002B070BD00BF341F0020F3
:10C17800DC100020401F00203C1F00207C1F0020F6
:10C18800441F002008010020741F0020100F002009
:10C19800701F00204279DFED2A5A2A4B9FED2A5A58
:10C1A80007EE902AF8EE677AC27BC7EEA57AB2EE60
:10C1B800047AC3ED007A07EE902AF8EE677A234AEC
:10C1C800DA60C7EEA57AC3ED017A8179204B07EED4
:10C1D800901AF8EE677A017CDA60C7EE877AC3EDC9
:10C1E800007A07EE901A817E06EE101AF8EE677A4A
:10C1F800B8EE466AC7EEA57A86EE056AC3ED017AFF
:10C2080083ED026AC179134B06EE901A417CDA601D
:10C21800F8EE666AC6EE876A07EE101AC17EC3EDAD
:10C22800006A07EE901AB8EE477AF8EE677A87EE5A
:10C23800257AC7EE857A83ED017AC3ED027A7047D5
:10C248000000C8424C1F002000007A440000FA4455
:10C258005C1F0020801F002010B50C4C23789B0722
:10C2680013D50B4B1B78042B0FD90A4A0A4B1068BD
:10C2780052685A601860FFF760FB084B1A88084B31
:10C288001A80237843F00103237010BDD4100020D6
:10C29800DA100020DC10002048100020B010002028
:10C2A800901F00201C4B1B681B0307B530D51B4A89
:10C2B8001B4BD2ED007A1B788DF80030B2EE047A71
:10C2C80067EE877A174B9FED187A1B788DF8013047
:10C2D800FCEEE77A0A2017EE903AD2ED017A8DF853
:10C2E800023067EE877A6946FCEEE77A17EE903AF5
:10C2F800D2ED027A8DF80330FCEEE77A17EE903A29
:10C308008DF80430094B1B788DF80530FBF7F4FAEB
:10C3180003B05DF804FB00BFE81F0020FC1F0020ED
:10C32800DA1F0020F81F002000007A44DE1F0020DA
:10C33800054A137883F001031370044A002313603D
:10C34800034A1360AEE700BFDE1F0020F41F002081
:10C35800F01F00200A4B10B519684FF6FB720A400F
:10C368001A60084A927A1C46074B0AB1052200E077
:10C3780001221A6003F0D6F94FF43643236010BD4A
:10C38800405C0040FC140020E42B002010F80A3C1C
:10C398000133DBB20A2B84BF10F8131C044A00F8DF
:10C3A8000A3C82BF002322F8113000F80A3C70478B
:10C3B800142B0020334A136C90681944081A40F66D
:10C3C8008C23984270B513469160D06051603BD978
:10C3D800127893F945108A4210460BD1111F08298B
:10C3E80008D893F84610182901D8013103E083F8DA
:10C3F800442002E0002183F8461093F94440214983
:10C40800A24219D191F84740B4B10C3100249442AA
:10C4180006DA1D4D51F8046F25F814600134F6E76B
:10C428000C2805D01849002421F810400130F7E7FE
:10C43800164801780131017083F845200022012156
:10C448001A7083F8471070BD92F84710C9B1A0F26E
:10C45800EF2440F2DA518C4208D811780B2905D81C
:10C468000B1D0131117042F8230070BD002283F8C2
:10C478004720074B03F13002002143F8041F934281
:10C48800FAD170BDC0010020142B002084060020C2
:10C49800CC010020024A136C01331944116470471F
:10C4A800C0010020024B53F820301B681960704708
:10C4B80030150020064B53F820301A681B89A1F567
:10C4C8007A7159434FF47A7391FBF3F11160704715
:10C4D80030150020F0B5046D8668236823F0010349
:10C4E80023608379054613F0020F40790CBF4FF0A3
:10C4F800000E4FF4005E13F0040F14BF4FF4806772
:10C50800002710F0010F14BF0421002183072068C1
:10C5180020F001002060626822F440524EEA0202D4
:10C528006260226822F4B05323F00C0348BF41F044
:10C5380008013B430B432360A36895B023F4407381
:10C54800A3606846F9F77AFF284B9C4201D10C9BFF
:10C558000EE0274B9C4201D10D9B09E0254B9C42E4
:10C5680001D10E9B04E0244B9C420CBF0F9B109BF7
:10C578002268A879170448BF5B00B3FBF6F206FBF4
:10C588001233B3EB560F236828BF01321E0441BF94
:10C598004FF6F073C2F34201134041EA03026B798C
:10C5A80092B213F0020FA28100F0010114BF4FF400
:10C5B80000320022DC0748BF42F480322B6D11B1F3
:10C5C80059680A4302E0596821EA02025A609A68E7
:10C5D80001074CBF42F0080222F008029A601A686C
:10C5E80042F001021A6015B0F0BD00BF00380140EA
:10C5F8000044004000480040004C00402DE9F0474E
:10C608001E46A14B8CB09842894690469DF85070C2
:10C6180040F085809D4B9E4A1A609E4A5A6102F5F9
:10C6280080729A614FF48072DA601A619A4A1A63CA
:10C63800143A5A63A2F54842203ADA6404329A64FA
:10C64800C3F808801865954B9A6942F480429A614C
:10C658005A6942F001025A6102238DF80830032317
:10C6680017F0010A8DF809304FF000038DF80A30F1
:10C6780014BF022301233A078DF80B3019D54FF068
:10C6880090444FF4007501958AF001038DF80A3043
:10C69800636A23F0F0036362636A43F070036362C2
:10C6A800204601A9FAF740F8BAF1000F27D1A56191
:10C6B80025E0B30710D50CA94FF4007341F82C3DC1
:10C6C8004FF09040436A23F0F0034362436A43F01B
:10C6D80070034362FAF728F8F50710D50CA94FF450
:10C6E800806341F82C3D4FF09040436A23F4706317
:10C6F8004362436A43F4E0634362FAF715F80E2392
:10C708008DF800300022012368468DF801308DF83D
:10C7180002208DF803305D4C03F062F973E0604B42
:10C72800984240F005815F4B594A1A604FF4807275
:10C73800DA601A615C4A5A6102F580729A61574A56
:10C74800C3F808801865D36943F40033D361022322
:10C758008DF80830032317F0010A8DF809304FF0DF
:10C7680000038DF80A3014BF022301233C078DF81B
:10C778000B3017D54D4C202501958AF001038DF813
:10C788000A30236A23F470032362236A43F4E00324
:10C798002362204601A9F9F7C7FFBAF1000F23D198
:10C7A800A56121E0B0070ED50CA9202341F82C3D46
:10C7B8003E48036A23F470030362036A43F4E00308
:10C7C8000362F9F7B1FFF1070ED50CA9402341F830
:10C7D8002C3D3648036A23F070630362036A43F012
:10C7E800E0630362F9F7A0FF26238DF800300022EA
:10C7F800012368468DF801308DF802208DF803304A
:10C8080003F0EEF8274CC4F82C900025012384F897
:10C8180044302562E561A56265626671C4F80880E6
:10C82800A7712046FFF756FEF20748D5236B002B69
:10C838003ED001A8F9F720FDE36C01934FF4805333
:10C848000A9380230693E368ADF8103020230993F8
:10C85800206B636902930B950595079508950395D9
:10C86800F9F735FD01A9206BF9F713FD236B216D4D
:10C878001A6842F001021A608A6842F040028A602F
:10C888005B689BB223641AE000380140741E0020E4
:10C89800286A0108E01800205800024000100240F1
:10C8A80000440040201E0020E01A0020000C004830
:10C8B800236D20221A621A6842F020021A60B30718
:10C8C8002FD5636B43B301A8F9F7D6FCA36C01938A
:10C8D8004FF480530A93802306932369ADF81030F0
:10C8E80000251023606B03930B9505950795089514
:10C8F8000995F9F7ECFC606B01A9F9F7CAFC636BC1
:10C908001A6842F002021A60226D5D605D609368E9
:10C9180043F08003936004E0226D136843F08003C2
:10C928001360226D136843F001031360204600E092
:10C9380000200CB0BDE8F0873D4B1B78012B30B5CB
:10C9480014BF00240324B1B9036A23F0010303626E
:10C958008169036A21F0F30123F00A0341F0010120
:10C9680042F001021A4341EA0411816102628369BB
:10C9780023F00C031BE004291DD1016A4FF6EF7365
:10C988000B4003628169056A120121F473414FF675
:10C998005F7342F0100241F480712B4092B213434E
:10C9A80041EA043181610362836923F4406383614E
:10C9B8008369836130BD0829016A1AD14FF6FF6384
:10C9C8000B400362C169036A9BB289B223F42063F6
:10C9D80043F4807321F0F30143EA022241F001019C
:10C9E80092B241EA0411C1610262C2694FF6F3735F
:10C9F80019E04EF6FF730B400362C369056A40F6FF
:10CA0800FF41194045F6FF732B4043F4805343EA36
:10CA1800023241F4807192B241EA0431C16102628A
:10CA2800C2694FF2FF331340C361C369C36130BDAC
:10CA3800BC01002038B510F80E2C50F8043C044610
:10CA480052B9012200F80E2C20F80C1C997A1868AB
:10CA58000222BDE838406FE730F80C2C20F80A1C99
:10CA6800891A89B220F8081C074A10F80F0C00250B
:10CA780022F8101004F80E5C1868997A2A46FFF715
:10CA88005BFF04F8065C38BD142B0020044B53F8F8
:10CA980020301BB107289CBF1B681960704700BF76
:10CAA800E802002038B500240B4D6059254402F0F7
:10CAB800E3F9696811B10948FAF7CBF9A96811B126
:10CAC8000748FAF7C6F90748103402F0D5F9B4F563
:10CAD800E07FE9D138BD00BF406A0108CE85010872
:10CAE800D4850108538F010870B50546284607F01C
:10CAF80014FD064658B91A4B1A485A791A4B03EBD3
:10CB08008203BDE87040D3F8BC11FAF7A2B92846F1
:10CB18001649324607F00AFD60B91548154C02F06F
:10CB2800ABF954F8041F19B11348FAF792F9F8E76A
:10CB3800124805E00024124B53F8241021B911487B
:10CB4800BDE8704002F098B92846324607F0EEFC7E
:10CB580001340028EFD1024B0B4D5C71C6E700BFD2
:10CB680048200020DA850108406A0108E6850108A6
:10CB7800EB850108FC6B0108FE850108538F01084D
:10CB8800006C01080E850108EA810108F0B585B03E
:10CB9800044607F0C2FC082826D1621EE01D1F4982
:10CBA80012F8013F09681944497801F00301022984
:10CBB80008BF203B82421370F1D1254604F10807D3
:10CBC80015F8016B1648314607F099FC20B1284644
:10CBD800314607F094FC10B1FBF73CFB1CE0BD426A
:10CBE800EED12046F9F73CF90E4802F045F900234A
:10CBF8000D4A1A4404A992F88A210A440849595C42
:10CC080002F80C1C0133082BF2D1002307488DF8D9
:10CC18000C3001A9FAF71DF905B0F0BD200100207C
:10CC28001E8301080286010848200020F78D0108AC
:10CC3800234B244C1D68206880B5FCF709F828466A
:10CC4800FCF706F8206841798B0704D4036841F0A3
:10CC580002015B6998471C4B4FF488521A854FF4C0
:10CC680088421A852068FEF71CFBA0B1164E4FF4C7
:10CC78008853B361134B1868FEF710FB0746FEF79D
:10CC8800BDFE08B101F084FB28463946FEF70CFBCF
:10CC98004FF4885333852846FEF703FB0028E1D07C
:10CCA800094ED4F800804FF48847B7612846FEF74C
:10CCB800F5FA01464046FEF7F7FA3785D2E700BF96
:10CCC800B01F0020E01C0020001000482DE9F047AC
:10CCD800054607F022FC314E0446D6F8088090B984
:10CCE8002F4802F0C9F82F4B53F8241049B10123FB
:10CCF800A34013EA080F02D02B48FAF7AAF8013428
:10CD0800F1E72A4822E028462949224607F00EFC86
:10CD180058B92848284C02F0AFF854F8041F0029E5
:10CD2800EFD02148FAF795F8F7E72B782D2B03BFBA
:10CD3800013504F1FF344FF0010A4FF0000A4FF0BB
:10CD48000009184B53F8297027B91C48BDE8F0476B
:10CD580002F092B828463946224607F0E7FBC8B9E0
:10CD6800012000FA09F0830501D51548EEE7BAF16C
:10CD7800000F03D0FAF7C2F9124803E040EA0800AE
:10CD8800B060114802F078F839461048BDE8F0471D
:10CD9800FAF75FB809F10109D3E700BF482000207E
:10CDA80008860108686C0108FE850108538F010890
:10CDB800E685010812860108646C01080E850108E1
:10CDC8001E8601082C86010835860108F68D0108A3
:10CDD80010B5084802F050F8074B00241C715C633A
:10CDE800064B1C70FEF7E4FB02F0F8F9044B1C60DC
:10CDF80010BD00BF3D860108E01C0020012C00206A
:10CE0800B01F002070B5064600240B4BE518AA8811
:10CE180016420AD0E1580948FAF71BF828460021BB
:10CE280001F0B7FF064802F027F8143440F694439F
:10CE38009C42EAD170BD00BFF06F01086986010805
:10CE4800538F0108F0B504788BB005460CB1002467
:10CE580036E04A4B19680E2303FB041101F58C7068
:10CE6800B1F91D51B1F91921B1F91B31009591F8AA
:10CE78002051019591F82151029590F907000390EE
:10CE880001F590713E4891F9021004912146013450
:10CE9800F9F7DFFF082CDCD16DE02D2B14D1072C1E
:10CEA8001BDC284607F090FB0AAB661C03EB440426
:10CEB80024F8100C15F8013F303B092BFAD93446F9
:10CEC8002B78002BE9D104E0A3F13002092A09D814
:10CED800E5E7082CBDF8182009D00BB0BDE8F040F4
:10CEE800FBF7B8B9202BF8D101352646E7E7072A22
:10CEF800F3D8BDF81A00214BA0F2EE2189B240F216
:10CF0800DC55A9421B68E8D8BDF81C10A1F2EE2434
:10CF1800A4B2AC42E1D8BDF81E7004B23EB2A6423B
:10CF2800DBDB0DB2AE42D8DCA542D6DBBDF924402E
:10CF3800642CD2D1BDF8266034B2112CCDDCBDF8FA
:10CF48002050B42DC9D8BDF82240B42CC5D812B28F
:10CF58004FF00E0E0EFB0233A3F81B116421A3F849
:10CF68001901A3F81D7183F8205183F8214183F832
:10CF78001F1183F822610BB0F0BD00BF2010002004
:10CF880073860108F0B504468FB0204607F0C5FA4D
:10CF9800C5B225BBAC48AD4C01F06EFF94F8D61075
:10CFA80009B9AB4854E049B294F8D42094F8D53084
:10CFB800009194F8D710019194F9D810029194F93E
:10CFC800D910039194F8DA100491A2482946013542
:10CFD800F9F73FFF102D04F10704DFD1E1E7204600
:10CFE8009D49052207F0A2FA0546B8B929469B488B
:10CFF800702207F04EFA9A4B196828460E2303FB55
:10D00800001301300022082883F8232183F8242103
:10D0180083F8252183F82621F0D113E12046914990
:10D02800042207F083FA05462046002D4AD1202124
:10D0380007F065FA002800F00581461C304607F025
:10D048006CFA2C460746884B53F824502DB987486C
:10D058000FB0BDE8F040F9F7FCBE30462946FAB2F9
:10D0680007F064FA01340028EDD1784A02F1700122
:10D078001646002382F8DA3082F8D63082F8D530A6
:10D0880082F8D43007328A42F3D1794901EBC401DE
:10D0980091F88022934210DAD1F88472C3EBC3026C
:10D0A800B0183A4400F1D4011768C0F8D4709088D9
:10D0B800888092798A710133E7E729466D48F9F744
:10D0C800C8FE90E06C49072207F030FA0546204672
:10D0D800002D4AD1202107F012FA064607F01DFA62
:10D0E800C4B274BB6548F9F7B4FE214664480134FC
:10D0F800F9F7AFFE0E2CF8D15548F9F7AAFE00242F
:10D1080060482146F9F7A5FE0025554A5E48116892
:10D118000E2202FB04120123D2F823215B49AB4003
:10D1280013425B4B05F1010508BF1946F9F791FE5B
:10D138000E2DEAD146480134F9F78BFE082CDFD1D1
:10D1480080E03046534907F043FA2C4600284CD07B
:10D15800022C4FD007F038FA06AB4E4943F82400AA
:10D16800002007F035FA0134F0E74A4907F030FAB1
:10D17800002460B1082C38D007F026FA06AB4549E0
:10D1880043F82400002007F023FA0134F1E7082CC3
:10D198002BD1069B0F2B28D8DDF81CE0BEF1070F1A
:10D1A80023D8089F0D2F20D8099E06F16402C82AAB
:10D1B8001BD80A9DFF2D18D80B98642815D80C99F0
:10D1C800642912D8884210DA0D9C032C0DD8324AF3
:10D1D800C3EBC303134483F804E05F719E71DD71F0
:10D1E800187259729C722D4CCFE60FB0BDE8F04012
:10D1F800FBF730B8069B072B20D807990D291DD8B7
:10D208000278722A0DD06E2A18D1154A12680E209B
:10D2180000FB032301228A40D3F8231121EA0202EA
:10D2280009E00F4A12680E2000FB032301228A40FE
:10D23800D3F823110A43C3F8232101E0FBF70AF8C6
:10D248000D4CA2E60FB0F0BD9B86010848200020D7
:10D25800538F0108C6860108DE8401081C210020BE
:10D268002010002009850108006C01080E850108BE
:10D27800406A01081D85010893860108D8850108C0
:10D28800E28601080F8E0108E7860108D49101089B
:10D298008E920108EB86010818210020EA81010816
:10D2A8002DE9F743047805468CB9324D95F89F125D
:10D2B800B5F89C2295F89E322F48009121460134FA
:10D2C800F9F7C7FD102C05F10405EFD14EE007F082
:10D2D8007BF90F28044636DC2846202107F00FF991
:10D2E800264EE4B2D6F83880451CA400002728460C
:10D2F80007F06AF95FFA87F9B9F1010F83B208D02C
:10D30800B9F1020F0BD0B3F5B47F24D2B26B13532B
:10D318000AE0FF2B1FD8B36B2344987004E0FF2B5F
:10D3280019D8B36B2344D87028462C2107F0E7F8A6
:10D33800054608B1013502E0B9F1020F0BD10137FA
:10D34800032FD4D112E00E4800210F2203B0BDE80C
:10D35800F043FAF7FCBE08EB04000021042207F0B2
:10D3680098F803B0BDE8F043FAF774BF03B0BDE81E
:10D37800F08300BF48200020ED860108E01C002053
:10D388009C8401082DE9F0412DED048BB3498AB046
:10D39800044607F087F8B249002820460CBF01264A
:10D3A800072607F07FF8AF490028204608BF022665
:10D3B80007F078F8002808BF0426F10740F1068135
:10D3C800A948AA4C01F058FD002001F05BFBA848D1
:10D3D80001F052FDA74801F04FFD6279A64BA7481E
:10D3E80003EB82032546D3F8BC11F9F732FDA448B4
:10D3F800F9F72FFD4FF00008274695ED058AB5EEA1
:10D40800408AF1EE10FA04D19E48F9F722FD002572
:10D4180070E09D48D5ED069A95ED079AD5ED088AF6
:10D428004146F9F716FDB5EEC08AF1EE10FA02D5BD
:10D43800202001F019FDB0EE480A06A8F9F79EFB76
:10D4480001469248F9F705FDF5EEC09AF1EE10FA9B
:10D4580002D5202001F008FDB0EE690A06A8F9F708
:10D468008DFB01468948F9F7F4FCB5EEC09AF1EE58
:10D4780010FA02D5202001F0F7FCB0EE490A06A800
:10D48800F9F77CFB01468148F9F7E3FCF5EEC08A21
:10D49800F1EE10FA02D5202001F0E6FCB0EE680AA1
:10D4A80006A8F9F76BFB08F1010801467848F9F777
:10D4B800D0FCB8F10C0F05F110059ED1A4E749B2D4
:10D4C80094F8D42094F8D530009194F8D7100191AD
:10D4D80094F9D810029194F9D910039194F8DA10BC
:10D4E80004916C4829460135F9F7B3FC102D04F175
:10D4F800070403D094F8D6100029E0D100254FF096
:10D508000E0808FB05F80024634AD26B4244012345
:10D51800D2F80A20A340134240F0948001340E2C24
:10D52800F2D10135082DEAD15C485D4C01F0A4FC2C
:10D53800D7F8088054F8041F19B15A48F9F789FC3C
:10D54800F8E70D46584B53F8254054B10123AB403A
:10D5580013EA080F03D055482146F9F77AFC01353C
:10D56800F0E7534801F088FC21467B180AAA93F893
:10D578008A3113444F4A8A5C03F8102C0131082978
:10D58800F3D1002306A94C488DF82030F9F761FC47
:10D598004A4801F071FC4A48FBF792F9494801F002
:10D5A8006BFC4748FAF75CFE474801F065FC4448C5
:10D5B800FFF776FE4548F9F74CFC4020FFF722FCC0
:10D5C800434801F059FC3E48FBF720FAB20726D53C
:10D5D800404801F051FC404801F04EFC384801F049
:10D5E80091FA3E4801F048FC3548FAF7BDFD3C4841
:10D5F80001F042FC3248FBF7B5F83A48F9F729FC44
:10D608002F48FAF739FF384801F036FC2C48FFF765
:10D6180019FC2E48F9F71DFC8020FFF7F3FB730770
:10D6280016D5324801F028FC314801F025FC244881
:10D6380001F042FA2548F9F70CFC4FF48070FFF727
:10D64800E1FB05E0294622462A48F9F702FC65E78E
:10D658000AB0BDEC048BBDE8F08100BF018701086A
:10D668003C8B0108088701080E8701084820002024
:10D678001C8701082E870108406A01083A870108BB
:10D6880045870108528701085F870108D785010887
:10D69800F78D010867870108E01C002086870108CC
:10D6A800646C010896870108686C0108A487010862
:10D6B800B18701081E830108BD870108C6870108D4
:10D6C800EA810108D5870108E1870108538F01081D
:10D6D800EF870108FC8701080F8801081D880108E9
:10D6E80027880108368801084488010850880108FD
:10D6F8006188010873880108054B98420CBF054AE8
:10D70800054A138801339BB213800020704700BF7D
:10D7180000540040E00F0020E20F0020084A136880
:10D728009B050BD5074B00211970074908684FF670
:10D73800FE7303400B604FF400735360704700BFE3
:10D7480000000240FC2B0020300002402DE9F04789
:10D75800664D2B6866490A78581C02F0FF068E460B
:10D768000AB10346F6E72B60687BAB6895F80C8036
:10D77800AA7B374639B2202900F09B80DFF880C1A8
:10D788000CEB81033CF82110DC789B78C3F1FF0394
:10D798009BB2002B65D0C3F1FF0363434FF03C0CF1
:10D7A8001B12B1FBFCF9B9F1050F5DD8DFE809F0F0
:10D7B800030B1A293A4AE01ADAB24143B1FBFCF0EA
:10D7C8001044C0B251E0B1FBFCF00CFB101189B25F
:10D7D800DAB2C1F13C01E31A4B432046B3FBFCFC2F
:10D7E80094442CE0B1FBFCF00CFB10115FFA83F8B9
:10D7F800E21A89B24A43B2FBFCF24244D2B2204652
:10D8080032E0B1FBFCF90CFB191189B25FFA83F81D
:10D81800E01AC1F13C014843B0FBFCF04044C0B2FF
:10D82800224621E0B1FBFCF80CFB1811D8B289B2F2
:10D83800E31A01FB03F2B2FBFCFC224684445FFAC4
:10D848008CF412E0B1FBFCF80CFB181189B2D8B2C9
:10D85800C1F13C01E31A4B43B3FBFCF20244D2B2E0
:10D8680003E02246204600E044464FEA042C4CEAF6
:10D87800004C4CEA020C172306F117014FF001087F
:10D8880008FA03F8C91A18EA0C0F89B2DFF874808D
:10D8980014BF4FF011094FF0090913F1FF3308F8CD
:10D8A8000190E9D218360137B6B2BFB2114BA04683
:10D8B80060E7AA73AB60104AE98001238EF8003054
:10D8C8000E4985F80C8040F22A336873AE805360A5
:10D8D80000234B620B889BB243F001030B80136853
:10D8E80043F001031360BDE8F08700BF201D00204E
:10D8F800FC2B00202C1D0020300002400044014079
:10D908007A0D00203103002073B506460D46002429
:10D9180001232A88A34013421AD0AA78009302F060
:10D9280003038DF80430EB78022B03D0032B0CBFD4
:10D93800032301238DF805303046C2F301136946ED
:10D94800C2F381028DF806308DF80720F8F7ECFE57
:10D958000134102CDCD102B070BD2DE9F04F734EAC
:10D96800F57B07460C4687B011469A4600686B1C43
:10D97800914622464FF0020BF37300F041FB3B89BE
:10D988007868ADF8043001A98DF806B08DF807B0B5
:10D99800FFF7BAFF0023ADF80A30ADF81230ADF842
:10D9A800163070230193BA7A3C68CDF80CA0012395
:10D9B80006F110082D01ADF808304FF48073A84423
:10D9C800ADF810B0ADF814300C2A7ED8DFE802F0BC
:10D9D800077D7D7D0F7D7D7D387D7D7D5E002046C8
:10D9E80001A9F8F7EDFCA36943F0080326E0236AD0
:10D9F8004F4823F010032362236A6168A26922F06A
:10DA0800807222F4E642844242F4E04206D000F5F5
:10DA18000060844202D043F0300307E023F0E003C3
:10DA280021F4406143F0300341F480616160A261F8
:10DA3800C4F838A02362A36943F40063A36144E0F7
:10DA4800236A3B4823F480732362226A6168E3698E
:10DA5800844223F0730343F0700306D000F500609E
:10DA6800844202D042F4407207E022F4606221F45A
:10DA7800405142F4407241F480516160E361C4F85E
:10DA88003CA02262E36943F008031DE0236A2848AA
:10DA980023F480532362226A6168E369844223F491
:10DAA800E64343F4E04342F4405203D000F50060FB
:10DAB800844201D141F480416160E361C4F840A02F
:10DAC8002262E36943F40063E3613A7B3B681AB17D
:10DAD8005A6C42F400425A641A8892B242F0010227
:10DAE8001A80BA7A0C2A18D8DFE802F00717171735
:10DAF8000B1717170F1717171300721903F13401B3
:10DB08000AE0721903F1380106E0721903F13C01C9
:10DB180002E0721903F14001116135444046A5F84D
:10DB280018906B6107B0BDE8F08F00BF201D002082
:10DB3800002C0140F8B53A4E3A4C4000C7B24FF4B9
:10DB480020453068C4F8D050D0F818E01EF4004FD3
:10DB580005D0AE46013DBEF1000FF5D116E0D0F874
:10DB680004E0314D0EEA050545F490353D43456026
:10DB78004FF42045C4F8D050D0F818E01EF0020F3A
:10DB88002DD1AE46013DBEF1000FF5D1C4F8D050FD
:10DB98001FE02946013D0029F8D081694906F8D5DA
:10DBA800C4F8D05020494568294041F0007141F43B
:10DBB800105141EA0241394341604FF42041A2B17A
:10DBC800306885696D071ED411F1FF31F9D2C4F8A8
:10DBD800D010FFF791FD003018BF0120F8BD4FF4B9
:10DBE80020458162C4F8D050D7E73068C4F8D01017
:10DBF8000B46826992060CD41A46013B002AF8D1DA
:10DC0800C4F8D030E5E7416A03F8011B013AD2B203
:10DC1800D3E7C4F8D0302023C3610120F8BD00BF8A
:10DC2800DC0F0020201D0020009800FC400070B58B
:10DC3800C5B23248324B00684FF42044C3F8D04094
:10DC48008669360404D52646013C002EF8D113E037
:10DC580046682C4C344044F0807444F490342C438F
:10DC680044604FF42044C3F8D0408669B60729D4ED
:10DC78002646013C002EF8D1C3F8D0401CE02146CE
:10DC8800013C0029F8D081690E06F8D544681D4981
:10DC9800214041F0007141F48031294341604FF443
:10DCA8002041C3F8D0108469A40711D40C46013967
:10DCB800002CF8D1C3F8D010FFF71EFD003018BFB4
:10DCC800012070BD4FF420448162C3F8D040DAE7E8
:10DCD80082624FF42042C3F8D0208169890606D4B5
:10DCE8001146013A0029F8D1C3F8D020E4E7C3F877
:10DCF800D0202023C361012070BD00BFDC0F0020AD
:10DD0800201D0020009800FC026D036B70B50446CE
:10DD1800D5699BB9A90611D5C36A1BB1908C80B28D
:10DD280098470BE0E169928C40694E1CD2B2E661DB
:10DD38004254E169E268914228BFE361616BA1B98D
:10DD48002A0612D5636AA26A9A42236D09D0501C2A
:10DD5800A669A062B25C1A852369984205D3A162BC
:10DD680003E01A6822F080021A602B0742BF236D75
:10DD780008221A6270BD026BC168034610B540697B
:10DD880042B11A6C8C1A013A005D08BF0A46C0B24B
:10DD98001A6410BD1A6A805C01328A4228BF0022C8
:10DDA800C0B21A6210BD436B13B190F844007047BB
:10DDB800836A406A1B1A584258417047036B13B173
:10DDC8005B68016C01E0C369016A8B423CBFC268B1
:10DDD8009B18581AC0B27047836A8169426B19440C
:10DDE800D160416A99429DBF0169CB1A5360CB1A31
:10DDF80096BF0023536083624FF0000380F84430DD
:10DE0800136888BF816243F0010313607047436A57
:10DE18008269D154436A02690133934228BF0023BF
:10DE28004362436B1BB11B68DB0705D4D4E7026D63
:10DE3800136843F0800313607047274A73B553692A
:10DE4800264C43F400135361032369460825012631
:10DE58008DF80530204600238DF806308DF8073000
:10DE680000958DF80460F8F75FFC1D4AA5611388DA
:10DE780023F040031B041B0C1380138823F0380382
:10DE88001B041B0C2B43138013889BB243F04003E5
:10DE980013802420258501F07BFD802001F078FD8A
:10DEA800A5616420FCF7FCFF2585202001F070FDAA
:10DEB800AF2001F06DFD3046A561FCF7F1FF258527
:10DEC800232001F065FD602001F062FDA56164205A
:10DED800FCF7F1FF02B070BD0010024000100048CE
:10DEE800003001402DE9F0410369C76805460E4638
:10DEF8001F40002F35D0B7FA87F24FF00043D340C8
:10DF0800DB432B611F40A2F11B03042BF1D8DFE890
:10DF180003F0221F1C190300746A24B1013C00237A
:10DF2800A4B2736201E0EC6AA4B2D6F82080B8F11A
:10DF3800000FDED0D8F80030404621469847D8F880
:10DF48000480F4E73068696B07E07068A96B04E047
:10DF5800B068E96B01E0F068296C036889B29847FA
:10DF6800C7E7BDE8F0814171FEF7B4BA8160FEF7FA
:10DF7800B1BA01480149B5E70048014054160020EC
:10DF880001480249AEE700BF0034014004160020F2
:10DF980001480249A6E700BF0034014004160020EA
:10DFA800014802499EE700BF00080040DC15002038
:10DFB8000148024996E700BF00040040B41500205C
:10DFC8004FF0804000498DE78C15002010B5054CB6
:10DFD80005482146FFF786FF04F1C8010348BDE85C
:10DFE80010407FE764150020002C014000440140E8
:10DFF8000148024976E700BF002C01406415002063
:10E00800224B10B5224C5A43224BB3FBF2F2038841
:10E018000139013AA04289B292B29BB20ED004F5FE
:10E028000064A0420AD0B0F1804F07D0A4F598341C
:10E03800A04203D004F58064A04202D123F070030B
:10E048009BB2154CA04206D004F58064A0421CBFC8
:10E0580023F440739BB203800D4BC1629842028542
:10E068000FD003F5006398420BD003F54063984244
:10E0780007D003F58063984203D003F58063984284
:10E0880001D1002303860123436110BD40420F00E4
:10E09800002C014000A24A0400100040134B800AE3
:10E0A800984220D00AD84A3B984212D0013398426D
:10E0B80011D0B0F5801F14D1012070470C4B984245
:10E0C8000BD0013398420AD0053B984209D104206D
:10E0D80070470220704703207047052070470620CC
:10E0E8007047FE2070470020704700BF4B001000AB
:10E0F80051001000F8B50468064620460F4615463C
:10E10800FFF7CCFF06284BD8B27A910847B902230B
:10E118008B40D4F80CE0DB439BB203EA0E03E360C8
:10E128000A23204A03FB001342F82370043342F801
:10E13800235015463FB1B17AE268890802238B4023
:10E148009BB21343E360282202FB00522032EFF314
:10E158001286502383F3128803B203EB8303DB0098
:10E1680003F10C011C3329442B4451F8047F17B1E7
:10E1780017600A6804329942F7D100231360F3B29A
:10E1880083F31188282303FB0050036A1BB1E3685B
:10E1980043F0010303E0E2684FF6FE731340E360C7
:10E1A800F8BD00BF641500200048ADE5201E002022
:10E1B8000048A9E5741E00200D4B0E484FF400528C
:10E1C8005A600D4A11684FF6FE730B401360D0F881
:10E1D800882011684FF6FE730B401360826FC36F7F
:10E1E8009A4201D05430F7E5012380F898307047FF
:10E1F80000000240201E00204400024010B54B8859
:10E20800DC0641BF2F4B14791B6853F8244044BFE8
:10E218002D4B43F820404B889B0641BF294B54792E
:10E228001B6853F8244044BF274B43F820404B88D1
:10E238001C070ED5254B0C781B78B3EB141FA1BF18
:10E24800204BD4781B6853F82440A4BF1E4B43F8D6
:10E2580020404B889B070ED51D4B0C781B78B3EBE1
:10E26800141FDFBF174B54781B6853F82440DCBFDA
:10E27800154B43F820404B88DC070FD5154C0B781D
:10E28800247803F00F03A342DFBF0E4B14781B68FA
:10E2980053F82440DCBF0C4B43F820404B885B0705
:10E2A8000FD50B780C49097803F00F038B42A1BFF7
:10E2B800044B92781B6853F82220A4BF024B43F802
:10E2C800202010BD181D00207A0D00209714002072
:10E2D800951400209414002096140020254A2648FE
:10E2E80026490023F0B5156803700B701C461A46C2
:10E2F8002E1976884EB92F5D3FB9037000230A7036
:10E308004B7007781C461A460CE0360548BF0132A8
:10E3180004F1040403F1010348BFD2B2802CDBB23C
:10E32800E6D1EAE7E0B2B8420CD215F824000609B3
:10E338009E4200F00F00A8BF731C9042A8BF421C69
:10E348000134EFE78A704B70C2F3470102F0010213
:10E358000A444C1E0A490B480A70C3F3470203F0EB
:10E368000103134404700849501E084A08701370CA
:10E37800F0BD00BF801300208C140020C81E0020B0
:10E38800961400209414002097140020951400205F
:10E398002DE9F04FC24BDA682DED028B1A61C14AA4
:10E3A8001168D960C0490B6843F020030B60BF4B6C
:10E3B8001978012990460CBF002201221A70BC4B23
:10E3C8001A78910789B040F13D83BA490978042940
:10E3D80040F23883B849097801F0040101F0FF00E0
:10E3E80011B922F001021A701B78DB0702D408B1B8
:10E3F800FDF732FFB149CA78531C052293FBF2F2AC
:10E4080002EB82029A1AAE4BCA701B7803939200F1
:10E418000023AC4CDFF8CCC2DFF8D8925CF82310AC
:10E4280091FBF9F504F1080004F1100640F82350B7
:10E43800A54844F8231000FB051142F2107091FB27
:10E44800F0F080B226F813004FF0140E04F1140611
:10E4580004F13C0A0EFB036E5AF823605EF8027062
:10E468004EF80210F61B314444344AF823100526AE
:10E4780091FBF6F109FB051144F82310039C012CCC
:10E488004FEA830BE24605D10238B0F5797F98BF91
:10E498004BF80C100BB90123BBE7884CD8F80030B7
:10E4A800226D9FED8A7A8A4E8A4D9B1A07EE903A22
:10E4B800F8EE677AD8F800302365C7EE877A7C4B88
:10E4C8001B78B7EE008AF4EEC87AF1EE10FA58BF5E
:10E4D800F0EE487A13F00103C4ED157A12D005AABC
:10E4E80000927D4B06AA01920CCB9AE80300FDF737
:10E4F800B1FD6421059A069BB2FBF1F293FBF1F39F
:10E50800328000E033802B8094F858306B48002B21
:10E518003BD0D0ED157AC26DDAF80030C8EE276A24
:10E528009B1A026E022507EE103AB8EEC77ADAF89F
:10E53800043027EE267A9B1AFDEEC77AB0F96620DA
:10E5480017EE901A07EE903A644BB8EEE77AD3EDDF
:10E55800007A67EE277A67EEA67AFDEEE77A17EE7D
:10E56800903A02FA83F3B0F9642093FBF5F302FAC8
:10E5780081F29BB292FBF5F292B2A0F86A30A0F851
:10E588006820A0F86630A0F86420012384F8583089
:10E59800534BDAF804101B88DAF80000474D514E47
:10E5A800216603F03003E065002B00F04B8205F193
:10E5B8007403009305F178030193EA6E2B6FFDF75E
:10E5C80049FD72682B6F9B1A07EE903A434B3268ED
:10E5D80093ED007AEB6EF8EEE77A9B1AEB67384B0F
:10E5E80067EE877A1B78FDEEE77A012BC5ED207A76
:10E5F80003D0022B00F0DF8024E2D5ED287A3A4BD5
:10E60800D5ED215A95ED255A95ED156A95ED264AD1
:10E61800D5ED274A35491D68B1EE677ABDEEC77A50
:10E62800FDEEE77A17EE10EA17EE90CA0020304A9E
:10E6380091ED007A52F8207007EE907AF8EEE77ABA
:10E64800A2F1140367EEA57A33F81060FDEEE77ABD
:10E65800283217EE903A9B1B9BB222F810301BB25F
:10E6680007EE903AF8EEE77A3B4467EE857A440085
:10E67800FDEEE77ACDED037A07EE903AF8EEE77A09
:10E68800BDF80C8067EE847AA7EE867AFDEEC77A2D
:10E6980017EE902A724531DB6245A8BF62462EE02C
:10E6A800AC0600200C200020D010002046100020CE
:10E6B800D4100020DA100020FD2B0020C81E0020F6
:10E6C8000C0F0020CC1E0020806967FF00007A44F0
:10E6D8004E11002050110020481000200801002091
:10E6E80098110020DC100020100F0020400F00209F
:10E6F800441F002080969800DB0FC940724607EE41
:10E70800902AF8EEE77A5FED046AC1ED007AFDEE33
:10E71800E77A313617EE903A43449AB2AB78D1EDA6
:10E72800027A07EE103AB8EE477A4B684F6027EE48
:10E73800267AFB1A88EE077AB6B2622E06EE903A6F
:10E74800F8EEE66A37EE067AC6EE866A86EE077A4D
:10E7580076EEE76AE7EE267AC1ED047AC1ED027A31
:10E768000FD964EEA77ABA4EFDEEE77A17EE903A23
:10E77800B3F5FA6FA8BF4FF4FA63B342B8BF334694
:10E7880000E0002313441BB240F6B8329342A8BFFE
:10E798001346B04A9342B8BF1346AF4AA352AF4A92
:10E7A800142303FB002351F8142B1A60002840F0AF
:10E7B800498101203BE7AA4BD5F874801F68D4F83B
:10E7C80078903E89DFEDA78A4FEA58039E4228BF1A
:10E7D8001E46B5F8A8301AB29642C3BFD5ED157AD1
:10E7E8009FEDA17A67EE877AB6B2C1BFFDEEE77AF0
:10E7F80017EE906AF618B6B2C8BFA5F8A860D4F8A4
:10E80800AC50C5EB09052846FDF768FC0028D8BFC1
:10E81800404241F293129042CCBF0020012088B3BD
:10E8280007EE905AB8EEE70A20EE280AF8F73FFB01
:10E8380007EE908AF8EE677A40F6B83320EE270A9A
:10E84800FDEEC07ACDED037ABDF80C20A4F8B02017
:10E8580012B29A42A8BF1A467E4B9A42ACBF09EB45
:10E8680002034B4448F6A042934203DDA3F50C4350
:10E87800A03B04E0002BBCBF03F50C43A033C4F855
:10E88800B43001E0C4F8B490D4F8B450C5F50C53D2
:10E89800283307EE903AF8EEE77A67EEA88AB0EEEA
:10E8A800680AF8F767FB8DED070AB0EE680AF8F713
:10E8B800FEFAD4ED317AD4ED2E4AD4ED155A94ED02
:10E8C8002F4A94ED305A65498DED060AB1EE677A04
:10E8D800BDEEC77AFDEEE77A0DF1180E17EE10AA15
:10E8E80017EE90BA0020614AFEEC016A32F9103046
:10E8F800DFF88C9107EE903A07EE106AF8EEE77AA7
:10E90800B8EEC77A3C32D6EE877A4FEA400CFDEE75
:10E91800E77ACDED037ABDF90C30B3F57A7FA8BF5D
:10E928004FF47A734B45B8BF4B461FFA83F922F868
:10E9380010900FFA89F207EE902AF8EEE77A27EEA0
:10E94800A47ABDEEC77A8DED037A27EE847AD1EDED
:10E95800007ABDF80C90E7EE257AFDEEE77A17EE1F
:10E96800902A524503DB5A45A8BF5A4600E0524652
:10E9780007EE902AF8EEE77A9FED3D6AC1ED007A3E
:10E98800BA7891ED027A06EE902AF8EE666A4A683D
:10E998004B6066EE866A9A1AC8EE266A143106EE4D
:10E9A800102AB8EEC66A76EEA56A86EE256AC5EE26
:10E9B800A66A36EE476AA6EE867A01ED017A01ED7F
:10E9C800037A25EE077ABDEEC77A17EE103ABDEE48
:10E9D800E77A4B4417EE102A13441BB240F6B832BC
:10E9E8009342A8BF13461B4A9342B8BF13461A4A1C
:10E9F8002CF802301F4A142303FB0023C3ED007ACE
:10EA080008B901206FE73B7923B1642395FBF3F53F
:10EA1800194B1D803B8898450DD9D4F8AC30A06FB0
:10EA2800C01AFDF75BFB80EAE072A2EBE07242F2EB
:10EA380010739A4206DD114B01221A700E4BB4F87E
:10EA4800C8201A8009B0BDEC028BBDE8F08F00BF6A
:10EA580030F8FFFF48F4FFFF940F0020680F0020F4
:10EA6800100F0020D30237390000C842301F0020A1
:10EA7800DB0FC940400F0020080F00200C0F0020BA
:10EA880018FCFFFF07B5064B0093064B0193064998
:10EA9800064A074B0748F8F7DCF903B05DF804FBB2
:10EAA800047F0108D97E01088E8D01089F8D010819
:10EAB800F87E01086E8D010808B5037833B90C4B50
:10EAC8000C481978BDE80840F8F7C3B905F07CFD93
:10EAD80002280CD8064B1870074B0C2202FB00309A
:10EAE800064B06301860F8F7D1FB0548E5E708BD86
:10EAF800941F0020A68D0108E82700204010002060
:10EB0800EA81010808B503783BB90B4B0B4893F829
:10EB1800A417BDE80840F8F79CB905F055FD022890
:10EB280008D8054B83F8A407F8F71AFBF8F7D2FBC7
:10EB38000348E8E708BD00BF48200020AA8D010867
:10EB4800EA81010838B5037803BB214B1B68013300
:10EB58000F2B07D81F490C2202FB03121C4695688D
:10EB68002DBB00E01C4601340F2C01DD002400E021
:10EB780005D818490C2202FB04129568BDB99C42BD
:10EB8800F1D11548BDE83840F8F763B905F01CFD28
:10EB98000F28044605D80F4A0C2303FB00239D6861
:10EBA8002DB921460D48BDE83840F8F752B9084B51
:10EBB8001C60FCF7DDFA21462A460948F8F749F9AE
:10EBC8000C235C43034B185DBDE83840FCF7E8BAFA
:10EBD8000C010020506E0108B78D0108CD8D010889
:10EBE800E58D010873B5037813B9F9F733FB3DE0F8
:10EBF8001F4901AA05F049FD00240146264625467D
:10EC080099B134B1012C08D1084605F0DDFC06465F
:10EC180003E0084605F0D8FC05461549002001AA7E
:10EC280005F033FD01340146EAE70B2D02D91148FE
:10EC38000C220BE0022C10D1A6F57A73B3F57A7F7B
:10EC480007D90D484FF47A714FF4FA62F9F77FFA51
:10EC58000CE00A4B03EB45035E80084B084803EBC6
:10EC680045032946B3F90220F8F7F3F802B070BD5E
:10EC7800EB8601089C8401085E8A0108941F002025
:10EC8800FC8D010838B50D4C23688342054606D132
:10EC9800F9F7E9FF204600214C2205F0FAFBE36C66
:10ECA800AB4209D12846F9F7DEFF054800214C227E
:10ECB800BDE8384005F0EDBB38BD00BFAC11002001
:10ECC800F8110020034B1A68D379591C1344D171E9
:10ECD800187A70477811002010B5FFF7F3FF84B257
:10ECE800FFF7F0FF04EB002080B210BD10B5FFF76E
:10ECF800F3FF0446FFF7F0FF04EB004010BD064B9E
:10ED080010B5044621461868FCF7CEFA034B1B6879
:10ED180098796040987110BD7C110020781100200E
:10ED2800014B1B689879EAE77811002038B504464A
:10ED380024200D46FFF7E3FF4D20FFF7E0FF002CEE
:10ED4800084C14BF21203E20FFF7D9FF236800227A
:10ED580028469A71FFF7D3FF236893F84900BDE866
:10ED68003840CCE77811002001460020DEE710B5D6
:10ED78000446C0B2FFF7C3FF200ABDE81040BEE753
:10ED880010B5044680B2FFF7F2FF200CBDE8104032
:10ED9800EDE737B582888368044610060D4641BF03
:10EDA8002B4991F8A4174FF4CC7000FB0133D1051F
:10EDB80044BF2849097802F03F0244BF01EB4101F2
:10EDC80003EB8103042A12D006D8012A0DD0022AA7
:10EDD80032D193F9001030E0102A0AD0202A0AD044
:10EDE800082A29D1B3F9001027E0197825E01988F5
:10EDF80023E0196821E093ED000A6846F7F7BEFEA4
:10EE080001461548F8F725F805B3D4ED037A6846A6
:10EE1800B8EEE70AF7F7B2FE01461048F8F719F816
:10EE280094ED040A6846B8EEC00AF7F7A7FE014653
:10EE38000A48F8F70EF809E000210948F8F709F838
:10EE480025B10848E1682269F8F703F803B030BD36
:10EE580048200020941F0020D7850108D08501088C
:10EE68000F8E01080B8E0108024B0146D869FCF78A
:10EE78001BBA00BF941F002010B5441E14F8011FD0
:10EE880021B1034BD869FCF70FFAF7E710BD00BFB3
:10EE9800941F002010B503781BB90A48BDE810403C
:10EEA800EAE705F091FB0446062899BF2146064883
:10EEB80006480621F7F7CDFF601E40B2BDE81040B6
:10EEC800F9F73ABE128E0108598E0108858E01089D
:10EED800F7B52B492B4B08782B4D1C682B4B05EBB2
:10EEE80080001A882A4BD0F8C0101B782948009156
:10EEF8004FF47A71B4FBF1F1F7F7ABFF26484821DC
:10EF0800F7F7A7FF254B1F680026F3B205EB83022E
:10EF1800D2F8D010E9B101249C403C4217D0220716
:10EF280015D01F4AD25C0B2000FB0323164A1D484C
:10EF380002EB8303D3F8F020F7F78BFF022C06D1FE
:10EF4800194B93F8281011B11848F7F782FF0136CA
:10EF5800DBE71748FFF790FF164B17481A68174B5F
:10EF68009A420CBF164B174B1A88174B198892B246
:10EF78004FF4FA6303B0BDE8F040F7F76ABF00BF8B
:10EF8800201100200C200020506E0108C010002025
:10EF980010010020B08E0108F38E0108D010002067
:10EFA80018010020038F0108941F00200B8F01080F
:10EFB800538F0108DC0F00200F8F01080054004018
:10EFC800E00F0020E20F0020D80F00202DE9F041CB
:10EFD8000024804625460F4EA7594146384605F07D
:10EFE800DBFA58B139460C48F7F733FF30190021DE
:10EFF800FFF7CFFE0948FFF73FFF0135143440F60D
:10F0080094439C42E7D11DB90548BDE8F04133E778
:10F01800BDE8F081F06F01086D860108538F010883
:10F028000E8501082DE9F04F2DED028B83B00546C2
:10F0380005F073FA064620B1012818D12B782A2B3F
:10F0480015D15C48FFF718FF00245B4D5B486159F8
:10F05800F7F7FFFE28193146FFF79BFE5848FFF7E0
:10F068000BFF143440F694439C42EED19CE02846B2
:10F078003D2105F044FA002800F08F8003469946A8
:10F0880013F8012D202AFAD0441C204605F09CFADA
:10F0980080462046F7F7E8FCC5EB0909B0EE408A40
:10F0A8000026DFF834A1142202FB06F40AF5D07B0F
:10F0B80054F80B70384605F030FA03461A462846CD
:10F0C8003946019305F032FA019B00285BD15FFABB
:10F0D80089F29A4257D10AEB0402D2ED6B7AF8EE24
:10F0E800E77A0BEB0405B4EEE78AF1EE10FA48DB99
:10F0F800D2ED6C7AF8EEE77AB4EEE78AF1EE10FA20
:10F108003FD8B2F8A431D2F8A82113F0200F08BFD5
:10F1180008EE108A1C0641BF2A4991F8A4174FF43B
:10F12800CC7404FB0122D90544BF2749097803F0B0
:10F138003F0344BF01EB410102EB8102042B18EEAF
:10F14800100A0BD004D8013B012B0ED810700CE02C
:10F15800102B05D0202B06D0082B06D1108004E0F8
:10F1680082ED008A01E082ED008A39461748F7F7F8
:10F1780070FE2846002103B0BDEC028BBDE8F04FBD
:10F1880007E6134803E00136A12E8AD1114803B0DF
:10F19800BDEC028BBDE8F04F6EE6284603B0BDEC2F
:10F1A800028BBDE8F04F11E703B0BDEC028BBDE860
:10F1B800F08F00BF418F0108F06F01086D860108CC
:10F1C800538F010848200020941F0020568F010803
:10F1D800618F01080E850108506E010808B50748BF
:10F1E800FFF74AFE064BD869F9F732FDFCF7BCF980
:10F1F800F7F78CFF034B044ADA6008BD818F0108DA
:10F20800941F002000ED00E00400FA0508B5054849
:10F21800FFF732FE00F036F8F7F7A2FFBDE8084026
:10F22800DCE700BF8D8F010808B50448FFF724FE0E
:10F23800F7F796FFBDE80840D0E700BFA38F0108A5
:10F248000E4B1A78692A16D15A88B2F5FA6F12D17C
:10F258001A79BE2A0FD193F8CD27EF2A4FF0000074
:10F268000BD113F8012B5040054A9342F9D1B0FA5B
:10F2780080F04009704700207047704700F8030885
:10F28800D0FF03082DE9F04FEF4C00214FF4FA624C
:10F2980085B0204605F0FDF8EC4B04F537721A608E
:10F2A800EB4B00221A70EB4B04F2A671196069232C
:10F2B8002370032363714FF48073A3604FF41673B4
:10F2C800A4F86631FA23A4F86831BC23A4F86431A1
:10F2D8004FF4FA732021A4F86E31012384F86231C7
:10F2E80084F86A1184F87E316E2184F8863105230A
:10F2F80084F87C1184F81B320A2140F2DC5384F82C
:10F308007D11A4F898312B2140F24C4384F87F11E9
:10F31800A4F89A31212140F26C7384F88011A4F882
:10F328009C31232140F2753384F88111A4F89E3171
:10F338004FF4C87140F64303A4F8A031A4F8821131
:10F3480023469918023200254FF01E09242ABE4C84
:10F3580081F8A25181F8A391F3D14FF4FA6340F2F6
:10F368007E4040F27E57DFF8E4B2A4F8C831A4F832
:10F37800CC31A4F8D031A4F8D431A4F84401052341
:10F3880040F23A70A4F84C7140F2EA5701264FF463
:10F398007A78C82219214FF0320A84F8DE31A4F8AD
:10F3A80046014FF4C87340F2DC50A4F84E7140F2A5
:10F3B800B457A4F8E221039284F8959184F8DD61AA
:10F3C80084F8DF11019184F8E06184F8E16184F840
:10F3D800E461A4F8E63184F8EA61A4F84A010290ED
:10F3E800A4F85071A4F8543184F8ED61A4F8C681EA
:10F3F800A4F8CA81A4F8CE81A4F8D281A4F84881DF
:10F40800A4F852A1A4F856A1F6F7E4FCDBF8003002
:10F4180026744FF0170E83F815E083F816E04FF0C6
:10F42800550EE673A573A58183F803E04FF00F0E20
:10F4380083F805E00199D9714FF0220E83F806E0B0
:10F4480021214FF00E0E83F80B9083F80C9083F86F
:10F4580010E059744FF0350E53214FF064092827F6
:10F468004FF02D0C83F81AE0D9764FF05A0E0A2186
:10F4780083F81C904FF0780983F80DC083F808E0F2
:10F48800997483F80A901D705F709F70DD7583F81A
:10F4980004A09D731D76DD735D765F7283F814C0DA
:10F4A8004FF4FA7CA3F84EC0DFF8C0C1C3F838C0E7
:10F4B800C3F83CC0DFF8B8C1C3F828C04FF07E5C81
:10F4C800C3F834C0F7EE087ADFF8A891DFF8A8C1CE
:10F4D800C3ED087AC3F82C90C3ED097AC3F83090CD
:10F4E800C3F848C0F1EE047A02989E774FF04B0CAF
:10F4F8004FF0000983F8501083F8525083F8517088
:10F50800C3F84090C3ED117A83F84CC084F8A6E79D
:10F51800A4F8B0074FF0410E042084F8A7E784F858
:10F52800A8A784F8A95784F8AD5784F8AE5784F88B
:10F53800AA5784F8AB5784F8AC5783F85C001520B9
:10F548000191A3F85850A3F85A50A3F85650C3EDA8
:10F55800187A83F868004048D866404818674048D9
:10F56800586783F878603F4883F8647083F865705B
:10F57800F6F776FCDBF800300199039A83F81461FA
:10F588004FF4487083F8115183F8125183F81371BE
:10F5980083F81851A3F816015E4684F8D81184F848
:10F5A800D921A4F8DA8119460E2202FB05326FF040
:10F5B800170082F81901032082F81A016FF02F0052
:10F5C80082F81B01072082F81C016FF0230082F8E3
:10F5D8001D01052082F81E0101355A2081F82001FD
:10F5E80081F821016422FF20082D81F81F2181F86C
:10F5F800220101F10E01D7D1002183F88911C82118
:10F60800A3F88A11142183F88C11A3F890211E21E4
:10F618004FF4967283F88D11A3F8922101212822C4
:10F62800A3F8942183F88E11074B03F1C0021F46FB
:10F63800C3F8149010339342FAD10B4800214022AA
:10F6480004F027FF1AE000BF482000202010002007
:10F65800941F0020401000209A99193FF6287C3FFB
:10F668003D0A773F97990108E42200208FC2F53CB4
:10F6780000002040CDCCCC3E000040400023264D69
:10F68800264C5959FA1804330868C2F89C02382BDA
:10F69800F5D104F507700021802204F0FAFE05F187
:10F6A8003801702204F5077004F0E8FEFEF716FE34
:10F6B800366800230125314604F274404FF4CC72B9
:10F6C80084F8CC3784F8CA5784F8CB5704F0D6FEB0
:10F6D80004F20C6031464FF4CC7204F0CFFE104BAC
:10F6E8001B681A68C4F8B2275A68C4F8B6279A681B
:10F6F800C4F8BA271A68C4F8BE275A68C4F8C227DB
:10F708009A68C4F8C627022384F8C85484F8603677
:10F7180005B0BDE8F08F00BFE47C01084820002058
:10F72800401000201549D1F8883043F47003C1F81F
:10F738008830134B1A6842F001021A605868114A5F
:10F7480002405A601A6822F0847222F480321A60E9
:10F758001A6822F480221A605A6822F4FE025A605B
:10F76800DA6A22F00F02DA62186B074A02401A635B
:10F7780000229A604FF000638B60704700ED00E054
:10F78800001002400CC07FF8CCFC00FF38B5094BD4
:10F7980093F8CC5765B9084C2068F9F764FA074B19
:10F7A80025601B78022B03D1BDE83840F6F7D1BAA3
:10F7B80038BD00BF48200020802800207C28002079
:10F7C800044B93F8CC371BB9034B1868FBF760BDA3
:10F7D80000207047482000208028002038B50546C2
:10F7E8000446204614F8011B21B1034B1868FBF7A7
:10F7F8005BFDF6E7401B38BD802800200FB407B535
:10F8080004AB064953F8042B01930020F7F734FAA8
:10F8180003B05DF804EB04B0704700BF93F900082B
:10F82800024B01461868FBF73FBD00BF8028002047
:10F83800F8B5011F06460023083051F8042F02F1DD
:10F8480020043F2C3AD802F108040F2C06D80232C3
:10F85800032A04D9002B08BF012300E002238142B8
:10F86800EBD1012B30680ED0022B1AD0736803F04D
:10F8780003039B0000F0030043EA0010B36803F0A1
:10F888000303184317E000F00F0040F04000FFF7B3
:10F89800C7FFB068736800F00F0040EA0310C0B2F9
:10F8A80009E000F03F0040F08000FFF7B9FF307931
:10F8B800FFF7B6FF307ABDE8F840B1E706F10C076C
:10F8C80034463A46002552F8043D03F18001FF29E9
:10F8D8004FEA850510D903F50041B1F5803F02D202
:10F8E80045F0010508E003F50003B3F1807F34BF5C
:10F8F80045F0020545F00305B242E4D165F03F004A
:10F90800C0B2FFF78DFF05F00303022B207807D064
:10F91800032B0CD0012B13D1FFF782FF60780FE087
:10F92800FFF77EFF6078FFF77BFFA07808E0FFF71E
:10F9380077FF6078FFF774FFA078FFF771FFE07832
:10F948000434FFF76DFFBC424FEAA505DBD1F8BDD3
:10F9580010B50446C0B2FFF763FFC4F30720BDE843
:10F9680010405DE710B504467F2C06D964F07F008F
:10F97800C0B2FFF755FFE409F6E7E0B2BDE8104072
:10F988004EE7430083EAE070ECE7084648E700BF2B
:10F9980040F2E9330F4A1289920704D4013B9BB223
:10F9A800002BF7D10BE00C4A40F2E93310700949FB
:10F9B8000989C9070AD4013B9BB2002BF7D1074A32
:10F9C800138801339BB21380FF2070471078C0B2B0
:10F9D800704700BF003001400C300140D81F0020A4
:10F9E8000C4B0D49DA684378D243C2F30222C2F1C4
:10F9F8000402934002781B010A44DBB282F8003308
:10FA080003780122580903F01F0302FA03F341F8AF
:10FA18002030704700ED00E000E100E073B50546D6
:10FA2800002100680122FEF7EBFA2A6813889BB2CE
:10FA380043F001031380EB7A8DF80430012400268B
:10FA480001A88DF805408DF806608DF80740FFF78E
:10FA5800C7FFEB7A1B2B0BD1192301A88DF80430B3
:10FA68008DF805408DF806608DF80740FFF7B8FF60
:10FA780002B070BDF0B5BE4CA3782DED028B013BF2
:10FA8800012B85B000F26F81E578854240F06B81EB
:10FA98002379022B00F06781B64B5B5D6371A37914
:10FAA8006D00F2EE048A1BB16319B3F9083009E05E
:10FAB8006319D4ED037AB3F90830F1EE677AC4ED2F
:10FAC800037A5B4208EE103A2369A94EB8EEC88A59
:10FAD8001A0388EE288A35D5D6ED037AFDEEE77A43
:10FAE80028EE280A17EE903AD6ED057A8DF80A30F6
:10FAF800FDEEE77A17EE903A8DF80B3004F01EFF12
:10FB0800FCEEC07A96ED060A17EE903A20EE280A27
:10FB1800ADF8083004F012FFFCEEC07A96ED070A43
:10FB280017EE903A20EE280AADF80C3004F006FFE4
:10FB3800FCEEC07A0C2017EE903A02A9ADF80E3010
:10FB4800F7F7DAFED4ED077A894BF5EE407AF1EE55
:10FB580010FA60D1D3ED067AB4EEE78AF1EE10FA26
:10FB680004DDDA6883ED068A5A61E8E0F5EEC07ACA
:10FB7800F1EE10FA40F3E38093F8202042B1022A14
:10FB880000F2DD805A6B83ED078AFA329A63D6E079
:10FB9800D3ED037A38EE678AF7EE007AB4EEE78A97
:10FBA800F1EE10FAACBF01210021D3ED0A7A69B158
:10FBB8009FED717A27EE877ADFED707AB4EEE77AF7
:10FBC800F1EE10FA58BFF0EE477A03E09FED6C7A39
:10FBD80067EE877AC3ED0A7A2369654A1B0311D554
:10FBE8008DF808105379116B0B440B205A788DF857
:10FBF8000920DA7A8DF80A205B7D8DF80B3002A98E
:10FC0800F7F77AFE0123226B84F8203063791344D6
:10FC18000022DA7291E0B4EEE78AF1EE10FA48BFFA
:10FC280083ED078AA16B636B94ED067AD4ED076ABE
:10FC3800591AC943C90F77EE667A59B9B7EE006AFF
:10FC4800F4EEC67AF1EE10FA79DDB4EEE68AF1EE5A
:10FC580010FA74DDD4ED056A454BB4EEE67AF1EEA0
:10FC680010FACCBF0126002666B1D3ED097A9FEDC4
:10FC7800427A67EE877A9FED427AC3ED097AD3ED2F
:10FC88000B7A0AE0B0EE007AF4EEC77AF1EE10FAD9
:10FC980008DDD3ED0B7A9FED387A67EE877AC3EDEE
:10FCA8000B7A07E0D3ED097A9FED357A67EE877A0C
:10FCB800C3ED097AD4ED097A206B627967EEA87AE8
:10FCC8001044FCEEE77ACDED017A9DF804304370DC
:10FCD800D4ED0B7A2769FCEEE77A3F03CDED017A84
:10FCE8009DF8042042750ED546EA41018DF80810AA
:10FCF8008DF80930C37A8DF80A300B2002A98DF8E7
:10FD08000B20F7F7F9FD94F82020194B022A11D19E
:10FD1800D3ED0A7A9FED1B7A196B67EE877A00227A
:10FD280083F82020FCEEE77A5A7917EE903A0A44D5
:10FD3800D37202E0022283F82020FCF7F9FAA279B4
:10FD48000B4B0AB1104A00E0104ADA602544D4EDA2
:10FD5800037AB5F9083000EE103AB8EEC00A80EE22
:10FD6800280A37EEC00A05B0BDEC028BF0BD00BF13
:10FD7800D81F0020BC7D0108EC51783F6F12833AF0
:10FD88000AD7833F00007A440000A0410000A0C1C8
:10FD98002B4BF0B52B4D1E6805F110002F78F31989
:10FDA8002C46597801F00401013501F0FF0219B120
:10FDB8008542F3D10020F0BD224D631B022B0ADDE2
:10FDC8001AB102EB82025200D2B215F8013B303B65
:10FDD8001A44D2B2F1E70021AC420AD919B101EBB9
:10FDE80081014900C9B215F8013B303B1944C9B239
:10FDF800F2E72E2F16D10134042000232578771935
:10FE080003EB83037F785B007F079BB244BF303DE1
:10FE18005B1900F1FF3044BF01349BB210F0FF00C2
:10FE2800ECD100E0002308484143642000FB0313A1
:10FE38000620B3FBF0F3054800FB0230F0BD00BF1D
:10FE4800200100201420002040420F0080969800D6
:10FE580030B500231A4610498C1894F83C40BCB1C0
:10FE68002E2C06D1013298B18C180444002584F850
:10FE78003C5011440A2491F83C106343A1F130042A
:10FE8800092C9CBF303B5B180E2A03D80132E2E7ED
:10FE9800184630BD002030BDD81F00200EB40FB565
:10FEA8000749019006AB01A8064A0393F6F7E4FE5A
:10FEB800019B00221A7004B05DF804EB03B0704790
:10FEC800B1690008B08401080B4A136913F4805F14
:10FED800B2F9523006D0B2F80822111A8B4208DD66
:10FEE800104401E0B2F80A028342B4BF00200120A6
:10FEF80070470120704700BFD81F0020064B1B78B1
:10FF080003F0040303F0FF001BB1044B1888C0F38F
:10FF1800C01000F001007047FD2B00209811002050
:10FF28002DE9F04F2DED028B87B000260493B24BDC
:10FF38000392B3F90270B3F900300190002FB8BFF3
:10FF48007F42002BB8BF5B429F42B8BF1F46B7F540
:10FF5800FA7F8146A8BF4FF4FA77B0460296B346B7
:10FF68003446A64D2B8813F0030F4FEA440A58D0A5
:10FF7800022C56D0A04BA24A33F80A3032F90A2094
:10FF8800022113FB0122039B5B429A4203DB039B82
:10FF98009342A8BF13469B4A32F90A209B1A049A37
:10FFA80032F91420134408EE103AFFF7A7FF68B19E
:10FFB800B8EEC80A944BB2EE048A80EE080A185DBF
:10FFC800FFF758FD20EE080ABDEEC08A18EE102A89
:10FFD80099F808305343642293FBF2F399F81C20F4
:10FFE8006FF0040B0BFB02FB5B4504DB02EB820B9F
:08FFF8009B45A8BF9B4685490B
:020000040801F1
:1000000018EE103A51F82420134442F21072934231
:10001000A8BF1346804A9342B8BF134699F81220EE
:1000200041F8243053431B1302932B8803F003023F
:10003000012A01D1022C3FD17848714A30F90A00D7
:1000400032F90A807649019A51F82460557880EA9D
:10005000E07EAEEBE07EBEF5206F4FEA84021EDC50
:10006000022C15D008EB8801090191FBF5F504215C
:1000700090FBF1F02D1A2E44B6F57A5F6849694875
:10008000A8BF4FF47A568642ACBF5650505008E095
:1000900088EAE87EAEEBE87EBEF1640FE2DD002088
:1000A00088505F497D26525892FBF6F6019AD27A23
:1000B0007243402692FBF6F69A0713D5022C11D014
:1000C0000298C7F5FA7307FB06F507FB08F203FB76
:1000D0000B224FF4FA7103FB005392FBF1F293FBF6
:1000E000F1F508E0DB0704D5022C02D0029D5A4648
:1000F00001E035464246494B33F91410042391FB85
:10010000F3F34949615C4B436FF04F0193FBF1F30B
:1001100099F85110D3184FEA440A08EE103AB1B1D9
:10012000022CB8EEC80A414B08D14A0803D09142CC
:10013000A8BF114600E001213D4802E03D4800EB28
:10014000C400D3ED000AF6F769FCBDEEC08A334B5C
:10015000394A3AF803003AF902302AF8020001B2AB
:1001600002F108001432CB1A50F824E0042193FB6A
:10017000F1F152F8243040F8241073440B4499F8FC
:10018000501042F824E04FEA840C00EE103A79B1A6
:10019000264B2A48D3ED000ACDF814C0B8EEC00AA9
:1001A00000EBC400F6F73AFCDDF814C0BDEEC00A5F
:1001B000234A2449125D10EE103A5343202293FB48
:1001C000F2F318EE102A2A44D21A2AF801201E4A05
:1001D00018EE101A4CF802101C4A4CF802501C4A37
:1001E0005B424CF80230019B01340133032C019334
:1001F0007FF4BBAE07B0BDEC028BBDE8F08F00BF53
:10020000B410002098110020F62B0020E01F0020E1
:100210005069010824140020F0D8FFFF04100020CA
:10022000B013002080C1FFFF2C140020AC1300206D
:10023000A4130020941300201C280020E0130020A9
:1002400044140020F8130020001400200C14002097
:10025000181400202DE9F04F2DED088BC94F83B005
:10026000044600933B88019713F0020F0AEE102A10
:10027000F7EE009A4CD0149BC348DD89B0F90030EA
:100280005B1B03F2F31640F2E632964203D8002BD2
:10029000B8BF5B4201E04FF4FA73B0F90220521B81
:1002A00002F2F31540F2E630854203D8002AB8BFC7
:1002B000524201E04FF4FA7294F84C0058B3934262
:1002C000B8BF1346C3F5FA7307EE903A9FEDAF7AC5
:1002D000F8EEE77A6423C7EE877A93FBF0F307EE34
:1002E000103A77EEE97AB8EEC77AB0EE699AA7EEDF
:1002F000879AF7EE006AB5EEC09AF1EE10FA0AD4CA
:10030000B4EE669AF1EE10FAC8BFB0EE669A04E059
:10031000B0EE699A01E09FED9E9ACE1C25464FF003
:10032000000ABAF1020F16F801BF9A4F4FEA4A09C4
:10033000F2EE04AA0ED1B7F904209FED977A0BF1E3
:100340000A0B02FB0BF307EE903AF8EEE77AC7EEE2
:10035000877A68E0F8EE4A7A9FED8C6A37F91A30AE
:10036000C7EE867A06EE903A8C4B33F91A3007EED8
:10037000103A1AEE103AF8EEE66AB8EEC77A5B4227
:10038000A6EEA77A07EE903AF8EEE77AB4EEE77AAF
:10039000F1EE10FA08D4F8EECA7AB4EEE77AF1EE8C
:1003A00010FAD8BFF0EE477A7D4B33F9093008EEEA
:1003B000103A009BB8EEC88A33F91A3077EEC87A43
:1003C00008EE103AB8EEC88A37EE888A88EE2A8A94
:1003D000FFF798FD40B1734B13F80A00B0EE480ADE
:1003E000FFF74CFBB0EE408A019B1A88D10704D579
:1003F000D4ED117A68EE277A15E037F909309FEDD0
:10040000667A0BF1140B03FB0BF307EE903AF8EE50
:10041000E77A9307C7EE877A42BF94ED127A28EE07
:10042000078AE8EE097A604BDFF8ACB133F909309E
:1004300095ED08BA9FED5D8A94F85110DFF89C8124
:1004400007EE103A5A4BB8EEC77AD3ED0C6A1AF899
:100450000B30E7EE667AF0EE48BAF0EE678A67EEA8
:100460008B7A0BEE103AB8EECBBA27EE8BBA8BEE46
:1004700008BAC1B1BAF1020F0AD14B0803D09942B0
:10048000A8BF194600E00121B0EE4B0A494804E03C
:100490004948B0EE4B0A00EBCA00D8ED000AF6F767
:1004A000BDFAB0EE40BAD8ED000A444995ED0B7A9A
:1004B0004FEA8A0768EEA07A394467EE877A91EDB1
:1004C000007AA7EEAA7ADFED3E7AB4EEE77AF1EE93
:1004D00010FAF0EE47AA09D4DFED3A7AB4EE677A63
:1004E000F1EE10FAC8BFF0EE67AA01E0F0EE67AADD
:1004F00089EEA07A344AC1ED00AAD119D1ED007A73
:10050000C1ED008A78EEE77A02F10C013944183225
:1005100067EE877A3A4491ED007A92ED000AC1EDD8
:10052000007A82ED007A37EE000A94F8501030EE2F
:10053000270A21B1254800EBCA00F6F76FFAF0EE62
:10054000087A80EE270A1BF80A30D5ED0E7A08EEFD
:10055000103A60EE277AB8EEC88A27EE880ADFEDF7
:100560001C7A80EE2B8AB4EEE78AF1EE10FA37D4CB
:10057000DFED187AB4EE678AF1EE10FAC8BFB0EE7C
:10058000678A2FE098110020242000200000FA4301
:1005900000000000B410002000004842F62B0020AC
:1005A000E01F002050690108041000200000C8422C
:1005B0001C280020A4130020941300206C14002099
:1005C00000007AC300007A4350280020E013002086
:1005D000000096C30000964390130020AC13002047
:1005E000B0EE678A3BEE2A0A0AF1010A30EE080AE9
:1005F00004F062F9144AB0F57A7FA8BF4FF47A701C
:100600009042B8BF1046BDEECBBA104A1BEE103A6E
:1006100022F80900FDEEEAAA0D4ABDEEC88ABB50D9
:100620000C4A1AEE903ABB500B4A18EE103ABAF147
:10063000030FBB5005F104057FF473AE03B0BDECAE
:10064000088BBDE8F08F00BF18FCFFFFF8130020F7
:10065000001400200C14002018140020044B002269
:100660001A605A60034B00221A605A60704700BF3C
:1006700024140020781400202DE9F04FAC490B78A9
:1006800013F0010F87B003F0040200F04881002A44
:1006900040F0748103F0020000F0FF04002840F0F5
:1006A0003E8143F004030B70A24B1A88A24B1A80C0
:1006B000A24B1A6812F4002F984600F01181A04B4B
:1006C00080201C70F5F748FC08B1FEF7DFFA9D4C5E
:1006D0002778012F40F004819B4D95F8CA2722B15D
:1006E00095F8CB370BB19A4203D3012385F8CA376B
:1006F0000FE01846114630B191FBF0F600FB1616DC
:1007000001463046F7E792FBF1F285F8CA2793FBE2
:10071000F1F385F8CB3795F8CC371BB18A4B002223
:1007200083F8CC27636895F8CC6703EBC30341F6E5
:100730006902934284BF40F2E242B3FBF2F3834A80
:100740008CBFDBB204231370FEB98020FAF7C6FA1F
:100750008146D0B18021FAF79DFA99F806207C4BAA
:10076000207253F8223099F90000DFF8D891B3F5E0
:10077000613F0CBF0222002202218DE80600802189
:100780003246FAF7A6FBE06008B90023A7E009F1BA
:1007900010003146142203F080FE09F13003C9F83D
:1007A000243009F1A003C9F8283009F58873C9F885
:1007B0002C30684BD8F800201B88A9F8803195F8B8
:1007C0009431654895F886910590002B634B1B6822
:1007D000C3F3C00E6B79A3F1190B02F4006CC2F3E2
:1007E000400AC2F3C03218BF0122DBF1000141EB25
:1007F0000B01012B14BF0B46012395F8CAB70493D4
:1008000095F8CB3705689B45554B1B7803932CBF58
:100810004FF0000B4FF0010B791EC9B24B1E132B8A
:1008200039D8DFE803F00C0C0C0C0C0C0C0C0A8310
:100830003BA7273B33121212353B049B9BE0039BE3
:100840008B42B4BF0023012324E02B78022B0BD171
:1008500005EB810353ED027AF5EE407AF1EE10FAE2
:1008600014BF0123002315E06B185B79003318BF18
:1008700001230FE0BCF1000F04D009F1FF30434227
:10088000434100E0634603F0010374E0134672E065
:100890005B4670E013B101238B401E43142F02D836
:1008A0000137FFB2B8E7059BC4F8846118681921C5
:1008B0007930FAF7A3FA0023C4F88C31A4F8903108
:1008C000A4F89231C4F89C31264BD4F898211B68C7
:1008D000C4F8A03184F88801C4F89421022323705D
:1008E000204B194A1B6892F8DE214FF47A7101FB04
:1008F00002331D4A1360D8F800301A0609D51B4B85
:100900001B789B0705D51A4B1B78042B01D90620B1
:1009100000E0052007B0BDE8F04FFAF745BC6ABB20
:10092000012007B0BDE8F04FFAF764BC734622E03F
:10093000FD2B0020B01000200A0F0020E81F00202F
:100940004D12002074280020482000201C010020A7
:10095000F0630108C012002020100020D0100020F9
:10096000601500200C200020BC0E0020D4100020B8
:10097000DA1000205346002B8DD191E707B0BDE877
:10098000F08F10B5154A1378590725D523F00403C5
:100990001370134B1B681B0319D5124C2378A3F15A
:1009A0000802012A0BD8FF200021F6F7A9FF0E4B01
:1009B0001B68C4F8A031FEF707FF0A2306E0012BED
:1009C00005D90A2B03D0FEF7E5FE0123237004208E
:1009D000BDE81040FAF7E8BB10BD00BFFD2B0020BA
:1009E000E81F0020742800200C200020034B1A78F8
:1009F000202A04BF00221A70704700BF002C00207C
:100A0000014B04221A607047E42B0020034B9B7AB1
:100A100013B1034B05221A60704700BFFC1400207D
:100A2000E42B00200D4B0E491A680E4B92B2134472
:100A30005B000D4A1B68C3F3090310B5136013680C
:100A40009BB201335B1000229A4206D0074851F84E
:100A5000044B20F812400132F6E710BD505C004014
:100A6000206200401E3000200C17002011170020CB
:100A7000014B00221A607047081700202DE9F84347
:100A8000664B674E1B68DFF8B881664A00254FF059
:100A9000C0099D7283F80990DD723560D8F8003086
:100AA00023F4EC4323F0700343F400739BB2C8F8C3
:100AB0000030D8F8003023F4E04323F040039BB229
:100AC00048F2800483F010032343C8F800303368F1
:100AD00012FA83F35B0040271A681F6033689BB2E9
:100AE00003F1005303F540535B0028461A68802247
:100AF0001A60D8F8003023F4F8731B051B0D23434C
:100B0000C8F80030484B93F82C10F5F7EDFAD8F8F8
:100B10000030464A464923F4804323F070039BB2D9
:100B200083F440532343C8F80030136823F4EC43A4
:100B300023F070039BB21360336811FA83F35B00F8
:100B400003201968C3F8009013683A4923F4E0437E
:100B500023F040039BB283F0200323431360136808
:100B600023F4804323F0700323439BB21360536844
:100B700023F4EC4323F0700343F4C0639BB253604F
:100B8000336811FA83F35B0019684FF480711960C0
:100B9000536823F4804323F0700323439BB25360D4
:100BA000536823F4E04323F040039BB283F0200317
:100BB00023435360D8F80C301F4A23F4EC4323F04E
:100BC00070039BB2C8F80C30336812FA83F35B00F1
:100BD00039461A684FF488721A60F5F785FAD8F822
:100BE0000C3023F4804323F070039BB283F4405312
:100BF0002343C8F80C30D8F80C3023F4E04323F03A
:100C000040031C43A4B2C8F80C402846F5F7E0F9AD
:100C10000A4B01221A60BDE8F88300BFA41100202E
:100C2000505C0040043000201C000020045C0040A8
:100C300008300020103000201C300020E42B002061
:100C4000005C0040134A144B50681B68181810B51C
:100C5000146808D011490822F8F7A5FD204610496C
:100C60000422F8F7A0FD0F4B1A68002393720E4A76
:100C7000012111600D4913604FF4E0500B601060CA
:100C80000B480B604FF4364101801160094A136034
:100C900010BD00BFB0F7FF1FACF7FF1FEE00002034
:100CA000FE000020A4110020405C0040445C004095
:100CB0001C2A0020E42B0020024B4FF480221A60F3
:100CC000704700BF1404014003788B4286BF024B7B
:100CD00033F8110000207047202A002070B5002250
:100CE0001346234914180C44247E83EA0423082461
:100CF00013F4004F4FEA430318BF83F4815304F108
:100D0000FF3418BF83F0010314F0FF049BB2EFD14E
:100D10000132192AE5D100F1190200F11A050A443D
:100D20000D44167E2A7E02EB062292B29A421ED112
:100D30000F4B93F83950E2B2AA4215D2431C03EB91
:100D40004203DBB2CA1801330B44127E1B7E03EB55
:100D500002239BB24FF4AF6253431B1303F5487356
:100D600021F814300134E6E7012381F83A3070BDF0
:100D7000202A002003788B420BD9074B1A78074BA7
:100D800089001944C86B02B1400800F5777080B241
:100D900070470020704700BF4C120020202A00201E
:100DA00007299DBF034B03EB8101B1F86C000020C4
:100DB000704700BF202A0020034B03EB4101B1F82C
:100DC0008C00C008704700BF202A00200A4BDFEDCE
:100DD0000B7A03EB810191ED2B7AB8EE477AF6EEB0
:100DE000046AE7EE267A82B0FCEEE77ACDED017A6E
:100DF000BDF8040002B07047202A002000005C44C7
:100E0000014B33F81100704724200020024B03EB04
:100E10004101B1F8F4007047202A0020024B03EB97
:100E20004101B1F8F4007047202A002000207047EB
:100E300070B5334C0546FAF71BF8D4F80C31C4F8FA
:100E40000C01C31AB3F5FA5FC4F8103182BF002356
:100E500084F8143184F8153194F814312BB9A12D8C
:100E600002BF274A012182F8151194F81511244A6E
:100E700029B1D118EDB201330D7682F8143194F80E
:100E8000145194F81631AB4239D11D4B93F81731F8
:100E9000052B02D0062B03D02CE00020FFF71EFF0D
:100EA000637E1E2B26D100200246C1B26B1E9942E2
:100EB00019DA21440B7E0821DBB283EA0206F60729
:100EC00044BF83F01803C3F3460301F1FF3154BF5D
:100ED0005B0843F0800311F0FF01C2F34702ECD13D
:100EE00001301A46E1E723441B7E9A4202D10320D7
:100EF000FFF7F4FE002384F8153184F8143170BD37
:100F0000202A002010B50446F9F7B2FF0F4BD3F8A2
:100F10001821C3F81801821A41F288318A42C3F8B5
:100F20001C2184BF002283F8202193F82021074947
:100F300013440F2AE4B218BF013283F8214112BFD3
:100F400081F82021012381F8313110BD202A0020B1
:100F500010B50446F9F78CFF0F4BD3F83421C3F8D2
:100F60003401821A41F288318A42C3F8382184BFA1
:100F7000002283F83C2193F83C2107491344142AAA
:100F800018BF013283F83D4112BF81F83C21012393
:100F900081F8523110BD00BF202A002038B5044628
:100FA000F9F766FF274A2749D2F85431C2F85401AD
:100FB000C31AB3F57A6F84BF002382F8583192F8D0
:100FC000583133B9A82C3BD181F85931A1F85A31A5
:100FD00006E0022B02D181F85C4101E0242B02D80B
:100FE000D11881F85D4192F85C11164D0133023140
:100FF000DBB249008B4282F8583118DAB5F85A3121
:10100000E0B283EA0020082310F4004F4FEA4000CA
:1010100018BF80F4815003F1FF3318BF80F0010046
:1010200013F0FF0380B2EFD1A2F85A0138BD0131AD
:101030008B4201BF002385F85831012385F85931CF
:1010400038BD00BF202A002010B50446F9F710FF74
:10105000104AD2F8843140F6AC51C31A8B42C4BF57
:10106000002382F8883192F88831D11881F88941BB
:1010700023B90F2C0DD10749C1F884010133DBB22C
:10108000192B044982F888310CBF0123002381F811
:10109000A23110BD202A0020094B1A68137844F6AB
:1010A000FB7103EB431300FB03135078C0EB0030DC
:1010B000B3FBF0F39078B3FBF0F080B2704700BF61
:1010C000BC100020114BD3F8A43103EB4002117E79
:1010D00001290DD002290FD0022805D9032807D1F4
:1010E0000B4A1268D20401D5D8897047988A704794
:1010F000084B33F810007047507E00EB800000EB87
:10110000800000F2EE2080B2704700BF202A00204D
:10111000E81F002024200020044B1B6842F201023B
:101120001A420CBF01200020704700BFE81F0020BA
:10113000114B93F8A821012A10B51C460ED008D3F4
:10114000022A0FD10D4A938A9BB283F4885393826B
:1011500008E00A4B4FF488521A8503E0074B4FF41E
:1011600088529A61F9F784FE00F5F42000F590703A
:10117000C4F8AC0110BD00BF202A002000100048B8
:10118000022803D0431E584258417047064B1B6843
:101190001B7823B1054B1868C0F3C0407047044B5F
:1011A0001878C0F3800070475C060020E40F002030
:1011B000FD2B002010B50A4C5E280146206805D1A1
:1011C0005D21FAF775F820683E2105E05D2903D11D
:1011D000FAF76EF820683D21BDE81040FAF768B8CC
:1011E000D02B002030B50028104C114AB8BF404227
:1011F0003C2590FBF2F304FB030068430D4D90FB8C
:10120000F2F22D682D7B25B903EB830303EB8303F7
:1012100001E0C3EB031302EB83030B8004FB020228
:101220004FF47A7392FBF3F24A8030BD806967FF16
:1012300080969800C410002010B50446C0B2FFF795
:10124000B9FFC4F30720BDE81040B3E7024B5E21AD
:101250001868FAF72DB800BFD02B002038B5064C1F
:1012600005465E212068FAF723F820682946BDE884
:101270003840FAF71DB800BFD02B0020674B73B57C
:101280001878674DFFF77CFF2B788342044620D007
:10129000C8B1644B1B68E3B193F9000002230093CB
:1012A000614B1B685B78003318BF01230193042155
:1012B0004FF416530022F9F70CFE5C4B186040B156
:1012C00001232B7005E0594E3068F7F7D0FC3460ED
:1012D0002C70574B574D1878FFF752FF2B788342ED
:1012E000044618D088B1544B1B68A3B100220124D6
:1012F00093F9000000944FF4964301920821F9F706
:10130000E8FD4E4B186028B905E04C4E3068F7F701
:10131000AEFC34602C704A4B4A4D1878FFF730FF12
:101320002B78834204462E4642D0002837D0464BC5
:101330001A68002A3CD0D37992F90000434C002B64
:1013400008BF022302220092002254F823300192A7
:101350001021F9F7BEFD3E4B0546186040B33D4CE9
:1013600094F84A30022B0BD094F89620022A01D12F
:101370004C3405E023B1002A04F14C0418BF0024CA
:10138000354B1C6044B1204600214C2203F085F807
:101390000223256084F84A300123337008E02C4E84
:1013A0003068FDF773FC3068F7F761FC34602C702F
:1013B0002A4B2B4D1878FFF7E3FE2B788342044627
:1013C00029D000B3274B1B682BB3274A93F90000A1
:1013D00012685278002A0CBF0822092203230093C6
:1013E00001924FF4614320210022F9F772FD1F4B57
:1013F000186080B11E4A012313702B701D4B1A68B0
:101400001D4B1A6007E0194E3068F7F730FC184B97
:1014100034601C702C7002B070BD00BF64060020E8
:10142000A010002060060020C4100020D02B002057
:1014300065060020E41000206811002058110020EB
:10144000700600206E1100206C060020F063010879
:1014500070110020AC110020741100207C060020C7
:1014600084110020780600207406002088110020D6
:101470008C1100200C2000209011002008B5044B96
:101480001B7803F00503052B01D1FAF771F8FEE78D
:10149000D42B0020D0400B1C1141203A03D49C4691
:1014A000134118436346524293401843704700BFAC
:1014B0007BB972B90029BEBF00204FF0004106E0A1
:1014C00008BF00281CBF6FF000414FF0FF3000F054
:1014D00073B882B0EC462DE9005000F03DF8DDF81D
:1014E00004E002B00CBC704707EE900AF5EEC07A3B
:1014F000F1EE10FA01D400F009B808B580F0004010
:1015000000F004F8404261EB410108BDD0B500F0A5
:10151000B9F900220E4B06460F4600F007FA00F01C
:1015200017FC044600F08CF900220A4B00F0FEF98B
:1015300002460B463046394600F044F800F008FCFD
:101540002346002242EA000210461946D0BD00BFE1
:101550000000F03D0000F0412DE9F041069C1546E9
:1015600006460F46984600F013FC05FB01F300FB0E
:101570000838A5FB0023B21A434467EB0303C4E910
:101580000023BDE8F08100BF2DE9F041069C9046A4
:1015900006460F461D4600F049FD00FB05F5A0FB81
:1015A000082308FB0155B21A2B4467EB0303C4E977
:1015B0000023BDE8F08100BF704700BF81F000410B
:1015C00002E000BF83F0004330B54FEA41044FEA28
:1015D000430594EA050F08BF90EA020F1FBF54EAC3
:1015E000000C55EA020C7FEA645C7FEA655C00F05F
:1015F000E2804FEA5454D4EB5555B8BF6D420CDD30
:101600002C4480EA020281EA030382EA000083EAB2
:10161000010180EA020281EA0303362D88BF30BD52
:1016200011F0004F4FEA01314FF4801C4CEA1131A8
:1016300002D0404261EB410113F0004F4FEA033307
:101640004CEA133302D0524263EB430394EA050F92
:1016500000F0A780A4F10104D5F1200E0DDB02FA01
:101660000EFC22FA05F2801841F1000103FA0EF295
:10167000801843FA05F359410EE0A5F120050EF15B
:10168000200E012A03FA0EFC28BF4CF0020C43FA8C
:1016900005F3C01851EBE37101F0004507D54FF099
:1016A000000EDCF1000C7EEB00006EEB0101B1F5E9
:1016B000801F1BD3B1F5001F0CD349085FEA30002F
:1016C0004FEA3C0C04F101044FEA445212F5800F3A
:1016D00080F09A80BCF1004F08BF5FEA500C50F1D7
:1016E000000041EB045141EA050130BD5FEA4C0CBA
:1016F000404141EB010111F4801FA4F10104E9D143
:1017000091F0000F04BF01460020B1FA81F308BF39
:101710002033A3F10B03B3F120020CDA0C3208DD05
:1017200002F1140CC2F10C0201FA0CF021FA02F1E0
:101730000CE002F11402D8BFC2F1200C01FA02F150
:1017400020FA0CFCDCBF41EA0C019040E41AA2BF75
:1017500001EB0451294330BD6FEA04041F3C1CDA3D
:101760000C340EDC04F11404C4F1200220FA04F05D
:1017700001FA02F340EA030021FA04F345EA030107
:1017800030BDC4F10C04C4F1200220FA02F001FAC9
:1017900004F340EA0300294630BD21FA04F029464B
:1017A00030BD94F0000F83F4801306BF81F48011E4
:1017B0000134013D4EE77FEA645C18BF7FEA655C57
:1017C00029D094EA050F08BF90EA020F05D054EA29
:1017D000000C04BF1946104630BD91EA030F1EBF2E
:1017E0000021002030BD5FEA545C05D14000494132
:1017F00028BF41F0004130BD14F580043CBF01F525
:10180000801130BD01F0004545F0FE4141F470010A
:101810004FF0000030BD7FEA645C1ABF19461046E5
:101820007FEA655C1CBF0B46024650EA013406BFE6
:1018300052EA033591EA030F41F4002130BD00BFA5
:1018400090F0000F04BF0021704730B54FF4806462
:1018500004F132044FF000054FF0000150E700BFE3
:1018600090F0000F04BF0021704730B54FF4806442
:1018700004F1320410F0004548BF40424FF000012F
:101880003EE700BF42004FEAE2014FEA31014FEA72
:1018900002701FBF12F07F4393F07F4F81F06051C1
:1018A000704792F0000F14BF93F07F4F704730B530
:1018B0004FF4607401F0004521F0004120E700BFC3
:1018C00050EA010208BF704730B54FF000050AE04A
:1018D00050EA010208BF704730B511F0004502D54B
:1018E000404261EB41014FF4806404F132045FEA4D
:1018F000915C3FF4DCAE4FF003025FEADC0C18BFF2
:1019000003325FEADC0C18BF033202EBDC02C2F1E7
:10191000200300FA03FC20FA02F001FA03FE40EA79
:101920000E0021FA02F11444C1E600BF70B54FF079
:10193000FF0C4CF4E06C1CEA11541DBF1CEA13555B
:1019400094EA0C0F95EA0C0F00F0DEF82C4481EAC3
:10195000030621EA4C5123EA4C5350EA013518BFE3
:1019600052EA033541F4801143F4801338D0A0FBD0
:1019700002CE4FF00005E1FB02E506F00042E0FB7D
:1019800003E54FF00006E1FB03569CF0000F18BF83
:101990004EF0010EA4F1FF04B6F5007F64F540742B
:1019A00004D25FEA4E0E6D4146EB060642EAC621BE
:1019B00041EA55514FEAC52040EA5E504FEACE2E2B
:1019C000B4F1FD0C88BFBCF5E06F1ED8BEF1004F2E
:1019D00008BF5FEA500E50F1000041EB045170BDAA
:1019E00006F0004646EA010140EA020081EA0301EE
:1019F000B4EB5C04C2BFD4EB0C0541EA045170BDEA
:101A000041F480114FF0000E013C00F3AB8014F163
:101A1000360FDEBF002001F0004170BDC4F10004AC
:101A2000203C35DA0C341BDC04F11404C4F120052D
:101A300000FA05F320FA04F001FA05F240EA020088
:101A400001F0004221F0004110EBD37021FA04F6BE
:101A500042EB06015EEA430E08BF20EAD37070BD78
:101A6000C4F10C04C4F1200500FA04F320FA05F0D7
:101A700001FA04F240EA020001F0004110EBD370D9
:101A800041F100015EEA430E08BF20EAD37070BD49
:101A9000C4F1200500FA05F24EEA020E20FA04F322
:101AA00001FA05F243EA020321FA04F001F00041D1
:101AB00021FA04F220EA020000EBD3705EEA430E42
:101AC00008BF20EAD37070BD94F0000F0FD101F071
:101AD0000046400041EB010111F4801F08BF013CAA
:101AE000F7D041EA060195F0000F18BF704703F0E8
:101AF0000046520043EB030313F4801F08BF013D6F
:101B0000F7D043EA0603704794EA0C0F0CEA13552A
:101B100018BF95EA0C0F0CD050EA410618BF52EAE4
:101B20004306D1D181EA030101F000414FF00000EA
:101B300070BD50EA410606BF1046194652EA4306F8
:101B400019D094EA0C0F02D150EA013613D195EA6C
:101B50000C0F05D152EA03361CBF104619460AD1B4
:101B600081EA030101F0004141F0FE4141F47001BE
:101B70004FF0000070BD41F0FE4141F4780170BDAE
:101B800070B54FF0FF0C4CF4E06C1CEA11541DBF13
:101B90001CEA135594EA0C0F95EA0C0F00F0A7F815
:101BA000A4EB050481EA030E52EA03354FEA013142
:101BB00000F088804FEA03334FF0805545EA131355
:101BC00043EA12634FEA022245EA111545EA10651D
:101BD0004FEA00260EF000419D4208BF964244F1B4
:101BE000FD0404F5407402D25B084FEA3202B61AD3
:101BF00065EB03055B084FEA32024FF480104FF4A7
